:020000040800F2
:10600000005000201962000885710108897101089B
:106010008D7101089171010895710108000000005F
:10602000000000000000000000000000997101085D
:106030009D71010800000000A1710108A57101080F
:106040004562000845620008456200084562000894
:106050004562000845620008456200084562000884
:106060004562000845620008456200084562000874
:106070004562000845620008456200084562000864
:106080004562000845620008456200084562000854
:106090004562000845620008456200084562000844
:1060A0004562000845620008456200084562000834
:1060B000E1100108456200084562000845620008D9
:1060C0004562000845620008456200084562000814
:1060D0004562000825120108711501084562000893
:1060E00045620008456200084562000800000000A3
:1060F00000000000000000000000000000000000A0
:1061000000000000000000005FF808F100B583B057
:10611000304B314A1360314A1360314B3149002210
:1061200001E01A6004338B42FBD32B4B1B6813B97D
:106130002A4B1B6803B1FEE7264B2B4A13602B4A00
:1061400013602B4B2B4A2C4803E011681960043371
:1061500004328342F9D3244B1A68284B9A4204D163
:10616000224B1A681B689A4200D0FEE702F0E0FB5F
:1061700001A8694602F05CFB214B224EF61AB610CC
:1061800000241D4603E055F8243098470134A64208
:10619000F9DC1D4B1D4EF61AB61000241D4603E017
:1061A00055F8243098470134A642F9DC019800994B
:1061B00010F0E6FE0546164B164CE41AA4101E46D7
:1061C00003E0013C56F824309847002CF9DC2846BF
:1061D00002F000FBBABADECA8C020020684500203B
:1061E0008C0200206C450020000000208802002066
:1061F0000000002010B801088C02002078563412EC
:1062000048620008486200084862000848620008C6
:10621000486200084862000808B5FFF777FF00BF32
:10622000FEE700BFFEE700BFFEE700BFFEE700BFDE
:10623000FEE700BFFEE700BFFEE700BFFEE700BFCE
:08624000FEE700BFFEE700BF0E
:1062480010B50446B0F5E06F0FD0B0F5C06F0CD0B4
:10625800B0F5A06F09D0B0F5806F06D0B0F5407FDB
:1062680003D00548632102F007FB44F0BF6444F4FF
:106278000034024BDC6010BDE487010800ED00E04B
:1062880010B50446C378012B03D92048752102F0C4
:10629800F3FA63780F2B03D91C48762102F0ECFA45
:1062A800A3780F2B03D91948772102F0E5FAE37890
:1062B80003B3174BDB68DB43C3F30223C3F10402C8
:1062C8000F2121FA03F3617801FA02F2A17819404B
:1062D800114309012278C9B20E4B1A4482F80013FF
:1062E8002278510902F01F02012000FA02F243F855
:1062F800212010BD2378590903F01F03012202FA57
:1063080003F32031034A42F8213010BDE487010825
:1063180000ED00E000E100E038B504460D46B0F1BC
:10632800005F06D0B0F1006F03D00948AA2102F03F
:10633800A3FA084B9D4203D90548AB2102F09CFA09
:1063480025F0604121F07F012143034B996038BD5E
:10635800E4870108FEFF0F0000ED00E010B50446D9
:10636800042806D010F1050F03D00748D52102F004
:1063780083FA042C054B1A680CBF42F0040222F081
:1063880004021A6010BD00BFE487010810E000E0B5
:1063980038B505460C464D4B98420BD003F5806343
:1063A800984207D003F5A053984203D04848E52106
:1063B80002F062FA2368F3B1B3F5803F1BD0B3F55E
:1063C800003F18D0B3F5403F15D0B3F5802F12D059
:1063D800B3F5A02F0FD0B3F5C02F0CD0B3F5E02F35
:1063E80009D0B3F5002F06D0B3F5102F03D03848E5
:1063F800E62102F041FA2379012B03D93448E72139
:1064080002F03AFA6379012B03D93148E82102F006
:1064180033FAA36843B3B3F5003F25D0B3F5802F13
:1064280022D0B3F5C02F1FD0B3F5002F1CD0B3F581
:10643800202F19D0B3F5402F16D0B3F5602F13D005
:1064480093B1B3F5003F0FD0B3F5C02F0CD0B3F51F
:10645800002F09D0B3F5202F06D0B3F5402F03D075
:106468001B48E92102F008FAE36833B1B3F5006F7D
:1064780003D01748EA2102F0FFF9237C013BDBB285
:106488000F2B03D91248EB2102F0F6F96B6823F4BD
:10649800702323F480732268217942EA012213438E
:1064A8006B60AA680B4B1340E168A2680A436179E4
:1064B80042EA41021343AB60EA6A22F47002237C89
:1064C800013BDBB242EA0353EB6238BD00240140D2
:1064D8000C880108FDF7F1FF38B504460D46114B4D
:1064E80098420CD003F58063984208D003F5A05376
:1064F800984204D00C484FF49A7102F0BDF9012D6E
:1065080004D9094840F2351102F0B6F925B1A3685B
:1065180043F00103A36038BDA36823F00103A3601F
:1065280038BD00BF002401400C88010838B5044676
:106538000D460F4B984208D003F5C053984204D03B
:106548000C4840F24D1102F097F9012D04D9094881
:106558004FF4A77102F090F925B1A36843F4807352
:10656800A36038BDA36823F48073A36038BD00BF5F
:10657800002401400C88010810B504460A4B9842D3
:106588000CD003F58063984208D003F5A0539842D5
:1065980004D006484FF4C27102F06EF9A36843F0C4
:1065A8000803A36010BD00BF002401400C88010847
:1065B80010B504460B4B98420CD003F58063984203
:1065C80008D003F5A053984204D007484FF4C97186
:1065D80002F052F9A06800F00800003018BF01204E
:1065E80010BD00BF002401400C88010810B5044606
:1065F8000A4B98420CD003F58063984208D003F503
:10660800A053984204D006484FF4D57102F034F9EB
:10661800A36843F00403A36010BD00BF0024014039
:106628000C88010810B504460B4B98420CD003F5B2
:106638008063984208D003F5A053984204D00748D5
:106648004FF4DC7102F018F9A06800F00400003083
:1066580018BF012010BD00BF002401400C880108AC
:1066680038B504460D46114B98420CD003F58063AB
:10667800984208D003F5A053984204D00C484FF430
:10668800E97102F0F9F8012D04D9094840F2D31153
:1066980002F0F2F825B1A36843F4A003A36038BD63
:1066A800A36823F4A003A36038BD00BF0024014001
:1066B8000C880108F8B504460D4616461F46374BA8
:1066C80098420CD003F58063984208D003F5A05394
:1066D800984204D032484FF4167102F0CDF8112DCB
:1066E80004D92F4840F2592102F0C6F8731EDBB2D4
:1066F8000F2B04D92A4840F25A2102F0BDF8072F7F
:1067080004D9274840F25B2102F0B6F8092D0DD9CB
:10671800E168A5F10A0303EB430307229A4021EA43
:1067280002029F4042EA0703E3600AE0216905EBA1
:10673800450307229A4021EA02029F4042EA0703E2
:106748002361062E0CD8626B013E06EB86061F23DA
:10675800B34022EA0303B54043EA05066663F8BD81
:106768000C2E0DD8226B073E06EB86061F23B3407E
:1067780022EA030305FA06F643EA06052563F8BD8F
:10678800E26A0D3E06EB86061F23B34022EA0303A6
:10679800B54043EA0506E662F8BD00BF00240140A3
:1067A8000C88010810B504464F4B984225D0143385
:1067B800984222D0143398421FD0143398421CD0E8
:1067C8001433984219D01433984216D0143398428F
:1067D80013D003F5627398420FD0143398420CD04B
:1067E8001433984209D01433984206D0143398428F
:1067F80003D03E486F2102F03FF8236823F00103DD
:106808001B041B0C2360002323606360A360E36008
:10681800354B9C4205D1083B5A6842F00F025A603A
:1068280010BD334B9C4205D11C3B5A6842F0F00224
:106838005A6010BD2F4B9C4205D1303B5A6842F438
:1068480070625A6010BD2C4B9C4205D1443B5A687B
:1068580042F470425A6010BD284B9C4205D1583B07
:106868005A6842F470225A6010BD254B9C4205D1EB
:106878006C3B5A6842F470025A6010BD214B9C422E
:1068880005D1803B5A6842F070625A6010BD1E4BB9
:106898009C4205D1083B5A6842F00F025A6010BD6D
:1068A8001A4B9C4205D11C3B5A6842F0F0025A60D0
:1068B80010BD174B9C4205D1303B5A6842F47062B8
:1068C8005A6010BD134B9C4205D1443B5A6842F4B0
:1068D80070425A6010BD104B9C4204D1583B5A6814
:1068E80042F470225A6010BD080002403C8801083A
:1068F8001C000240300002404400024058000240A0
:106908006C00024080000240080402401C0402405F
:1069180030040240440402405804024038B5054699
:106928000C46504B984225D01433984222D0143349
:1069380098421FD0143398421CD01433984219D06F
:106948001433984216D01433984213D003F5627367
:1069580098420FD0143398420CD01433984209D07F
:106968001433984206D01433984203D03E48CF21BE
:1069780001F082FFA368102B04D01BB13A48D02144
:1069880001F07AFFE368013B4FF6FE72934203D9A8
:106998003548D12101F070FF2369402B04D01BB189
:1069A8003148D22101F068FF6369802B04D01BB104
:1069B8002D48D32101F060FFA3694BB1B3F5807F67
:1069C80006D0B3F5007F03D02748D42101F054FF47
:1069D800E3694BB1B3F5806F06D0B3F5006F03D010
:1069E8002148D52101F048FF236A202B04D01BB190
:1069F8001D48D62101F040FF636AB3F5405F0AD015
:106A0800B3F5005F07D0B3F5805F04D01BB116481B
:106A1800D72101F031FFA36AB3F5804F04D01BB131
:106A28001148D82101F028FF2B6823F4FF4323F0F5
:106A38007003A168226A11432269114362691143F4
:106A4800A2691143E2691143626A1143A26A0A43C7
:106A580013432B60E3686B602368AB606368EB608B
:106A680038BD00BF080002403C88010838B504461C
:106A78000D461F4B984226D01433984223D0143326
:106A8800984220D0143398421DD0143398421AD01B
:106A98001433984217D01433984214D003F5627314
:106AA800984210D0143398420DD0143398420AD02B
:106AB8001433984207D01433984204D00D4840F25A
:106AC800291101F0D9FE012D04D90A484FF4957116
:106AD80001F0D2FE25B1236843F00103236038BDDD
:106AE800236823F001031B041B0C236038BD00BF7F
:106AF800080002403C88010810B50446431E012BDB
:106B080040F29B80042800F09880082800F09580C7
:106B1800102800F09280202800F08F80402800F094
:106B28008C80802800F08980B0F5807F00F0858017
:106B3800B0F5007F00F08180B0F5806F7DD0B0F5B2
:106B4800006F7AD0B0F5805F77D0B0F5005F74D071
:106B5800B0F5804F71D0B0F5004F6ED0B0F5803FE2
:106B68006BD0B0F5003F68D0B0F5802F65D0B0F598
:106B7800002F62D0B0F5801F5FD0B0F5001F5CD049
:106B8800B0F5800F59D0B0F5000F56D0B0F1807F26
:106B980053D0B0F1007F50D0B0F1806F4DD0B0F13C
:106BA800006F4AD02B4B984247D00133984244D0CB
:106BB8000233984241D0043398423ED00833984279
:106BC8003BD01033984238D02033984235D04033E8
:106BD800984232D0803398422FD003F58073984280
:106BE8002BD003F50073984227D003F580639842B1
:106BF80023D0B0F1102F20D003F5C05398421CD0F9
:106C080003F50053984218D003F58043984214D0F6
:106C180003F50043984210D003F5803398420CD016
:106C280003F50033984208D003F58023984204D036
:106C3800094840F2B71101F01FFE14F0805F14BF3D
:106C4800064B074B1B6803EA0400003018BF0120FD
:106C580010BD00BF010000103C880108000402407C
:106C68000000024010B50446022804D9054840F245
:106C7800031101F001FE044B1A6802F038021443B4
:106C88001C6010BD6C8801080020024010B5044645
:106C9800102805D020B1074840F22F1101F0ECFD73
:106CA800054B1A6822F010021A601A6814431C6017
:106CB80010BD00BF6C88010800200240034B044A45
:106CC8005A6002F188325A60704700BF00200240C3
:106CD80023016745024B1A6942F080021A61704726
:106CE8000020024010B5044630F0350300D120B929
:106CF800034840F2CC5101F0BFFD024BDC6010BDEF
:106D08006C880108002002400B4BDB6813F0010F70
:106D18000DD1094BDB6813F0040F0AD1064BDB6871
:106D280003F01003002B0CBF042003207047012040
:106D380070470220704700BF0020024010B504468B
:106D4800FFF7E2FF02E0FFF7DFFF013C012801D176
:106D5800002CF8D1002C08BF052010BD38B504461A
:106D680000F17842114B9A4204D9114840F2A71118
:106D780001F082FD4FF43020FFF7E0FF042813D123
:106D88000C4D2B6943F002032B616C612B6943F0B6
:106D980040032B614FF43020FFF7D0FF2B6923F01D
:106DA8000203DB04DB0C2B6138BD00BFFEFF0F00C4
:106DB8006C8801080020024030B583B004460D46B7
:106DC8000023019300F178421A4B9A4204D91A48D9
:106DD80040F2B52101F050FD4FF40050FFF7AEFF2F
:106DE800042824D1154B1A6942F001021A61ABB28A
:106DF80023804FF40050FFF7A1FF042810D102347C
:106E08000194019B2D0C1D804FF40050FFF796FF55
:106E18000A4B1A6922F00102D204D20C1A6106E068
:106E2800064B1A6922F00102D204D20C1A6103B08F
:106E380030BD00BFFEFF0F006C8801080020024033
:106E48002DE9F04105460C46494B98421BD003F505
:106E58008063984217D003F58063984213D003F5F6
:106E6800806398420FD003F5806398420BD003F5F6
:106E78008063984207D003F58063984203D03D4869
:106E8800B22101F0F9FCE3788BB1042B0FD0282B49
:106E98000DD0482B0BD0142B09D0102B07D01C2B4E
:106EA80005D0182B03D03348B32101F0E5FC238823
:106EB8001BB93048B42101F0DFFCE37803F00F0779
:106EC8003E4613F0100F0AD0A378013BDBB2022B29
:106ED80003D92848BB2101F0CFFCA6783E4323788C
:106EE800FBB12F68002301204FF00F0C16E000FAC9
:106EF80003F22188114091420FD199000CFA01F850
:106F080027EA080706FA01F10F43E178282901D199
:106F18006A6102E0482908BF2A610133072BE6D9D4
:106F28002F602388FF2B21D96F68002301204FF0A1
:106F38000F0C18E003F1080200FA02F22188114050
:106F480091420FD199000CFA01F827EA080706FACE
:106F580001F10F43E178282908BF6A61E1784829DF
:106F680008BF2A610133072BE4D96F60BDE8F081BF
:106F780000080140A088010838B504460D462A4B90
:106F880098421CD003F58063984218D003F58063BB
:106F9800984214D003F58063984210D003F58063BB
:106FA80098420CD003F58063984208D003F58063BB
:106FB800984204D01D484FF48F7101F05DFC6B1EA0
:106FC8009BB2012B28D9042D26D0082D24D0102DB2
:106FD80022D0202D20D0402D1ED0802D1CD0B5F5DC
:106FE800807F19D0B5F5007F16D0B5F5806F13D026
:106FF800B5F5006F10D0B5F5805F0DD0B5F5005F21
:107008000AD0B5F5804F07D0B5F5004F04D0074832
:1070180040F21F1101F030FCA36803EA05000030BC
:1070280018BF012038BD00BF00080140A088010832
:1070380038B504460D462A4B98421CD003F58063A8
:10704800984218D003F58063984214D003F5806302
:10705800984210D003F5806398420CD003F5806302
:10706800984208D003F58063984204D01D484FF435
:10707800A27101F001FC6B1E9BB2012B28D9042DD3
:1070880026D0082D24D0102D22D0202D20D0402D00
:107098001ED0802D1CD0B5F5807F19D0B5F5007FA6
:1070A80016D0B5F5806F13D0B5F5006F10D0B5F5D3
:1070B800805F0DD0B5F5005F0AD0B5F5804F07D0D9
:1070C800B5F5004F04D0074840F2451101F0D4FB54
:1070D800E36803EA0500003018BF012038BD00BF8F
:1070E80000080140A088010838B504460D46144B35
:1070F80098421CD003F58063984218D003F580634A
:10710800984214D003F58063984210D003F5806349
:1071180098420CD003F58063984208D003F5806349
:10712800984204D0074840F2691101F0A5FB25B93F
:1071380004484FF4B57101F09FFB256138BD00BFCD
:1071480000080140A088010838B504460D46144BD4
:1071580098421CD003F58063984218D003F58063E9
:10716800984214D003F58063984210D003F58063E9
:1071780098420CD003F58063984208D003F58063E9
:10718800984204D0074840F2791101F075FB25B9FF
:1071980004484FF4BD7101F06FFB656138BD00BF55
:1071A80000080140A088010838B504460D46431E72
:1071B800012B40F29080042800F08D80082800F010
:1071C8008A80624B984200F086802033984200F013
:1071D80082805F4B98427ED0803398427BD05D4B53
:1071E800984278D003F58073984274D003F5807381
:1071F800984270D0584B98426DD003F580639842FE
:1072080069D0B0F5805F66D0B0F5EA1F63D0B0F5FD
:10721800EB1F60D0B0F5004F5DD0504B98425AD06C
:107228000133984257D00233984254D004339842DD
:1072380051D0083398424ED0B0F1201F4BD0303394
:10724800984248D0464B984245D003F580739842FF
:1072580041D003F5007398423DD0424B98423AD052
:1072680003F57063984236D0B0F5011F33D03E4B1A
:10727800984230D0013398422DD0023398422AD018
:107288000433984227D00833984224D010339842C8
:1072980021D0203398421ED0403398421BD08033EF
:1072A800984218D003F58073984214D003F5007300
:1072B800984210D003F5806398420CD003F5006320
:1072C800984208D003F58053984204D0274840F2EA
:1072D8002A2101F0D1FA012D04D9244840F22B21AA
:1072E80001F0CAFA002C224BB4BFDB695B68C4F317
:1072F8000340A1B204F44012B2F5401F07D123F0B5
:1073080070631B4A506820F07060506012E014F4FB
:10731800801F07D0032202FA00F023EA000343F09B
:10732800706307E0620D120101FA02F223EA020318
:1073380043F070631DB1620D120191400B43002CA4
:107348000B4AB4BFD361536038BD00BF10001400AE
:10735800400016000001180000081A000100200073
:10736800000130000011200001000080A088010801
:107378000000014010B5044645F25553984204D028
:1073880018B103485F2101F077FA024B1C6010BD69
:10739800D48801080030004010B50446062803D9F7
:1073A8000348732101F068FA024B5C6010BD00BF0E
:1073B800D48801080030004010B50446B0F5805F5D
:1073C80003D30348802101F057FA024B9C6010BD9B
:1073D800D4880108003000404AF6AA22014B1A60FE
:1073E800704700BF003000404CF6CC42014B1A6099
:1073F800704700BF003000400D4B1A6842F0010290
:107408001A6059680B4A0A405A601A6822F0847256
:1074180022F480321A601A6822F480221A605A68AC
:1074280022F4FE025A604FF41F029A60704700BFB0
:10743800001002400000FFF810B5044650B1B0F546
:10744800803F07D0B0F5802F04D0104840F21111CA
:1074580001F012FA0E4B1A6822F480321A601A6888
:1074680022F480221A60B4F5803F03D0B4F5802F4F
:1074780006D010BD064B1A6842F480321A6010BD5F
:10748800034B1A6842F4A0221A6010BD088901084B
:107498000010024038B50C46054650B1B0F5803FA3
:1074A80007D0B0F5403F04D01E4840F27F1101F0EC
:1074B800E3F974B3B4F5802F2BD0B4F5002F28D09E
:1074C800B4F5402F25D0B4F5801F22D0B4F5A01F05
:1074D8001FD0B4F5C01F1CD0B4F5E01F19D0B4F507
:1074E800001F16D0B4F5101F13D0B4F5201F10D00C
:1074F800B4F5301F0DD0B4F5401F0AD0B4F5501FB5
:1075080007D0B4F5601F04D006484FF4C07101F0ED
:10751800B3F9054B5A6822F47C122C4314435C607F
:1075280038BD00BF088901080010024010B50446A4
:10753800012804D903484FF4CA7101F09DF9024BA0
:107548001C6010BD088901086000424210B504465D
:10755800022804D905484FF40E7101F08DF9044B47
:107568005A6822F0030214435C6010BD08890108C0
:1075780000100240024B586800F00C00704700BF32
:107588000010024010B50446A0B1802812D09028FF
:1075980010D0A0280ED0B0280CD0C0280AD0D028EF
:1075A80008D0E02806D0F02804D006484FF4197116
:1075B80001F062F9044B5A6822F0F00214435C604F
:1075C80010BD00BF088901080010024010B504462C
:1075D80080B1B0F5806F0DD0B0F5A06F0AD0B0F5CE
:1075E800C06F07D0B0F5E06F04D0064840F27E21A6
:1075F80001F042F9044B5A6822F4E06214435C60DB
:1076080010BD00BF088901080010024010B50446EB
:1076180080B1B0F5806F0DD0B0F5A06F0AD0B0F58D
:10762800C06F07D0B0F5E06F04D006484FF426715C
:1076380001F022F9044B5A6822F4605242EAC40469
:107648005C6010BD088901080010024010B4284B86
:107658005B6803F00C03042B05D0082B06D0F3B9A4
:10766800244B03601DE0244B03601AE0204B5A684A
:107678005B68C2F38342023213F4803F04D11F4B8C
:1076880003FB02F202600CE0194B5B6813F4003F45
:1076980014BF1B4B184B03FB02F2026001E0154BB1
:1076A8000360134B5A68C2F3031216498A5CD2B2BC
:1076B800046824FA02F242605C68C4F302240C5D98
:1076C800E4B222FA04F484605C68C4F3C224095D5D
:1076D800C9B2CA40C2605B68C3F381330A49CB5C54
:1076E800DBB2B2FBF3F202615DF8044B704700BFF6
:1076F8000010024000127A00001BB70000093D008C
:10770800808D5B00080000200400002038B5044686
:107718000D4620F4AA6323F0070303B920B90C48E7
:1077280040F22B4101F0A8F8012D04D9084840F295
:107738002C4101F0A1F825B1064B5A6914435C614C
:1077480038BD044B5A6922EA04045C6138BD00BFA5
:10775800088901080010024038B504460D460E4B52
:10776800034003B920B90D4840F24A4101F084F8BA
:10777800012D04D9094840F24B4101F07DF825B1AB
:10778800074B9A6914439C6138BD054B9A6922EAF4
:1077980004049C6138BD00BF0200C0FF08890108CD
:1077A8000010024038B504460D460E4B184200D171
:1077B80020B90D4840F2694101F05EF8012D04D965
:1077C800094840F26A4101F057F825B1074BDA69D8
:1077D8001443DC6138BD054BDA6922EA0404DC6134
:1077E80038BD00BF00360181088901080010024039
:1077F80010B50446212818D0312816D0392814D0BD
:10780800412812D0612810D07A280ED07B280CD0BD
:107818007C280AD07D2808D07E2806D07F2804D06E
:107828000A4840F2345101F027F86309012B02D1CC
:10783800074B186804E0022B054B0CBF186A586AFE
:1078480004F01F04E04000F0010010BD08890108A1
:107858000010024010B582B0002301933124204665
:10786800FFF7C6FF019B01330193019BB3F5A06F9E
:1078780001D00028F3D03120FFF7BAFF003018BF3D
:10788800012002B010BD00BF024B5A6A42F080725C
:107898005A627047001002402DE9F84305460C462D
:1078A800464B98420BD0A3F57843984207D003F58E
:1078B8008063984203D04248A32100F0DDFF23886B
:1078C80063B1B3F5806F09D0B3F5004F06D0B3F5B7
:1078D800404F03D03A48A62100F0CEFF6388B3F5A5
:1078E800827F04D01BB13648A72100F0C5FFA388CA
:1078F800B3F5006F04D01BB13148A82100F0BCFFDC
:10790800E3882BB1022B03D02D48A92100F0B4FF46
:107918002389012B03D92A48AA2100F0ADFF6389E6
:10792800B3F5007F04D01BB12548AB2100F0A4FFBC
:10793800A3898BB1082B0FD0102B0DD0182B0BD08F
:10794800202B09D0282B07D0302B05D0382B03D07B
:107958001B48AC2100F090FFE3892BB1802B03D0AA
:107968001748AD2100F088FF238A1BB91448AE21BF
:1079780000F082FF2A8802F44152B4F8009063882C
:10798800B4F80480B4F806C027896689A089E1891B
:1079980049EA030348EA03034CEA03033B4333433E
:1079A80003430B4313432B80AB8B23F400631B046B
:1079B8001B0CAB83238A2B82BDE8F883003001407F
:1079C8003889010838B504460D46124B98420CD048
:1079D800A3F57843984208D003F58063984204D011
:1079E8000D4840F2B71100F047FF012D04D90A48AD
:1079F8004FF4DC7100F040FF2DB123889BB243F0B7
:107A08004003238038BD238823F040031B041B0C4C
:107A1800238038BD003001403889010870B504461C
:107A28000D461646164B98420CD0A3F5784398425B
:107A380008D003F58063984204D012484FF40871C7
:107A480000F01AFF012E04D90E4840F2212100F05F
:107A580013FF25F003039BB203B925B9094840F287
:107A6800222100F009FF26B1A3889BB21D43A580FF
:107A780070BDA388ED43ADB21D40A58070BD00BFA9
:107A8800003001403889010838B504460D46094BD5
:107A980098420CD0A3F57843984208D003F5806348
:107AA800984204D0044840F23A2100F0E5FEA5814E
:107AB80038BD00BF003001403889010810B50446C0
:107AC800094B98420CD0A3F57843984208D003F5A7
:107AD8008063984204D0054840F24A2100F0CCFE69
:107AE800A08980B210BD00BF00300140388901086C
:107AF80038B505460C46164B98420CD0A3F578438A
:107B0800984208D003F58063984204D0114840F2A7
:107B1800163100F0B1FE802C12D0402C10D0202C51
:107B28000ED0102C0CD0082C0AD0042C08D0022C13
:107B380006D0012C04D0074840F2173100F09CFE13
:107B48002B8904EA0300003018BF012038BD00BFAC
:107B5800003001403889010838B504460D46524BBB
:107B6800984242D0B0F1804F3FD0A3F59433984269
:107B78003BD003F58063984237D003F58063984281
:107B880033D003F5806398422FD003F58063984281
:107B98002BD003F59033984227D003F5C053984271
:107BA80023D003F5806398421FD003F58063984281
:107BB8001BD0A3F59E33984217D003F580639842F3
:107BC80013D003F5806398420FD003F590339842A1
:107BD8000BD003F58063984207D003F58063984281
:107BE80003D03248E72100F047FE6B885BB1102BC9
:107BF80009D0202B07D0402B05D0602B03D02B4871
:107C0800E82100F039FEEB884BB1B3F5807F06D050
:107C1800B3F5007F03D02548E92100F02DFE238825
:107C28009BB2214A944212D002F5006294420ED0CF
:107C3800B4F1804F0BD0A2F59832944207D002F5E8
:107C48008062944203D002F58062944203D123F00B
:107C580070036A881343164A944208D002F580627A
:107C6800944204D023F440739BB2EA8813432380E0
:107C7800AB88A3852B8823850B4B9C420FD003F53B
:107C880000639C420BD003F540639C4207D003F588
:107C980080639C4203D003F580639C4201D12B7A18
:107CA80023860123A38238BD002C0140688901087E
:107CB8000010004038B504460D462E4B984243D07C
:107CC800B0F1804F40D0A3F5943398423CD003F5EF
:107CD8008063984238D003F58063984234D003F526
:107CE8008063984230D003F5806398422CD003F526
:107CF8009033984228D003F5C053984224D003F516
:107D08008063984220D003F5806398421CD0A3F585
:107D18009E33984218D003F58063984214D003F537
:107D28008063984210D003F5903398420CD003F545
:107D38008063984208D003F58063984204D00E48C7
:107D480040F2293100F098FD012D04D90A4840F28B
:107D58002A3100F091FD2DB123889BB243F0010335
:107D6800238038BD238823F001031B041B0C2380C8
:107D780038BD00BF002C01406889010870B5044671
:107D88000D461646314B984243D0B0F1804F40D053
:107D9800A3F5943398423CD003F58063984238D0D9
:107DA80003F58063984234D003F58063984230D05D
:107DB80003F5806398422CD003F59033984228D07D
:107DC80003F5C053984224D003F58063984220D02D
:107DD80003F5806398421CD0A3F59E33984218D0CF
:107DE80003F58063984214D003F58063984210D05D
:107DF80003F5903398420CD003F58063984208D07D
:107E080003F58063984204D0114840F26B3100F0CA
:107E180033FD15F47F4F00D125B90D484FF45B7140
:107E280000F02AFD012E04D9094840F26D3100F016
:107E380023FD26B1A3899BB21D43A58170BDA389EB
:107E4800ED43ADB21D40A58170BD00BF002C0140BF
:107E58006889010870B504460E461546284B9842B5
:107E680043D0B0F1804F40D0A3F5943398423CD032
:107E780003F58063984238D003F58063984234D084
:107E880003F58063984230D003F5806398422CD084
:107E980003F59033984228D003F5C053984224D074
:107EA80003F58063984220D003F5806398421CD084
:107EB800A3F59E33984218D003F58063984214D0F6
:107EC80003F58063984210D003F5903398420CD0A4
:107ED80003F58063984208D003F58063984204D084
:107EE800084840F29B4100F0C7FC012D04D9054821
:107EF80040F29C4100F0C0FC2685A58270BD00BF01
:107F0800002C01406889010838B504460D462A4B03
:107F1800984243D0B0F1804F40D0A3F594339842B3
:107F28003CD003F58063984238D003F580639842CB
:107F380034D003F58063984230D003F580639842CB
:107F48002CD003F59033984228D003F5C0539842BB
:107F580024D003F58063984220D003F580639842CB
:107F68001CD0A3F59E33984218D003F5806398423D
:107F780014D003F58063984210D003F590339842EB
:107F88000CD003F58063984208D003F580639842CB
:107F980004D00A4840F6362100F06EFC15F4614F13
:107FA80000D125B9054840F6372100F065FCED43BE
:107FB800ADB2258238BD00BF002C01406889010898
:107FC80038B504460D46334B984243D0B0F1804F44
:107FD80040D0A3F5943398423CD003F5806398428F
:107FE80038D003F58063984234D003F58063984213
:107FF80030D003F5806398422CD003F59033984233
:1080080028D003F5C053984224D003F580639842E2
:1080180020D003F5806398421CD0A3F59E33984284
:1080280018D003F58063984214D003F58063984212
:1080380010D003F5903398420CD003F58063984232
:1080480008D003F58063984204D0134840F65821BD
:1080580000F012FC6B1E9BB2012B10D9042D0ED020
:10806800082D0CD0102D0AD0202D08D0402D06D078
:10807800802D04D0084840F6592100F0FDFB238AE2
:10808800A08928401D4203D0003018BF012038BD08
:10809800002038BD002C01406889010838B5044625
:1080A8000D462A4B984243D0B0F1804F40D0A3F5FB
:1080B800943398423CD003F58063984238D003F556
:1080C8008063984234D003F58063984230D003F53A
:1080D800806398422CD003F59033984228D003F55A
:1080E800C053984224D003F58063984220D003F50A
:1080F800806398421CD0A3F59E33984218D003F5AC
:108108008063984214D003F58063984210D003F539
:10811800903398420CD003F58063984208D003F559
:108128008063984204D00A4840F6822100F0A4FBFC
:1081380015F47F4F00D125B9054840F6832100F09A
:108148009BFBED43ADB2258238BD00BF002C01403A
:108158006889010830B587B004460D46644B9842DB
:1081680013D0A3F5744398420FD003F58063984267
:108178000BD003F58063984207D003F580639842DB
:1081880003D05C48B82100F077FB2B68013B5A4AC2
:10819800934203D95748B92100F06EFBAB8833B13D
:1081A800B3F5805F03D05348BA2100F065FBEB8834
:1081B80063B1B3F5805F09D0B3F5005F06D0B3F5BE
:1081C800405F03D04B48BB2100F056FB2B894BB1D5
:1081D800B3F5806F06D0B3F5C06F03D04548BC2116
:1081E80000F04AFB6B8923F00C0292B202B91BB96A
:1081F8004048BD2100F040FBAB8963B1B3F5807FF7
:1082080009D0B3F5007F06D0B3F5407F03D03948D5
:10821800BE2100F031FBAB8973B1354B9C420BD0CA
:10822800A3F574439C4207D003F580639C4203D0B6
:108238003048C22100F020FB238A23F440531B045A
:108248001B0CEA8813432382A28992B222F4B0520B
:1082580022F00C02A8882B89698903430B43134336
:10826800A381A38A23F440731B041B0CAA8913431C
:10827800A38201A8FFF7EAF91D4B9C420CBF049AA0
:10828800039AA3891BB2002B08DA02EB820202EBE5
:1082980082022B685B00B2FBF3F207E002EB82027A
:1082A80002EB820229688900B2FBF1F2134BA3FBAF
:1082B80002135B091801642103FB1123A18909B288
:1082C800002908DADB0032330C4DA5FB0323C3F386
:1082D8004213034307E01B013233084DA5FB031388
:1082E800C3F3431303439BB2238107B030BD00BFE0
:1082F80000380140988901081FAA44001F85EB51E6
:1083080070B505460C46234B98420CD0A3F5744330
:10831800984208D003F58063984204D01E484FF471
:10832800997100F0A9FA23883BB1B3F5006F04D026
:10833800194840F2331100F09FFA63883BB1B3F556
:10834800806F04D014484FF49A7100F095FAA3880E
:108358003BB1B3F5007F04D00F4840F2351100F06F
:108368008BFAE3883BB1B3F5807F04D00A484FF419
:108378009B7100F081FA2B8A23F470631B041B0C99
:1083880026886288A088E188324302430A4313435F
:108398002B8270BD003801409889010838B5044621
:1083A8000D46164B984214D0A3F57443984210D04A
:1083B80003F5806398420CD003F58063984208D097
:1083C80003F58063984204D00D484FF4B17100F072
:1083D80053FA012D04D90A4840F2631100F04CFA0F
:1083E8002DB1A3899BB243F40053A38138BDA3895F
:1083F80023F400531B041B0CA38138BD0038014033
:108408009889010870B505460C461646364B9842C1
:1084180014D0A3F57443984210D003F580639842B2
:108428000CD003F58063984208D003F58063984226
:1084380004D02E4840F2891100F01EFA282C1ED0D4
:1084480040F227739C421AD040F226639C4216D011
:1084580040F225539C4212D040F224439C420ED055
:1084680040F646039C420AD040F66A139C4206D066
:10847800602C04D01D484FF4C57100F0FDF9012EA1
:1084880004D91A4840F28B1100F0F6F940F66A1345
:108498009C420FD1144B9D420CD0A3F574439D42CE
:1084A80008D003F580639D4204D0104840F28F1134
:1084B80000F0E2F9C4F3421304F01F04012202FAA7
:1084C80004F4934201D10C3503E0022B0CBF1035A4
:1084D80014351EB12B681C432C6070BD2B6823EA31
:1084E80004042C6070BD00BF003801409889010861
:1084F80038B504460D46124B984214D0A3F5744380
:10850800984210D003F5806398420CD003F580633D
:10851800984208D003F58063984204D0094840F295
:108528005F2100F0A9F9B5F5007F04D305484FF4A1
:10853800187100F0A1F9C5F30805A58038BD00BF82
:10854800003801409889010810B504460D4B98423F
:1085580014D0A3F57443984210D003F58063984271
:108568000CD003F58063984208D003F580639842E5
:1085780004D005484FF41C7100F07EF9A088C0F3C0
:10858800080010BD003801409889010838B5054633
:108598000C46264B984214D0A3F57443984210D049
:1085A80003F5806398420CD003F58063984208D0A5
:1085B80003F58063984204D01D4840F2863100F0EC
:1085C8005BF9012C18D0802C16D0402C14D0202C0C
:1085D80012D0102C10D0B4F5807F0DD0B4F5007FE8
:1085E8000AD0082C08D0042C06D0022C04D010483D
:1085F80040F2873100F040F9B4F5007F0FD10B4B02
:108608009D420CD0A3F574439D4208D003F58063C6
:108618009D4204D0064840F28B3100F02DF92B889A
:1086280004EA0300003018BF012038BD00380140BB
:108638009889010838B505460C463A4B984214D03B
:10864800A3F57443984210D003F5806398420CD088
:1086580003F58063984208D003F58063984204D0FC
:10866800314840F2D93100F007F9282C25D040F2E2
:1086780027739C4221D040F226639C421DD040F2D1
:1086880025539C4219D040F224439C4215D040F611
:1086980046039C4211D040F66A139C420DD0B4F5B3
:1086A800587F0AD0B4F5187F07D0B4F5B07F04D04E
:1086B8001D4840F2DA3100F0DFF840F66A139C42B8
:1086C8000FD1184B9D420CD0A3F574439D4208D09E
:1086D80003F580639D4204D0134840F2DE3100F078
:1086E800CBF8C4F3421304F01F0201219140012B7F
:1086F80003D1AA8992B20A4005E0022B0CBF2A8A4C
:10870800AA8A92B20A40240A012000FA04F42888AE
:1087180080B220401AB1003018BF012038BD0020B7
:1087280038BD00BF003801409889010838B50446B3
:108738000D46244B984214D0A3F57443984210D0A8
:1087480003F5806398420CD003F58063984208D003
:1087580003F58063984204D01B4840F2224100F0A0
:108768008BF840F226639D4210D040F225539D427B
:108778000CD040F646039D4208D040F66A139D424D
:1087880004D0114840F2234100F076F840F66A130D
:108798009D420FD10B4B9C420CD0A3F574439C42D5
:1087A80008D003F580639C4204D0074840F2274173
:1087B80000F062F82D0A012303FA05F5ED43ADB286
:1087C800258038BD0038014098890108FEE700BFC0
:1087D80008B5034800F076F80120FFF7F7FF00BF5F
:1087E800CC89010808B50D4B1B6813B90C4A0B4B13
:1087F8001A600A4B1B68033020F003001844094A2A
:10880800904206D90EF0D0FC0C2303604FF0FF30E5
:1088180008BD024A1060184608BD00BF900200203B
:108828006C4500200048002001230360014B0B60C9
:10883800704700BF1800002008B50EF0B5FC58239B
:1088480003604FF0FF3008BD08B50EF0ADFC5823AB
:1088580003604FF0FF3008BD08B50EF0A5FC5823A3
:108868000360002008BD00BF08B50EF09DFC58232A
:1088780003604FF0FF3008BD08B503460A460348B9
:10888800194600F005F8FFF7A3FF00BF208A01088A
:108898000FB400B583B004AB53F8042B0193084818
:1088A80080210FF0CFFB011E03DD054800F038F8EA
:1088B8000146084603B05DF804EB04B0704700BFFA
:1088C8009802002010B504460EF04EFE01462046E0
:1088D80000F026F80248012100F022F810BD00BF80
:1088E800CC92010810B400244FF0604212E0D2F894
:1088F800803E13F0010F04D0D2F8003E13F0010FB0
:1089080001D1204609E01368002BFCD003781370CE
:10891800013401308C42EAD308465DF8044B7047B5
:1089280008B5FFF7DFFF08BD08B500F067F808BD18
:1089380082B000230193009303F1804303F50433CD
:108948001A6842F480321A601A46136803F4003336
:108958000093019B01330193009B1BB9019BB3F565
:10896800A06FF2D1214B1B6813F4003F14BF012301
:1089780000230093009B012B36D11D4B1A6842F04F
:1089880010021A601A6822F003021A601A6842F08C
:1089980002021A60A3F580535A685A605A685A60EE
:1089A8005A6842F480625A605A6822F47C125A600B
:1089B8005A6842F4E8125A601A6842F080721A60E3
:1089C8001A46136813F0007FFBD0084B5A6822F050
:1089D80003025A605A6842F002025A601A46536803
:1089E80003F00C03082BFAD102B0704700100240C4
:1089F8000020024008B5FFF79BFF08BD08B5104BE3
:108A08001A6842F001021A6059680E4A0A405A6010
:108A18001A6822F0847222F480321A601A6822F4EA
:108A280080221A605A6822F4FE025A604FF41F022C
:108A38009A60FFF7DFFF4FF00062034B9A6008BDB2
:108A4800001002400000FFF800ED00E008B54FF408
:108A5800C060FDF7F5FB4FF000604FF4C041FDF733
:108A68005BFC62B608BD00BF08B57D20FEF7C0FEFE
:108A780008B1FEF709FF45F25550FEF77BFC0520CB
:108A8800FEF78AFC40F6FF70FEF796FCFEF7ACFC9A
:108A980008BD00BF10B582B004460C4B53F8200047
:108AA8000121FEF759FE0A4B33F81430ADF80430B3
:108AB80010238DF8073003238DF80630054B53F843
:108AC800240001A9FEF7BCF902B010BD788A01089C
:108AD800888A01082000002008B50346044A52F895
:108AE8002000044A32F81310FEF72EFB08BD00BF21
:108AF80020000020888A010808B50346044A52F875
:108B08002000044A32F81310FEF7EEFA08BD00BF41
:108B180020000020888A010808B50346044A52F854
:108B28002000044A32F81310FEF782FA08BD00BF8D
:108B380020000020888A010882B0019002E0019B91
:108B4800013B0193019B002BF9D102B0704700BF94
:108B580010B586B004460420FDF700FC01A8FEF716
:108B680075FD1048029BA0FB0320800C04FB00F05D
:108B78000138B0F1807F09D20B4B5860F0210B4AC5
:108B880082F8231000229A6007221A60064B1A689E
:108B980022F002021A601A46136813F4803FFBD0D1
:108BA80006B010BD83DE1B4310E000E000ED00E0DE
:108BB80008B54FF47A7303FB00F0FFF7C9FF08BD4F
:108BC80010B5094C20464FF4DB7108F06FFD94F89E
:108BD800B431AE2B05D194F8B501AE3818BF0120D9
:108BE80010BD012010BD00BFD428002008B50548DD
:108BF800AE2380F8B43180F8B5314FF4DB7108F05A
:108C080061FD08BDD428002008B50548FF2380F879
:108C1800B43180F8B5314FF4DB7108F053FD08BD6D
:108C2800D428002008B5082007F03CFF012815D1FA
:108C3800092007F037FF012810D1094B1B686BB9D1
:108C480008480EF029FC08480EF026FC07480EF0EC
:108C580023FC0122024B1A60FFF7D6FF08BD00BFB4
:108C680018030020908A0108B88A0108E48A0108DC
:108C780008B5FEF7B1FB08BD00207047002070471B
:108C880010B5BBB101280DD1012B03D1104600F05E
:108C980023FB03E01046DAB200F09AFB003018BF5D
:108CA800012010BD28B950025A0200F0FFFD002033
:108CB80010BD10BD042010BD10B51C46DBB1012845
:108CC8000DD1012B03D1104600F01EFB03E0104626
:108CD800DAB200F0AFFB003018BF012010BD48B970
:108CE800074B1B68012B08D15002620200F054FEAA
:108CF800002010BD10BD042010BD002010BD00BF15
:108D08002C13002038B5154601281FD1012918D089
:108D180011B1032910D032E01B484FF48061FEF7EF
:108D280013FA00F005FC041C18BF012416484FF480
:108D38008061FEF7D9F925E04FF400731380002411
:108D480020E000F07FFA286000241BE0D0B9032956
:108D580017D8DFE801F0020F060B00F0E7FC00244B
:108D680010E04FF40073138000240BE001231380FC
:108D7800002407E04FF400631360002402E0042499
:108D880000E00424204638BD000C01400C4B1A6852
:108D9800A2F2BC720B4B1B685B0543EA42630A4AAA
:108DA800126843EA0243094A128843EAC223084A7E
:108DB800128843EA4213074A108843EA4000704782
:108DC800300000203C000020340000204400002037
:108DD800400000203800002000B583B04FF48063C5
:108DE800ADF8043003238DF8063010238DF80730D2
:108DF800034801A9FEF724F803B05DF804FB00BF9F
:108E0800000C014070B5064640F6FF74FF2501E0EE
:108E1800013CA4B2284600F0CDFBB04201D0002CA2
:108E2800F6D1002C14BF0020FF2070BD70B50024BF
:108E3800FF264FF6FE75304600F0BCFB00F01F0021
:108E4800AC421AD001340B2807D00D2817D00528BA
:108E580018BFFF20FF28EED001E00B2070BD0024D2
:108E6800FF2503E0013414F1030F0AD8284600F067
:108E7800A1FB0028F6D0002070BD012070BD0D2098
:108E880070BDFF2070BD00BFF8B507460C461646FA
:108E98001F4D28464FF48061FEF726F9FF2000F0A9
:108EA80089FBFF2000F086FBFF2000F083FB2846AB
:108EB8004FF48061FEF748F947F0400000F07AFB74
:108EC800200E00F077FBC4F3074000F073FBC4F3F7
:108ED800072000F06FFBE0B200F06CFB304600F0BA
:108EE80069FB0024FF2603E00134A4B2FF2C05D857
:108EF800304600F05FFB0546FF28F5D004484FF4E4
:108F08008061FEF7F1F8FF2000F054FB2846F8BD19
:108F1800000C014070B506460C461546FF2000F0CF
:108F280049FBFF2000F046FB13484FF48061FEF731
:108F38000BF946F0400000F03DFB200E00F03AFB34
:108F4800C4F3074000F036FBC4F3072000F032FBFF
:108F5800E0B200F02FFB284600F02CFB0024FF2590
:108F680003E00134A4B2FF2C04D8284600F022FB09
:108F7800FF28F6D070BD00BF000C014070B500237B
:108F880001E001339BB2B3F5706FFAD30024FF25DB
:108F980004E0284600F00EFB0134A4B2092CF8D9ED
:108FA800002426469525304631462A46FFF76CFFB1
:108FB8000134A4B2012801D0FE2CF4D9FF2C14BF2F
:108FC8000020012070BD00BFF0B587B075484FF490
:108FD8008061FEF789F80023ADF804304FF48272FF
:108FE800ADF80620ADF808300222ADF80A200124B9
:108FF800ADF80C404FF40072ADF80E203822ADF8F1
:109008001020ADF812300723ADF81430664D28460D
:1090180001A9FEF741FC28462146FEF7D3FC0420AF
:1090280000F090FAFF2000F0C5FAFFF7A7FF00282C
:1090380040F0B1805B484FF48061FEF785F8082066
:109048004FF4D5718722FFF765FF044605284BD1F9
:109058000222564B1A7053484FF48061FEF774F899
:10906800FF2000F0A7FA0024372625462927304696
:1090780029462A46FFF708FFFF2800F09180384666
:1090880029462A46FFF700FF0134A4B208B1FE2C96
:10909800EDD9FF2C11D1002401262546304629465A
:1090A8002A46FFF7F1FE0134A4B208B1FE2CF5D927
:1090B800FF2C72D001223D4B1A70012000F042FAB9
:1090C800FF2000F077FA3B2000219522FFF7DCFE15
:1090D800002864D110204FF400719522FFF7D4FEC8
:1090E8000446002855D05BE0012852D1FF2000F04B
:1090F80061FAFF2000F05EFAFF2000F05BFAFF2023
:1091080000F058FA27484FF48061FDF7EDFFFF2083
:1091180000F050FA37250024292628462146224601
:10912800FFF7B2FE01283BD130464FF0804122467E
:10913800FFF7AAFE0028F0D13A2000210A46FFF7DF
:10914800E9FE044630B117484FF48061FDF7CCFFC3
:10915800204625E0FF2000F02DFA0546FF2000F00C
:1091680029FAFF2000F026FAFF2000F023FA0D4824
:109178004FF48061FDF7B8FFFF2000F01BFA15F0EF
:10918800400F14BF04220322084B1A70012000F07C
:10919800D9F9204604E0012002E0012000E0FFE7C1
:1091A80007B0F0BD000C0140003800401C0300204F
:1091B8002DE9F84305460C46914619484FF480615D
:1091C800FDF7C2FFFE20FFF71DFE804670B1144870
:1091D8004FF48061FDF788FF4FF001081CE0384626
:1091E80000F0E8F905F8010B344600E0FF27631E9C
:1091F8009EB2002CF3D1FF2000F0DCF9FF2000F034
:10920800D9F9B9F1010F07D105484FF48061FDF78D
:109218006BFFFF2000F0CEF94046BDE8F88300BFA1
:10922800000C014010B5044609200021FF22FFF779
:109238002BFE30B9204610210122FFF7B9FF00208C
:1092480010BD10BD00B585B06846FFF7EBFF0028DC
:109258003ED19DF8003003F0C003402B08D19DF8A3
:1092680008009DF8093003EB00200130C00430E00D
:109278009DF8060000F003009DF8073003EB00207E
:109288009DF808309B0903EB80009DF8092002F047
:1092980003029DF80A30DB0903EB42030233012283
:1092A80003E0520092B2013BDBB2002BF9D100FB84
:1092B80002229DF8053003F00F03012103E0490065
:1092C80089B2013B9BB2002BF9D102FB01F000E00F
:1092D800002005B05DF804FB10B503460C46094AAA
:1092E8001278042A18BF4302112019460022FFF7FA
:1092F800CBFD30B920464FF400710122FFF758FF2B
:1093080010BD10BD1C03002070B503460C462E4A44
:109318001278042A18BF4302182019460022FFF7C2
:10932800B3FD00284FD129484FF48061FDF70CFFA9
:10933800FF2000F03FF9FF2000F03CF9FF2000F08B
:1093480039F9FE2000F036F9002506E0661C207881
:1093580000F030F90135ADB23446B5F5007FF5D3EC
:10936800FF2000F027F9FF2000F024F9FF2000F08B
:1093780021F9044600F01F03052B11D013484FF4C0
:109388008061FDF7B1FE204670BD0134A4B2B4423D
:109398000AD10E484FF48061FDF7A6FE012070BD8A
:1093A8000024FF254FF6FF76284600F003F9002831
:1093B800EBD006484FF48061FDF796FEFF2000F0E1
:1093C800F9F8002070BD70BD1C030020000C01409E
:1093D800F8B503460C461546144A1278042A18BFF5
:1093E8004302122019460022FFF74EFDE8B94FF458
:1093F80000770026204639463246FFF7D9FE28B9BD
:1094080004F50074681E10F0FF05F3D10C2000214C
:109418000A46FFF739FD06484FF48061FDF764FE00
:10942800FF2000F0C7F82846F8BDF8BD1C0300204F
:10943800000C01402DE9F04704460D4692463A4B90
:109448001B78042B18BF4402012B04D017201146A7
:109458000022FFF719FD192021460022FFF714FD0D
:10946800044600285CD131484FF48061FDF76CFE5A
:10947800FF2000F09FF8FF2000F09CF84FF0FC0957
:109488004FF00008FF27484600F094F8444606E0ED
:109498006E1C287800F08EF80134A4B23546B4F575
:1094A800007FF5D3384600F085F8384600F082F89A
:1094B800384600F07FF8044600F01F03052B05D05E
:1094C8001A484FF48061FDF70FFE29E0FFF7AEFC64
:1094D8000446012805D115484FF48061FDF704FEC4
:1094E8001EE00AF1FF3313F0FF0ACCD1FD2000F093
:1094F80061F8002808BF4FF0FE0AFFF797FC30B16B
:109508000A484FF48061FDF7EFFD012408E00748A1
:109518004FF48061FDF7E8FDFF2000F04BF854465A
:109528002046BDE8F08700BF1C030020000C014066
:1095380010B5FF24204600F03DF8FF28FAD100209E
:1095480010BD00BF1A4A138823F038031B041B0CF4
:109558001380042824D8DFE800F003080F161D0044
:10956800134B1A8892B21A801AE0114B1A8892B2D9
:1095780042F008021A8013E00D4B1A8892B242F0AA
:1095880010021A800CE00A4B1A8892B242F01802B4
:109598001A8005E0064B1A8892B242F038021A8007
:1095A800034B1A8892B242F040021A80704700BFFB
:1095B80000380040F8B507460024154E022504E09F
:1095C8000134A4B2B4F5C87F1DD830462946FEF749
:1095D8008FFA0028F4D00E483946FEF755FA0024D1
:1095E8000B4E012504E00134A4B2B4F5C87F0CD8B1
:1095F80030462946FEF77CFA0028F4D00448FEF7E6
:109608005DFAC0B2F8BD0020F8BD0020F8BD00BF6B
:109618000038004070B506460C4D02242846214605
:10962800FEF766FA0028F9D008483146FEF72CFA0A
:10963800064D012428462146FEF75AFA0028F9D09B
:109648000248FEF73BFAC0B270BD00BF00380040C8
:1096580000B583B04FF40063ADF8043003238DF8F0
:10966800063010238DF80730034801A9FDF7E8FB01
:1096780003B05DF804FB00BF000C014008B5FFF71C
:10968800E7FF03484FF40061FDF72EFD08BD00BF5A
:10969800000C014008B50023034A1380034A1380D5
:1096A800FFF7ECFF08BD00BF1E03002020030020C9
:1096B80070B58AB0194E02AC35460FCD0FC495E887
:1096C8000F0084E80F006B46324652F8200F5168AD
:1096D80003C3134D28464FF40061FDF735FDD7202D
:1096E800FFF798FF0020FFF795FF0446C0F3C20379
:1096F8000AAA1A4412F8281C0A4A11700AAA02EB8C
:10970800830353F8202C084B1A6028464FF4006155
:10971800FDF7EAFC20460AB070BD00BF088B0108BF
:10972800000C0140401300204413002008B50948EC
:109738004FF40061FDF708FDFF20FFF76BFFFFF70F
:10974800B7FF10F0800FFAD002484FF40061FDF720
:10975800CBFC08BD000C014038B504460D461A483C
:109768004FF40061FDF7F0FC72B6012C15D15320BF
:10977800FFF750FF154C2078C0F1100025FA00F0D3
:10978800C0B2FFF747FF2078083805FA00F0C0B2EA
:10979800FFF740FF0020FFF73DFF0B4C20464FF43A
:1097A8000061FDF7A1FC20464FF40061FDF7CCFCF9
:1097B800FFF77EFF10F0800FFAD062B602484FF430
:1097C8000061FDF791FC38BD000C014040130020FA
:1097D80038B504460D461A484FF40061FDF7B4FC4D
:1097E80072B6012C15D18320FFF714FF154C207891
:1097F800C0F1100025FA00F0C0B2FFF70BFF207887
:10980800083805FA00F0C0B2FFF704FF0020FFF7A0
:1098180001FF0B4C20464FF40061FDF765FC204624
:109828004FF40061FDF790FCFFF742FF10F0800F46
:10983800FAD062B602484FF40061FDF755FC38BD16
:10984800000C014040130020F8B504460F461646A8
:109858001D4615484FF40061FDF776FC72B6012CE1
:109868001AD1D420FFF7D6FE0020FFF7D3FEC7F3A6
:109878000720FFF7CFFEF8B2FFF7CCFE0020FFF776
:10988800C9FE0024274605E03846FFF7C3FE05F861
:10989800010B0134B442F7D362B603484FF40061B8
:1098A800FDF722FCF8BD00BF000C01402DE9F04F88
:1098B80083B0894601924FEA122A060AC5B208B94E
:1098C80000252E4601203146FFF746FFC5F5807476
:1098D800019B9C4228BF1C460120294622464B4634
:1098E800FFF7B2FF711C264600250127AB4612E0A0
:1098F80001F101083846FFF72FFF384659464FF463
:10990800807209EB0403FFF79FFF04F5807406F5E6
:109918008076013541465545EAD3019BB3420BD9C0
:109928009E1B09D00120FFF717FF012000213246B6
:1099380009EB0403FFF788FF03B0BDE8F08F00BF11
:10994800F8B504460F4616461D4612484FF4006106
:10995800FDF7FAFB72B6012C15D18420FFF75AFEE9
:109968000020FFF757FEC7F30720FFF753FEF8B2B2
:10997800FFF750FE002404E015F8010BFFF74AFE3C
:109988000134B442F8D362B602484FF40061FDF7DF
:10999800ABFBF8BD000C01402DE9F04F83B08A46BF
:1099A80001924FEA122B10B1060AC1B201E0002160
:1099B8000E46C1F58074019B9C4228BF1C460120BD
:1099C80022465346FFF7BCFF01203146FFF700FF50
:1099D8000136274600254FF0010813E040460021D4
:1099E8004FF480720AEB0403FFF7AAFF06F101099E
:1099F80040463146FFF7ECFE04F5807407F58077A2
:109A080001354E465D45E9D3019BBB420BD9DA1BB4
:109A180009D0012000210AEB0403FFF791FF012080
:109A28003146FFF7D5FE03B0BDE8F08F30B4002310
:109A380003E08C4208BF2A700133C518C45C002CAF
:109A4800F7D130BC704700BF03463038C0B2092890
:109A580012D9A3F16102D2B2052A03D8A3F15700A3
:109A6800C0B27047A3F14102D2B2052A03D8A3F1CC
:109A78003700C0B270471846704700BF2DE9F04163
:109A880006460024254611E073555BB2252B0BD101
:109A9800B7187878FFF7D8FF8046B878FFF7D4FF73
:109AA80000EB081070550234013501342246335D4D
:109AB800002BE9D17355BDE8F08100BF30B585B002
:109AC8000446012918D0022918D0032918D00429DE
:109AD80018D0052918D0092918D00A2918D00C2916
:109AE80018D00B2918D0082918D00D2918D00E29FC
:109AF800184D18BF002514E0174D12E0174D10E05F
:109B0800174D0EE0174D0CE0174D0AE0174D08E011
:109B1800174D06E0174D04E0174D02E0174D00E021
:109B2800174D01A817490DF0CFFC204629460DF026
:109B380013FD204601A90DF0EBFC20460DF014FDA5
:109B480002462118104B1868A0501B790B7105B0FC
:109B580030BD00BF208E0108348B0108888B0108B6
:109B6800C48B0108008C01083C8C01088C8C01080E
:109B7800E08C01081C8D0108608D0108A88D010882
:109B8800E48D0108608E0108E0B50108F8B50546C6
:109B98000C4608464D490DF02AFD20B920464C498F
:109BA8000DF025FD10B101232B70F8BD2046494961
:109BB8000DF01DFD10B102232B70F8BD204646495B
:109BC8000DF015FD20B9204644490DF010FD10B1E7
:109BD80003232B70F8BD204641490DF008FD20B93C
:109BE800204640490DF003FD10B104232B70F8BD49
:109BF80020463D490DF0FBFC10B105232B70F8BD44
:109C080020463A490DF0F3FC064628B92046384963
:109C18000DF0EDFC074610B108232B70F8BD204667
:109C280034490DF0E4FC20B9204633490DF0DFFC3F
:109C380010B10C232B70F8BD204630490DF0D7FC2D
:109C480020B920462E490DF0D2FC10B10B232B7001
:109C5800F8BD07B916B108232B70F8BD204629496D
:109C68000DF0C5FC20B9204627490DF0C0FC10B105
:109C780009232B70F8BD204624490DF0B8FC20B903
:109C8800204623490DF0B3FC10B10A232B70F8BD10
:109C9800204620490DF0ABFC20B920461E490DF0A6
:109CA800A6FC10B10D232B70F8BD20461B490DF002
:109CB8009EFC20B920461A490DF099FC10B10E23DC
:109CC8002B70F8BD00232B70F8BD00BF648E01080F
:109CD800989001086C8E0108748E01087C8E01082A
:109CE800848E01088C8E0108948E010818B0010832
:109CF8009C8E0108A48E0108AC8E0108B48E010860
:109D0800B88E0108BC8E0108C48E0108CC8E0108EB
:109D1800D48E0108DC8E0108E48E0108EC8E01085F
:109D2800F48E010838B50546084624490DF078FC3C
:109D3800044610B900232B7038BD21490DF002FCF0
:109D480020B120461F490DF0FDFB38B901232B70C7
:109D580000201A490DF064FC044625E020461A4903
:109D68000DF0F0FB20B1204618490DF0EBFB38B997
:109D780002232B70002011490DF052FC044613E019
:109D8800204613490DF0DEFB20B1204611490DF0A5
:109D9800D9FB38B9002010490DF042FC04460323D2
:109DA8002B7001E000232B7014B900232B7038BDF1
:109DB800A81C21460DF0D0FB38BD00BFDC8C010883
:109DC800FC8E0108008F0108048F01080C8F010820
:109DD800148F01081C8F0108308B010810B5ADF5F0
:109DE800B76D014670B168460DF0B6FB6846074985
:109DF8000DF016FC044606490DF0A4FB00B1013431
:109E0800204600E000200DF5B76D10BD248F010835
:109E1800288F010870B504460E46002305E003FBB1
:109E280006F50134FFF710FE2B18207808B120281A
:109E3800F5D198B270BD00BF2DE9F04188B0034656
:109E48000E46684619460DF087FB68460024104DFB
:109E58000A274FF0100816E029460DF0E1FB0378B9
:109E6800302B08D14378782B05D102304146FFF7D3
:109E7800D1FFC0B203E03946FFF7CCFFC0B230557E
:109E88000134E4B20020032CE6D908B0BDE8F08123
:109E98002C8F0108F8B50F4615461E460DF0A7FB96
:109EA800044638460DF060FB0444204629460DF070
:109EB8009EFB001B85B2304621462A460DF072FBF8
:109EC80000237355F8BD00BF70B584B00C4600235D
:109ED80001930293ADF80C30054600283FD00029C5
:109EE8003FD02249224A01ABFFF7D4FF01A80A213B
:109EF800FFF790FF064628461E490DF078FB043010
:109F08000023835521460DF072FB054658B32046C1
:109F18000DF02AFB01302C18204626210DF005FBF8
:109F2800034618B920460DF01FFB2318181B83B2EF
:109F38008BB11A46104D00235355284621460DF083
:109F480031FB2846FFF79AFD28462B212022FFF7F0
:109F58006DFD284608E008480023037004E000204F
:109F680002E0002000E0002004B070BD308F01083E
:109F78007C920108E0B5010848130020704700BF33
:109F8800704700BF014B185C704700BF34030020C6
:109F98000023074906E0CA5C824201D1D8B204E036
:109FA8000133DBB2072BF6D9FF2040B2704700BF60
:109FB8003403002010B5400100F5847420460821C0
:109FC80001F0CEFF204601F0ADFF0028FAD10120B4
:109FD80010BD00BF30B583B005460C460092084658
:109FE8000549064A0DF070FA82B22846214602F069
:109FF800ADFA03B030BD00BF58900108A88D010824
:10A0080038B505461C46B3F5C87F0FD0B3F5CA7FEF
:10A0180013D0C82B19D1A1F10803DBB2012B13D936
:10A02800104B186849B2FFF749FD0EE00D4B186850
:10A038000D4976220DF0FBF807E00A4B18680B492A
:10A0480099220DF0F4F800E000244CB1054B1C688F
:10A0580020460DF089FA82B22846214602F076FAA7
:10A0680038BD00BF28030020448F0108BC8F0108B9
:10A078002DE9F04383B080460F46164699460A9D5F
:10A08800FFF786FF0446B0F1FF3F7CD000EBC0022B
:10A098003E4B03EB0212D2F88820C2B9B5F5006F27
:10A0A8003CD300EBC00003EB0010C0F88490C0F86C
:10A0B8008850451C2846002180220DF0C1F828460A
:10A0C80039460DF049FA002740F2FF7529E000EB08
:10A0D800C0032E4901EB0313D3F88C50551BB5F57B
:10A0E800006F26BF002740F2FF75012700EBC00173
:10A0F800264B03EB011126480131012205F054F9E2
:10A10800244B187060B904EBC403204A02EB031314
:10A118001F48D3F88C1005F0EFFB02E0002700E0A1
:10A1280000251B4831462A460DF1060305F0F0F9D3
:10A13800184B187018B96B1C0022F25400E0002567
:10A148002DB140463146AAB202F000FA00E00127DC
:10A1580067B10E4AE100081902EB00100023C0F8AD
:10A168008430C0F88830C0F88C3009E0074BE20032
:10A17800111903EB0111D1F88C301D44C1F88C5032
:10A18800034805F0A9FB03B0BDE8F0833C030020B9
:10A19800501B0020741F00202DE9F0418CB00546AB
:10A1A8000C4600230B93039304930593069307939C
:10A1B800089309930A93FFF7EBFEB0F1FF3F00F015
:10A1C800C980664B1A68664B1A602378032B00F225
:10A1D800BA80DFE803F0020A0A7F284600210A460F
:10A1E8004FF4C873FFF70CFFB4E0A01CFFF7F6FDAF
:10A1F80006465C490DF0A6F938B95B4B03CB3060D5
:10A2080071601A889B783281B372304657490DF0D5
:10A2180099F930B9564B07CB30607160B2601B7842
:10A228003373304653490DF08DF938B9524F0FCF7B
:10A2380030607160B260F3603B883382601C3146E5
:10A24800FFF7A4FC6378082B1CD130464B4B1968E8
:10A258000BAA00F097F968B10B9B40F2BE729342CB
:10A2680008D828463E4A1168444A12689BB2FFF74C
:10A27800B1FE6FE02846082100224FF4CA73FFF7A9
:10A28800BFFE67E03E483146012205F08DF83D4BA0
:10A29800187030B93A4BDA680B92D3F81080012263
:10A2A80001E000229046002A14BFC8274FF4CA775D
:10A2B800284661780B9A3B46FFF7A2FEC82F49D182
:10A2C800274B1A680B9B0093284631464346FFF7F5
:10A2D800CFFE3FE0A01C23492B4A03ABFFF7DAFD72
:10A2E800601C03A9FFF752FC6378082B23D103A84D
:10A2F80021461B4B1A680BAB00F0A0F9044690B13D
:10A308000B9B40F2BE7293420DD828461B4A116837
:10A31800134A12689BB2FFF75DFE022C1AD11B4B41
:10A328001B68984716E02846082100224FF4CA7394
:10A33800FFF766FE0EE0284600210A464FF4CA736E
:10A34800FFF75EFE06E0284600210A464FF4C87370
:10A35800FFF756FE0CB0BDE8F08100BF4C1B002093
:10A3680028030020288F01086490010870900108D4
:10A3780074900108849001088C900108481B002003
:10A38800501B0020741F0020A09001084C000020E2
:10A3980010B40023054C03E0CA5CE2540133DBB27D
:10A3A8008342F9D35DF8044B704700BF34030020A3
:10A3B80010B5044C20600448016010461946FFF7A8
:10A3C800E7FF10BD481B00204C1B002008B1034AC2
:10A3D800106009B1024B1960704700BF4C000020A3
:10A3E8004800002070B582B006465B4B1A685B4B8C
:10A3F8001A605B4B1A685B4B1A60FFF7C3FD044693
:10A408004501083505F5407001F08CFD1338092821
:10A4180000F29680DFE800F0909A9A9A0594949456
:10A42800948C05F50075284601F07CFD10F0010FAD
:10A4380003D02846012101F093FD06EBC6031B015A
:10A44800494AD35C032B46D0042B5BD0002B7DD12B
:10A45800204601F02BFE82B213B2002B76DDB3F555
:10A46800006F20463D4B1968C8BF4FF4006202F0E8
:10A478000DF985B215F4004F68D1384B186808F00B
:10A48800C7FA30B106EBC60633010421364AD15467
:10A498005CE0324B19682DB200234B55314D2868CA
:10A4A800FFF740FC20462968FFF776FE06EBC60357
:10A4B8002D4A02EB0313D3F888302BB106EBC606FE
:10A4C80033010321D15441E006EBC60633010421D0
:10A4D800254AD1543AE0254B1A68002300932046B8
:10A4E8001946FFF7C5FD06EBC6031F4A02EB031327
:10A4F800D3F8883053BB06EBC606360104221A4B44
:10A508009A5523E01849F000821901EB0212002342
:10A51800C2F88830C2F88C30C2F884303044000168
:10A528000B54134B1B6898472046FFF743FD0DE07B
:10A538002046FFF73FFD09E0204601F015FF05E042
:10A54800204601215022002301F082FE084B1B689F
:10A55800984702B070BD00BF4C1B00202C030020A0
:10A56800481B0020300300203C0300202803002063
:10A5780048000020024B1A6801321A60704700BF79
:10A5880024030020F0B583B004460F46164602AAFD
:10A59800002522F8025D07F087FF00283BD12046FE
:10A5A80021490CF0CFFF30B938460DF1060107F00C
:10A5B8001FF9012032E020461C490CF0C3FF30B9D6
:10A5C80038460DF1060107F06FFA012026E0204613
:10A5D80017490CF0B7FF30B938460DF1060107F0FE
:10A5E80017FB01201AE0204612490CF0ABFF30B9E6
:10A5F80038460DF1060107F0F7FB01200EE0204672
:10A608000D490CF09FFF40B938460DF1060107F0DF
:10A61800C3FB012002E0012000E0002010B1BDF8DA
:10A628000630336003B0F0BDA8900108B49001086B
:10A63800BC900108CC900108E0900108F0B583B007
:10A64800054617461E4602AB002423F8024D8C1C13
:10A65800214608F055F900285AD1284631490CF00E
:10A6680071FF58B9204607F0CFFB014605203A464E
:10A678000DF1060307F07EFD02204CE028462A492A
:10A688000CF060FF58B9204607F086FC02463846B1
:10A6980026490CF019FF0120ADF806003BE02846DA
:10A6A80023490CF04FFF58B9204607F0BDFC02467D
:10A6B80038461E490CF008FF0120ADF806002AE0D4
:10A6C80028461C490CF03EFF58B9204607F0E4FC28
:10A6D8000246384615490CF0F7FE0120ADF8060091
:10A6E80019E0284614490CF02DFF20B9204607F040
:10A6F80013FD01200FE0284610490CF023FF48B94C
:10A70800204607F01FFD0023ADF80630022002E0C6
:10A71800012000E0002010B1BDF80630336003B01E
:10A72800F0BD00BFE8900108F4900108289C0108DA
:10A738000091010810910108209101083491010845
:10A7480038B50E4A0023D3701D2111710121917172
:10A7580005780B4C2570457865708578A570C078AC
:10A76800E07048F6B8040748048007480088A2F853
:10A778006B000220152201F06BFD38BD801F002000
:10A78800781F00207C1F0020288F010810B59AB080
:10A7980001AC074B0FCB84E80F00022021460F22A3
:10A7A80001F0D4FE0120034BD8701AB010BD00BFD1
:10A7B80050910108801F00202DE9F84381460024AC
:10A7C8001F4FDFF888801F4E12E02CB948464146DB
:10A7D8000CF026FF054604E0002039460CF020FF67
:10A7E800054628460A210CF0DBFC3055FDB1013442
:10A7F800032CEADD0025144B1D80DFF850802F461E
:10A808001C460FE0384641460CF00AFF06462388EE
:10A818001B0223800A210CF0C3FC238818442080E3
:10A828004EB10135012DEDDD0020BDE8F8834FF074
:10A83800FF30BDE8F8834FF0FF30BDE8F88300BF74
:10A8480064910108DC240020E024002060910108C4
:10A8580070B5B6B0064604468D490BE05AB20D688D
:10A8680015446A7802F00302012A5BB208BF20335C
:10A8780004F8013B23785DB2202D0ED0002BEDD1DA
:10A88800844D0BE020460CF06FFE02462046314610
:10A898000CF072FE28B1043500E07E4D2C68002CC7
:10A8A800F0D15CB904A87C4932460CF00DFE82B2A6
:10A8B800022004A901F04AFE0020EFE2774BDB7882
:10A8C800E3B9744BEB1A9B10022B17D0082B15D049
:10A8D800A3B104AC724D0FCD0FC40FCD0FC495E8D2
:10A8E800030044F8040B24F8021B090C2170022011
:10A8F80004A9262201F02AFE0020CFE220460CF00F
:10A9080033FE341800E0013494F90030202BFAD0DB
:10A91800604BED1AAD101C2D00F2B182DFE815F086
:10A928001D009E023E004B006901EC017E02AF0251
:10A93800A500CE00F8002D01BB02880188015E0247
:10A948005E029E029E029E029E0279019E029E0265
:10A9580099009401B3015901F80020460CF004FE57
:10A96800421E0023A354023823544E4821460CF0BB
:10A97800F3FD04AC4C4D0FCD0FC495E8070003C49C
:10A988002270022004A9182201F0E0FD041E80F2C2
:10A998008482022001F026FCE0B27FE220460CF01F
:10A9A800E3FD421E0023A354023823542046FFF738
:10A9B800EDFE012072E220460CF0D6FD421E002377
:10A9C800A3540238235494F90030413B282B34D83F
:10A9D800DFE803F01524333333333333243333338D
:10A9E800333333333333333333333333333333332F
:10A9F80033333333152433333333333324000022D2
:10AA0800264B9A7004A8294922460CF05DFD82B2B3
:10AA1800022004A901F09AFD01203FE201251F4B05
:10AA28009D7004A8214922460CF04EFD82B20220F6
:10AA380004A901F08BFD284630E204A81C492246EF
:10AA48000CF042FD82B2022004A901F07FFD012032
:10AA580024E204A8174975220CF0E9FB022004A996
:10AA6800742201F073FD012018E2134B04AC0FCBE4
:10AA780007C424F8023B1B0C2370022004A90E22F1
:10AA880001F064FD022001F019FD012006E200BF7B
:10AA9800200200205000002068910108801F00203B
:10AAA80084910108871F0020AC910108C891010812
:10AAB800E0910108F89101087092010820460CF015
:10AAC80053FD421E0023A35402382354A4480CF01B
:10AAD8004BFD012805D1A348A34922460CF0F4FCFC
:10AAE80006E0A04A1046A149643A23460CF0ECFC63
:10AAF8009C4C04A89E4922460CF0E6FC82B2022037
:10AB080004A901F023FD092304F8CB3C0120C5E189
:10AB180020460CF029FD421E0023A354023823547A
:10AB28008F480CF021FD012805D18E488E49224618
:10AB38000CF0CAFC06E08B4A10468C49643A23465E
:10AB48000CF0C2FC874C04A88A4922460CF0BCFCD5
:10AB580082B2022004A901F0F9FC0A2304F8CB3CD4
:10AB680003208549854B1A8801F036FC012840F0FE
:10AB780095810022824B1A7090E12046FFF71CFE57
:10AB8800B0F1FF3F0FD104AC7E4D0FCD0FC495E857
:10AB9800030044F8040B2180022004A9152201F0C7
:10ABA800D5FC01207AE1784B01269E715E7104ACD8
:10ABB800764D0FCD0FC495E80F0007C424F8023B6B
:10ABC8001B0C2370022004A91E2201F0BFFC304692
:10ABD80064E1634C04A86E4922460CF075FC82B20D
:10ABE800022004A901F0B2FC1B2304F8673C0120F1
:10ABF80054E15B4C04A8664922460CF065FC82B21D
:10AC0800022004A901F0A2FC042304F8673C0120F7
:10AC180044E104AC5F4D0FCD0FC495E80F0007C4A5
:10AC28002380022004A91D2201F090FC012035E1B7
:10AC380004A859494A4A0CF047FC82B2022004A9E8
:10AC480001F084FC012029E154490A784B788D7879
:10AC5800CC7853490988080AC9B200950194029032
:10AC6800039104A84F490CF02FFC82B2022004A9DA
:10AC780001F06CFC032001F021FC434B00229A7187
:10AC8800012058710AE120460CF06EFC421E002398
:10AC9800A354821EA35403281DDD20462F210CF047
:10ACA80093FC0146002301F8013B204605F02EF8ED
:10ACB800021E05DD04A83C490CF006FC024614E01F
:10ACC80004AC3A4D0FCD0FC495E8030044F8040BCB
:10ACD8002170142209E004AC344D0FCD0FC495E85F
:10ACE800030044F8040B21701422022004A992B234
:10ACF80001F02CFC0120D1E020460CF035FC421E6E
:10AD08000023A354821EA354032855DD03381E468E
:10AD1800235420462F210CF057FC0546014601F824
:10AD2800016B204604F0F2FF2F232B70024678B9FE
:10AD380004A81D490CF0C8FB094D284621460CF013
:10AD48000BFC04A81A492A460CF0BEFB02463EE05A
:10AD580004A8184922460CF0B7FB024637E000BFAA
:10AD6800EB1F00204F2000208092010884920108E8
:10AD78008C920108D0920108DC240020E0240020F5
:10AD8800BD07002010930108801F002028930108A8
:10AD98004893010884930108A4930108781F0020B0
:10ADA8007C1F0020C8930108F89301080494010847
:10ADB8001C940108509401083A4D284621460CF08D
:10ADC800CBFB04A838492A460CF07EFB0246022039
:10ADD80004A992B201F0BAFB01205FE020460CF012
:10ADE800C3FB421E0023A35402382354204605F017
:10ADF800A1F830B104A82D4922460CF065FB0246A3
:10AE080005E004A82A4922460CF05EFB024602200F
:10AE180004A992B201F09AFB01203FE020460CF011
:10AE2800A3FB421E0023A35402382354204605F0F6
:10AE380025F830B104A81F4922460CF045FB02460C
:10AE480005E004A81C4922460CF03EFB02460220FD
:10AE580004A992B201F07AFB01201FE004AC174D5F
:10AE68000FCD0FC40FCD0FC495E8030084E803008D
:10AE7800022004A9272201F069FB01200EE004A8A2
:10AE88000F4922460CF020FB82B2022004A901F0EF
:10AE98005DFB012002E0012000E0012040B236B055
:10AEA80070BD00BFEB1F00201C94010868940108C6
:10AEB8008C940108B0940108D0940108E494010826
:10AEC800689101082DE9F04182B005460023ADF8EC
:10AED80006304FF4527001F025F81C287ED8DFE8C0
:10AEE80000F0657D7D7D7D7D7D7D7D7D7D7D7D7DAC
:10AEF8007D7D7D7D7D737D7D7D0F7D7D7D7D5E008E
:10AF0800964B1B78DBB9964B1A88964B1A802846C5
:10AF18009549964A964B0CF0D7FA28460CF024FB34
:10AF280082B20220294601F011FB041E04DA022035
:10AF380001F058F9E4B2D8E10122884B1A700220D6
:10AF480001F0B4F80446ADF80600002846D02846BB
:10AF580000214FF400720CF073F9B4F5007F84BF40
:10AF680040F2FF13ADF8063002202946BDF806204E
:10AF780001F08CFB044600232B54BDF806308342B5
:10AF880009D0002800F0AA81002804DA022001F084
:10AF980029F9E4B2A9E12846FFF75AFC1EE002208D
:10AFA80001F08CFA012819D0C4B29EE102200121D7
:10AFB8001522002301F04CF9044602280ED0022085
:10AFC80001F010F9E4B290E1022001F0CDF9012876
:10AFD80001D0C4B289E10022604B1A704FF45A7054
:10AFE80000F0A0FF04461C2800F27A81DFE810F088
:10AFF80028017801780178017801780178017801D1
:10B008007801780178017801780178017801780170
:10B018007801780178015E017801780178011D00D6
:10B0280078017801780178012101524B1B7813B916
:10B038000122504B1A70504B1B79043B172B00F21E
:10B048005181DFE813F018004F014F014F014F0104
:10B058003D009F004F014F014F014F014F014F012C
:10B068004F014F014F014F014F014F014F014F0158
:10B078004F014F0118003B4C204629460DF10602AE
:10B0880004F05AFD28460CF06FFA82B2ADF806209B
:10B098000320294601F05AFA1D2304F8673C0320CF
:10B0A80001F00CFA2846354922460CF00DFA82B216
:10B0B800ADF806200220294601F048FA002414E1E0
:10B0C8002F4C2046A4F16501012204F06DF984F8A3
:10B0D800240468BBA4F59A73D3F840414FF4007672
:10B0E80003F59A77A7F59A78FDF7C2FD284600215F
:10B0F80032460CF0A5F8B4F5007F94BFA2B23246F0
:10B108003846294601AB04F003FA88F8580548B9CF
:10B1180003202946BDF8042001F018FABDF80430D0
:10B12800E41AE1D1164C204604F0D6FB84F8240436
:10B13800114C1D232371032001F0C0F928460F4943
:10B1480004F1CF020CF0C0F982B2ADF8062002205B
:10B15800294601F0FBF90024C7E000BFBC07002026
:10B16800288F0108EB1F00200C9501082C95010879
:10B1780034950108BD070020801F0020389501087C
:10B18800B42000205B4C2046A4F165010A2204F09B
:10B198000BF984F82404002836D12746A4F59A78B8
:10B1A800032000F083FF044610B34FF40076FDF748
:10B1B8005FFD2846002132460CF042F8B4F5007FC6
:10B1C80094BFA2B232460320294601F05FFA024634
:10B1D8003846294601AB04F055FA88F85805BDF8F9
:10B1E8000430E41A08B9002CE1D10028D8D005E0D1
:10B1F8004FF45A7000F096FE1728D1D03D4C2046E7
:10B2080004F06AFB84F824043B4C1D2323710320BB
:10B2180001F054F92846394904F1CF020CF054F9E9
:10B2280082B2ADF806200220294601F08FF90024E9
:10B238005BE0032001F042F9012855D0C4B254E084
:10B248002D4B5B79012B50D12B4B9B79E3B9032014
:10B2580001212B4B1A88002300F0FAFF054603282A
:10B2680004D0032000F0BEFFECB23EE0244A13886D
:10B2780001339BB213804CF25032934212D948F6F4
:10B28800B8021F4B1A800DE003200121142200236D
:10B2980000F0DEFF0546032804D0032000F0A2FFDB
:10B2A800ECB222E00222144B5A711EE0124B9B7939
:10B2B80033B9032001F058F801280BD0C4B214E0C8
:10B2C80003201049104B1A8801F086F8012801D094
:10B2D800C4B20AE000240D4B1C7006E0002404E010
:10B2E800002402E0002400E00024204602B0BDE86B
:10B2F800F08100BFB4200020801F0020389501088D
:10B308007C1F0020DC240020E0240020BD07002052
:10B3180008B54FF470600849042200F073FE4FF43A
:10B32800A0600649042200F06DFE4FF480700449C5
:10B33800042200F067FE08BDD0070020C0070020E7
:10B34800CC07002008B50020802100F009FE00206D
:10B3580000F0E8FDFFF7DCFF4FF410600249062219
:10B3680000F050FE08BD00BFE424002008B500200E
:10B37800802100F0F5FD002000F0D4FD4FF41060AE
:10B388000249062200F03EFE08BD00BFE42400206A
:10B3980010B40B4C0B4B1C600B4C0C4B1C600C4C36
:10B3A8000C4B1C60034608B10648036009B1074B03
:10B3B80019600AB1074B1A605DF8044B704700BF6B
:10B3C80019B30008D00000204DB30008CC000020BD
:10B3D80075B30008D400002010B582B04FF4106097
:10B3E8006946062200F0DCFD32490A680123137021
:10B3F8000A6853700A680623937008680022C270AE
:10B4080009682D480068040E0C71C0F307444C719C
:10B41800C0F307248C71C8710A8180208872CA72AF
:10B428000A734A738A73CA730A744A748A74CA7428
:10B438000A754A758A75CA750A764A768A76CA7608
:10B448001E4A107808775078487790788877D078AF
:10B45800C877107981F82000527981F821200020DE
:10B4680003E0CA1810770133DBB20F2BF9D9002398
:10B47800184604E0CA1882F82C000133DBB23F2BCF
:10B48800F8D90023184604E0CA1882F86C00013382
:10B49800DBB213F0800FF7D0632381F8EC308222FF
:10B4A80081F8ED20532281F8EE2081F8EF3002B0C8
:10B4B80010BD00BFF4240020EC240020E424002068
:10B4C800F0B585B0FFF788FF504B1968352381F830
:10B4D800F030012381F8F13081F8F2303D2281F813
:10B4E800F320072281F8F42081F8F530484B1A78C8
:10B4F80081F8F6205A7881F8F7209A7881F8F820B0
:10B5080093F803E081F8F9E01F7981F8FA705E7921
:10B5180081F8FB600C2381F8FC30002381F8FD30B2
:10B5280012223C4807E0541CC55C0A4482F8EC50DF
:10B5380001339BB2A2B2C45C002CF4D1541CA4B257
:10B548000A4482F8ECE0601C80B20C4484F8EC7089
:10B55800421C92B2084480F8EC60D51A0D440333BB
:10B5680085F8E830531C9BB20A44372082F8EC0077
:10B57800581C80B20B44062283F8EC20431C9BB273
:10B588000844012480F8EC40181980B20B440324C5
:10B5980083F8EC40431C9BB2084480F8EC205A1C0A
:10B5A80092B20B440F2083F8EC00531C9BB20A4460
:10B5B8003A2082F8EC005A1C92B20B443B2083F8E4
:10B5C800EC00531C9BB20A44FF2082F8EC000020D8
:10B5D80004E0CA1882F8EC0001339BB2B3F59C7FF3
:10B5E800F7D3FF238DF80C308DF80D308DF80E3021
:10B5F8008DF80F30084B1878432300934FF40972E5
:10B6080003AB01F0BBF805B0F0BD00BFF424002087
:10B61800E4240020DC000020F8240020F0B585B0E8
:10B62800FFF7DAFE7E4B1B78033BDBB2012B1BD8FE
:10B638007C4B1B6800229A72DA727B4A1178197364
:10B648005178597391789973D278DA73774B1A785D
:10B658008DF80C205A788DF80D209A788DF80E20E8
:10B66800DB788DF80F3008E0FF238DF80C308DF86B
:10B678000D308DF80E308DF80F306A4B1968352370
:10B6880081F8F030012381F8F130032281F8F220AB
:10B698003D2281F8F320072281F8F42081F8F53063
:10B6A800634B1A7881F8F6205A7881F8F7209A784F
:10B6B80081F8F82093F803E081F8F9E01F7981F820
:10B6C800FA705E7981F8FB609DF80F30FF2B26D168
:10B6D800322381F8FC30042281F8FD20524B18787F
:10B6E80081F8FE00587881F8FF00987881F8000109
:10B6F800DB7881F80131362381F8023181F80321A2
:10B708004A4B1A7881F804215A7881F805219A78E9
:10B7180081F80621DB7881F807311C2200E010222D
:10B728008B180C2083F8EC00501C023208440023CC
:10B7380080F8EC303F4D05E0541C0A4482F8EC00D8
:10B748000133A2B2E85C0028F6D1541CA4B20A4422
:10B7580082F8ECE0601C80B20C4484F8EC70421C67
:10B7680092B2084480F8EC60D01A0844033380F899
:10B77800E830531C9BB20A44372082F8EC005A1C6C
:10B7880092B20B44082083F8EC00531C9BB20A4485
:10B79800012082F8EC001A1892B20B44032083F8B7
:10B7A800EC00531C9BB20A44062082F8EC005A1C99
:10B7B80092B20B440F2083F8EC00531C9BB20A444E
:10B7C8003A2082F8EC005A1C92B20B443B2083F8D2
:10B7D800EC00531C9BB20A441F2082F8EC005A1C50
:10B7E80092B20B44212083F8EC00531C0A44FF203A
:10B7F80082F8EC009BB2002003E0CA1882F8EC0043
:10B808000133B3F59C7FF8DB0B4B18784323009387
:10B818004FF4097203AB00F0B1FF05B0F0BD00BFF3
:10B82800BE070020F4240020D0070020F0240020C8
:10B83800E4240020DC000020F824002000B585B0B6
:10B84800FFF7CAFD374B196800238B72CB7235237B
:10B8580081F8F030012381F8F130042281F8F220D8
:10B868003D2081F8F300072081F8F40081F8F530D5
:10B878002D4B187881F8F600587881F8F7009878F9
:10B8880081F8F800D87881F8F900187981F8FA0079
:10B898005B7981F8FB30322381F8FC3081F8FD2098
:10B8A800224B187881F8FE00587881F8FF009878C4
:10B8B80081F80001DB7881F80131362381F8023103
:10B8C80081F803211A4B1A7881F804215A7881F8F3
:10B8D80005219A7881F80621DB7881F80731FF2362
:10B8E80081F808311D23002003E0CA1882F8EC0013
:10B8F8000133B3F59C7FF8DBFF238DF80C308DF80E
:10B908000D308DF80E308DF80F300A4B1878432320
:10B9180000934FF4097203AB00F030FF05B05DF8F7
:10B9280004FB00BFF4240020E4240020D0070020FA
:10B93800F0240020F82400202DE9F04387B0684B5C
:10B94800187800F0B3FB0246002800F0B780644B7B
:10B958001878644B19680DF10E03009304AB00F0DE
:10B96800B1FFBDF80E30432B40F0A5805D4B1B683E
:10B97800197F5D4A1278914240F0A280597F5A4A55
:10B988005278914240F09E80997F574A927891422E
:10B9980040F09A80D97F544AD278914240F09680FC
:10B9A80093F82010504A1279914240F0918093F810
:10B9B80021104D4A5279914240F08C8080B203F1B7
:10B9C800F00103440020494F494E9846DFF82CC146
:10B9D800484D494C6CE00A78062A34D005D8012A2B
:10B9E80013D06AB1032A1AD05DE0352A0AD002D8EA
:10B9F800332A3CD057E0362A4BD0FF2A57D052E0A2
:10BA0800013155E08878033152E08A782A70CA7883
:10BA18006A700A79AA704A79EA70063148E04A7869
:10BA280091F8029084F8009091F8039084F80190BE
:10BA380091F8049084F8029091F8059084F80390A6
:10BA48001144023134E04A7891F8029087F8009066
:10BA580091F8039087F8019091F8049087F8029084
:10BA680091F8059087F803901144023120E08A7814
:10BA7800CCF8002091F8039009EB022291F8049089
:10BA880009EB02294A7902EB0922CCF80020063199
:10BA98000EE08A783270CA7872700A79B2704A7980
:10BAA800F270063104E08A1C4978114400E04146EE
:10BAB800994290D300E00020C0B20CE000200AE0D8
:10BAC800002008E0002006E0002004E0002002E05A
:10BAD800002000E0002040B207B0BDE8F08300BFBE
:10BAE800F8240020F4240020E4240020D4070020B7
:10BAF800F0240020C0070020CC070020D800002038
:10BB080030B583B04FF4D85000F00CFA05464FF426
:10BB1800D850032100F024FA104B187841F28833EA
:10BB280000930F4911220F4B00F028FE04464FF4F2
:10BB3800D850294600F014FA14F10D0F0AD0FFF777
:10BB48007DFE094B19681A4613685B1A012BFBD94D
:10BB5800002000E0012003B030BD00BFF824002021
:10BB680038960108D0070020C40700200023044AA3
:10BB780013600521034A1160034A1370704700BF20
:10BB8800C4070020C8000020D807002010B5214BAA
:10BB980093F90030012B23DC1F4B1A681F4B1B68DD
:10BBA8009A4234D21E4B93F90030022B06D0042B54
:10BBB80007D0012B07D1FFF783FC04E0FFF72EFD28
:10BBC80001E0FFF72BFD154B00221A601A680532B9
:10BBD800114B1A600F4B1A7801321A70012417E0C2
:10BBE8000F4B93F90030022B07D0042B05D0012B03
:10BBF80009D100240A4B1C7006E0FFF761FC012400
:10BC0800074B1C7000E00124FFF7B0FF00E001249F
:10BC1800204610BDD8070020C8000020C407002017
:10BC2800BE07002010B5654B93F90030062B00F0D5
:10BC3800C280634B1878400100F5427000F072F939
:10BC4800222806D05E4B187802214422002300F0F7
:10BC5800FFFAFFF771FEC0B2584B93F90030042B7E
:10BC680000F2A280DFE803F0030F274A6A00554B71
:10BC780000221A705A709A70DA70FFF721FC0124BA
:10BC88004E4B1C7095E0022811D14F4B1A68117C5D
:10BC98004C4B1970517C5970917C9970D27CDA7038
:10BCA800FFF7BCFC0222454B1A70012481E0FFF724
:10BCB8006DFF04467DE0052816D1FFF721FF48B146
:10BCC800424B1B689847FFF751FF03223B4B1A7002
:10BCD80001246EE0FFF74AFF3D4B1B68984700229E
:10BCE800364B1A70012464E0062803D10124334B33
:10BCF8001C705EE0FFF74AFF04465AE0354B1B68AC
:10BD0800B3F1FF3F52D0344A1268B2EB530F4FD908
:10BD18002C4A1178314B1970517859709178997073
:10BD2800D278DA702E4B1A6801321A60FFF776FC67
:10BD3800FFF71CFF0424214B1C703AE0052826D18C
:10BD48000022284B1A70254B1A781E4B1B789A42F2
:10BD580011D1224B5A781B4B5B789A420BD11F4B5F
:10BD68009A78184B9B789A4205D11C4BDA78154B78
:10BD7800DB789A4204D01C4B1B689847032400E0E8
:10BD88000424FFF7F3FE03220C4B1A7011E0062877
:10BD980006D1FFF7EBFE0122084B1A70042408E0D5
:10BDA800FFF7F4FE044604E0012402E0042400E066
:10BDB8000424204610BD052010BD00BFBE0700208A
:10BDC800F8240020D0070020F4240020D000002010
:10BDD800D4000020D8000020C4070020C807002095
:10BDE800EC240020D8070020CC000020F0B583B058
:10BDF80006460D4600238DF804308DF805308DF881
:10BE080006308DF80730224C4FF410602146062288
:10BE180000F0C6F894F800E06378A778E078217914
:10BE280062794EEA03033B4303430B4313430ED1AA
:10BE38000022227008216170DC21A170E270227159
:10BE480062714FF410602146062200F0DBF8114BB6
:10BE58001E70114B1D60114A114B1A604FF470602F
:10BE680001A9042200F0CEF84FF4706001A9042261
:10BE780000F0C8F84FF4807001A9042200F0C2F85D
:10BE8800FFF774FE0022074B1A7003B0F0BD00BF25
:10BE9800E4240020F8240020F424002078563412EA
:10BEA800EC240020BE070020024B1A6801321A60F9
:10BEB800704700BFC4070020044B1A7802705A78F4
:10BEC80042709A788270DB78C3707047D007002080
:10BED800044B1A7802705A7842709A788270DB782C
:10BEE800C3707047CC070020044B1A7802705A7848
:10BEF80042709A788270DB78C3707047C007002060
:10BF0800044B1A7802705A7842709A788270DB78FB
:10BF1800C3707047D4070020014B1868704700BFF2
:10BF2800D800002038B505460C4CA368984723690B
:10BF38009847E369C5F307409847E369C5F30720C5
:10BF48009847E369E8B29847A36998470546636943
:10BF58009847E3689847284638BD00BFE8000020A6
:10BF6800F8B505460E460D4CA368984723699847CF
:10BF780045F00407E369C5F307409847E369C5F34B
:10BF880007209847E369F8B29847E369304698472D
:10BF980063699847E3689847F8BD00BFE800002048
:10BFA800F8B507460E461546154CA3689847236909
:10BFB8009847E369C7F307409847E369C7F3072041
:10BFC8009847E369F8B29847236A43B1626A6AB945
:10BFD80007E0BB69984730550134A4B203E0002458
:10BFE80000E00024064FAC42F3D302E03046294675
:10BFF8009847034C63699847E3689847F8BD00BFC2
:10C00800E80000202DE9F04107460E461546154C7C
:10C01800A36898472369984747F00408E369C7F37A
:10C0280007409847E369C7F307209847E3695FFA31
:10C0380088F09847636A5BB905E0FB69305D98470B
:10C048000134A4B201E00024064FAC42F5D302E06B
:10C05800304629469847034C63699847E3689847F0
:10C06800BDE8F081E8000020F8B50025400100F1A6
:10C07800080606F5005706F504563846FFF752FF3E
:10C08800000284B23046FFF74DFF204484B24CB121
:10C098003846FFF747FF000285B23046FFF742FFF8
:10C0A800284485B2A542E8D12846F8BDF8B5002550
:10C0B800400100F1080606F5185706F51C563846E3
:10C0C800FFF730FF000284B23046FFF72BFF204411
:10C0D80084B24CB13846FFF725FF000285B23046DE
:10C0E800FFF720FF284485B2A542E8D12846F8BDCD
:10C0F8002DE9F8430D46144632B34FEA800909F199
:10C108000106F60006F510573846FFF70BFF804684
:10C1180006F514563046FFF705FF00EB08201FFA16
:10C1280080F809F10200C00000EB082029462246E9
:10C13800FFF768FF4444A4B23846210AFFF710FF0E
:10C148003046E1B2FFF70CFFBDE8F8832DE9F8436C
:10C158000D46144632B34FEA800909F10106F6008C
:10C1680006F520573846FFF7DDFE804606F52456CB
:10C178003046FFF7D7FE00EB08201FFA80F809F1D8
:10C188000300C00000EB082029462246FFF708FFFD
:10C198004444A4B23846210AFFF7E2FE3046E1B231
:10C1A800FFF7DEFEBDE8F883F8B50F46400100F161
:10C1B800080505F520563046FFF7B4FE044605F598
:10C1C80024552846FFF7AEFE00EB0420C419A4B29C
:10C1D8003046210AFFF7C4FE2846E1B2FFF7C0FE49
:10C1E800F8BD00BF70B50546082827D846010836AF
:10C1F80006F5807420461021FFF7B2FE2046FFF7AF
:10C2080091FE0028FAD106F500701F21FFF7A8FE5D
:10C218000122AA400B4B198821EA02021A80002346
:10C22800094A22F81530094A535506F54074204644
:10C23800FFF778FE0028FAD1012000E0FF2040B285
:10C2480070BD00BFDC070020E8070020E0070020E1
:10C258002DE9F04105460F4614461E4608286BD8BE
:10C2680000296BD0022901D9042967D116F0060FDD
:10C2780066D1A6B1012F02D0022F04D00FE016F02C
:10C28800210F0CD15EE016F0200F02D016F0800FBF
:10C298005AD016F0100F02D016F0800F56D028464C
:10C2A800FFF7A0FF4FEA451808F1080826F00F012C
:10C2B80040463943FFF754FE64B9264A1488631C84
:10C2C8009BB213804FF6F072934203D14FF4404271
:10C2D800204B1A8008F58060210AFFF741FE08F517
:10C2E800A060E1B2FFF73CFE08F58074204601210A
:10C2F800FFF736FE2046FFF715FE0028FAD106F0B4
:10C308000106AE40144B1A8816431E800122AA402B
:10C31800124B198821EA02021A800023104A22F8D7
:10C328001530104A535508F540742046FFF7FAFDBA
:10C338000028FAD0E8B20AE0FF2008E0FB2006E077
:10C34800FA2004E0FA2002E0FA2000E0FA2040B2E5
:10C35800BDE8F081E4000020DA070020DC070020B7
:10C36800E8070020E007002070B5064608282BD80B
:10C37800440108342046FFF7D5FD00F00F000128DE
:10C3880024D104F540752846FFF7CCFD13281FD1AA
:10C3980004F5807420460221FFF7E2FD2046FFF7EE
:10C3A800C1FD0028FAD108E02046FFF7BBFD20B9FF
:10C3B8003046FFF717FFFC200BE02846FFF7B2FDD9
:10C3C8001428F1D1012004E0FF2002E0FB2000E066
:10C3D800FD2040B270BD00BF2DE9F04107460D4673
:10C3E800904608285AD8440108342046FFF79AFD99
:10C3F80000F00F00012853D104F540763046FFF7CE
:10C4080091FD13284ED12A786B7803EB0223AA7882
:10C4180002EB0323EA7802EB0323013B13F1030F3A
:10C4280042D8B8F1000F41D004F5406029460422F3
:10C43800FFF7E8FD04F580504FEA1821FFF790FD5B
:10C4480004F588505FFA88F1FFF78AFD04F58075D6
:10C4580028460421FFF784FD2846FFF763FD0028DE
:10C46800FAD1154B1B8843FA07F717F0010F0CD0C8
:10C478001EE02046FFF756FD10F0080F07D02046B3
:10C488000821FFF76DFDF32013E004F50074304632
:10C49800FFF748FD1728ECD101200AE0FF2008E04B
:10C4A800FB2006E0FD2004E0F42002E0F52000E097
:10C4B800002040B2BDE8F081DA07002070B50646DA
:10C4C800082837D8450108352846FFF72BFD00F026
:10C4D8000F00012830D105F5807420460821FFF7A8
:10C4E8003FFD2046FFF71EFD0028FAD10122B24089
:10C4F800144B198821EA02021A80134B1B88334116
:10C5080013F0010F0BD019E02846FFF70BFD10F0D0
:10C51800080F08D03046FFF765FEF3200FE005F559
:10C52800407405F500752046FFF7FCFC0028EBD1A8
:10C53800012004E0FF2002E0FB2000E0002040B2E0
:10C5480070BD00BFDC070020DA0700202DE9F84F96
:10C5580006468B46144608287DD880464FEA401A7E
:10C568000AF1080A5046FFF7DDFC00F00F00012829
:10C5780075D1002C77D00AF540773846FFF7D2FC02
:10C58800172801D01C2872D13E4B1B88334113F069
:10C59800010F1DD00AF500752846FFF7C3FC10F0FF
:10C5A800100F0BD028461021FFF7DAFC0121B1400B
:10C5B800344B1A8822EA01021A8009E010F0080FA9
:10C5C80059D03046FFF70EFE6FF00C00BDE8F88F2B
:10C5D8000AF5F850FFF7A6FC850205F47C45A5424C
:10C5E80028BF2546DFF8A0903046FFF73DFD0446FA
:10C5F8003846FFF797FC172808D01C2806D0304685
:10C60800FFF7F0FD6FF00600BDE8F88FB9F80030CD
:10C6180043FA08F313F0010F01D0A5422ED8A54222
:10C62800E2D8304659462A46FFF762FD0AF5807A75
:10C6380050462021FFF794FC5046FFF773FC002872
:10C64800FAD1012303FA06F60E4B1A8816431E8008
:10C658002846BDE8F88F4FF0FF30BDE8F88F6FF03F
:10C668000400BDE8F88F6FF00D00BDE8F88F6FF09B
:10C678000600BDE8F88F0020BDE8F88F0020BDE86F
:10C68800F88F00BFDC070020DA0700202DE9F04F03
:10C6980083B0054601911446082860D880464FEAC1
:10C6A800401B0BF1080B5846FFF73CFC00F00F004D
:10C6B800012857D1002C58D00BF5F050FFF732FC69
:10C6C800800200F47C43A34228BF234600930BF565
:10C6D80040770BF5F85ADFF8A0902846FFF7E6FCFC
:10C6E80004463846FFF71EFC172818D01C2810D11E
:10C6F800FCB92846FFF7B8FC06465046FFF712FC7F
:10C70800B6EB802F0BD12846FFF76CFD6FF00600C3
:10C718002FE02846FFF766FD6FF0060029E0B9F81C
:10C72800003043FA08F313F0010F00D004B3002CD3
:10C73800D3D0009B9C4228BF1C462846019922461C
:10C74800FFF704FD0BF5807B58464021FFF708FCF6
:10C758005846FFF7E7FB0028FAD1204609E04FF0DA
:10C76800FF3006E06FF0040003E06FF00D0000E01A
:10C77800002003B0BDE8F08FDA0700202DE9F84F5C
:10C7880006468B4691461D46BDF82840082878D8AD
:10C7980080464FEA401A0AF1080A5046FFF7C2FBE2
:10C7A80000F00F00022801D004286ED1B9F1000F63
:10C7B8006FD02B68002B70D0002C72D00AF5407710
:10C7C8003846FFF7AFFB422801D022286DD10AF581
:10C7D800406029460422FFF715FC0AF58050210A1B
:10C7E800FFF7BEFB0AF58850E1B2FFF7B9FB0AF57F
:10C7F800F850FFF797FB850205F47C454D4528BFA7
:10C808004D46DFF8BC903046FFF72EFC044638460C
:10C81800FFF788FB00284CD0B9F8003043FA08F33A
:10C8280013F0010F01D0AC4247D3AC42EBD33046F2
:10C8380059462A46FFF75CFC0AF5807420462021F9
:10C84800FFF78EFB2046FFF76DFB0028FAD10AF5AB
:10C85800007A5046FFF766FB10F0100F06D05046DE
:10C868001021FFF77DFB2846BDE8F88F10F0080F70
:10C87800EFD050460821FFF773FB6FF00C00BDE8BE
:10C88800F88F4FF0FF30BDE8F88F6FF00400BDE877
:10C89800F88F6FF00D00BDE8F88F6FF00B00BDE862
:10C8A800F88F6FF00A00BDE8F88F6FF00600BDE85A
:10C8B800F88F6FF00300BDE8F88F0020BDE8F88F0F
:10C8C800DA0700202DE9F04F85B005460091934620
:10C8D8000193082800F2D88006464FEA401909F16A
:10C8E80008094846FFF71EFB824600F00F03022B9B
:10C8F80002D0042B40F0CB80BBF1000F00F0CA80BF
:10C90800694B33F81530CBB909F54077DFF8A081CA
:10C918002846FFF7CBFB04463846FFF703FB002801
:10C9280000F0BB80B8F80030334113F0010F02D09B
:10C93800002C00F0B580002CEAD000E00024002292
:10C948005A4B5A550AF0070ABAF1020F03D0BAF146
:10C95800040F41D077E0544B33F8153083BB284699
:10C9680002A90822FFF7F2FB09F58074204640214E
:10C97800FFF7F6FA2046FFF7D5FA0028FAD19DF816
:10C988000830019A13709DF8093053709DF80A30E9
:10C9980093709DF80B30D3709DF80C209DF80D30E6
:10C9A80003EB02220E9B1A809DF80E209DF80F3093
:10C9B80003EB02223C4B23F8152080223B4B5A55AF
:10C9C800394B33F815405C4528BF5C46284600992A
:10C9D8002246FFF7BBFB3DE0334B33F8153033BB42
:10C9E800284602A90222FFF7B1FB09F58074204608
:10C9F8004021FFF7B5FA2046FFF794FA0028FAD14C
:10CA08009DF808209DF8093003EB02239BB2264AC3
:10CA180022F8153040F2EA52934205D92846FFF72A
:10CA2800E1FB6FF47A703CE08022204B5A551E4B94
:10CA380033F815405C4528BF5C46284600992246D5
:10CA4800FFF784FB06E028462146FFF7ADFB164BAF
:10CA580023F8154009F5807948464021FFF780FA08
:10CA68004846FFF75FFA0028FAD10F4A32F8153026
:10CA78001B1B9BB222F8153023B10C4B5A5D42F0B8
:10CA880001025A5520460CE04FF0FF3009E06FF0E4
:10CA9800040006E06FF00D0003E06FF0030000E013
:10CAA800002005B0BDE8F08FE8070020E00700206F
:10CAB800DA07002070B504461546082800F28D8074
:10CAC8000C2900F28C80DFE801F0071019222F38BA
:10CAD8008A48585D626A7C0040010830FFF722FAF4
:10CAE80020F00F00287001207EE0400100F5B050D2
:10CAF8000830FFF717FA2870012075E0400100F5AB
:10CB0800A8500830FFF70EFA287001206CE04401A5
:10CB1800083404F59050FFF705FA04F59850FFF72C
:10CB280001FA287001205FE0400100F60840114634
:10CB38000422FFF735FA012056E04401083404F5D1
:10CB48008050FFF7EFF9064604F58850FFF7EAF939
:10CB580000EB06202880012046E0440108342046E6
:10CB6800FFF7E0F900F00F0001283AD104F53C5036
:10CB7800FFF7D8F92880012036E0FFF775FA2880FA
:10CB8800012031E0FFF792FA288001202CE04001D3
:10CB980000F54270FFF7C6F92870012024E0400133
:10CBA8000830FFF7BFF9012805D12046FFF77EFAC4
:10CBB8002880012018E00D4B33F814302B80012019
:10CBC80012E040010830FFF7ADF900F00F0001282E
:10CBD80009D1074B1B5D2B7006E0FF2004E0FE2007
:10CBE80002E0FB2000E0FB2040B270BDE807002017
:10CBF800E0070020704700BF704700BF704700BFC4
:10CC0800704700BF00787047017070470020704778
:10CC1800704700BF704700BF704700BF00B129B917
:10CC2800044B054A1A61054A5A617047014B18615D
:10CC380059617047E800002005CC000809CC0008BD
:10CC4800094A138803F400739BB2002BF9D000B192
:10CC580029B9054B054A9A61054ADA617047024BC2
:10CC68009861D961704700BFE800002015CC000822
:10CC780019CC0008094A138803F400739BB2002BEF
:10CC8800F9D000B129B9054B054A1A62054A5A621A
:10CC98007047024B18625962704700BFE8000020D5
:10CCA8001DCC000821CC000800B587B04FF41060F7
:10CCB80001A90622FFF774F94FF4807005A9042230
:10CCC800FFF76EF94FF4A06004A90422FFF768F992
:10CCD8004FF4706003A90422FFF762F90020802155
:10CCE800FFF73EF90020FFF71DF94FF4106001A986
:10CCF8000622FFF787F94FF4807005A90422FFF791
:10CD080081F94FF4A06004A90422FFF77BF94FF4DE
:10CD1800706003A90422FFF775F907B05DF804FBFA
:10CD280070B506460D46FFF7BFFF3EB91DE059B284
:10CD3800715C0A44D2B20133DBB201E0002213462F
:10CD480059B20729F3DD52B2102A31DC002409E078
:10CD580063B2580100F5F8500830F15CFFF700F9AC
:10CD68000134E4B263B2072BF2DD00201DB306E004
:10CD780059B2695C0A44D2B20133DBB201E0002245
:10CD8800134659B20729F3DD52B2102A12DC0024E7
:10CD980009E063B2580100F5F0500830E95CFFF78C
:10CDA800DFF80134E4B263B2072BF2DD002002E0C1
:10CDB800FF2000E0FF2040B270BD00BF10B5014663
:10CDC800040A4FF4A85001F0F001FFF7C9F84FF436
:10CDD800B8502146FFF7C4F810BD00BF10B54FF496
:10CDE800A850FFF79FF800F0F0044FF4B850FFF791
:10CDF80099F8000280B20444A0B210BD10B50146F3
:10CE0800040A4FF4B050C9B2FFF7AAF84FF4C05063
:10CE18002146FFF7A5F810BD10B54FF4B050FFF745
:10CE280081F804464FF4C050FFF77CF804EB00206B
:10CE380080B210BD08B54FF43850FFF773F800F012
:10CE4800010008BD08B54FF43850FFF76BF800F043
:10CE58003000003018BF012008BD00BF08B54FF4EE
:10CE68003850FFF75FF800F07F014FF43850FFF7B4
:10CE780077F84FF43850FFF755F860F07F014FF41A
:10CE88003850C9B2FFF76CF808BD00BF08B5037881
:10CE9800012B14BF002140214378012B03D141F01D
:10CEA8003801C9B20FE0C378012B07D18378012B71
:10CEB8000CBF41F0180141F0080104E08378012B10
:10CEC80008BF41F010014FF43850FFF749F8FFF759
:10CED800C5FF08BD10B504464FF43850FFF722F8D7
:10CEE800C0F38013237000F03803202B01D0382BB7
:10CEF80002D10122627001E000226270182B03D077
:10CF0800202B01D0102B02D10122A27001E00022B7
:10CF1800A270182B03D0202B01D0082B02D101239B
:10CF2800E37010BD0023E37010BD00BF10B50446C8
:10CF38004FF43850FEF7F6FF10F0400F1CD000F009
:10CF4800C701012C0CBF41F0300141F038014FF40A
:10CF58003850FFF705F8FFF781FF4FF43850FEF718
:10CF6800E1FF012C0CBF00F0300000F03800002871
:10CF780014BF0020FF2000E0FF2040B210BD00BF1A
:10CF880030B583B00C460023009301930F2809D8CD
:10CF9800DFE800F00A0E1D1822272C394755595E84
:10CFA8007763676FFF2071E0FFF77EFE00206DE07A
:10CFB80019B1009101F10804019400980199FFF753
:10CFC800AFFE63E00888FFF7F9FE00205EE0FFF798
:10CFD80005FF2080002059E00888FFF70FFF002098
:10CFE80054E0FFF719FF208000204FE009884FF434
:10CFF8009850090AFEF7B4FF4FF4A0502178FEF7C5
:10D00800AFFF002042E04FF49850FEF78BFF054633
:10D018004FF4A050FEF786FF00EB0520208000208B
:10D0280034E01C4B9A780A70DA784A701A798A7058
:10D038005A79CA709B790B710020487126E0FFF776
:10D048000DFF002022E00846FFF720FF00201DE02A
:10D058000846FFF73FFF002018E00878FFF766FF53
:10D0680014E0FFF7EFFEC0B2FF280CD020700020BC
:10D078000CE0FFF7DFFEC0B2FF2806D020700020CA
:10D0880004E0002002E0FF2000E0FF2040B203B0EF
:10D0980030BD00BFE800002010B504464FF4106012
:10D0A80021460622FEF7AEFF4FF4807004F10E0110
:10D0B8000422FEF7A7FF4FF4A06004F10A0104223E
:10D0C800FEF7A0FF4FF47060A11D0422FEF79AFF3F
:10D0D800A27C064B1A70E27C5A70227D9A70627D9F
:10D0E800DA70A27D024B1A7010BD00BFFC07002049
:10D0F800F807002010B504464FF4106021460622B8
:10D10800FEF74EFF4FF4807004F10E010422FEF783
:10D1180047FF4FF4A06004F10A010422FEF740FF24
:10D128004FF47060A11D0422FEF73AFF064B1A78EF
:10D13800A2745A78E2749A782275DB786375034B87
:10D148001B78A37510BD00BFFC070020F80700205E
:10D1580010B5044630F03A030AD10020FEF7E2FE8B
:10D1680040EA04010020C9B2FEF7FAFE002000E000
:10D17800FF2040B210BD00BF08B50020FEF7D2FE68
:10D1880008BD00BF10B504464FF4D8502178FEF70B
:10D19800E7FE61884FF4C850090AFEF7E1FE4FF434
:10D1A800D050A178FEF7DCFE10BD00BF38B50446AC
:10D1B8004FF4D850FEF7B6FE20704FF4C850FEF773
:10D1C800B1FE05464FF4D050FEF7ACFE00EB05204B
:10D1D800608038BD10B50C46052821D8DFE800F07E
:10D1E80003080D11161B0846FFF756FF002018E02C
:10D1F8000846FFF77FFF002013E00878FFF7A8FF35
:10D208000FE0FFF7B9FF207000200AE00846FFF79B
:10D21800B9FF002005E00846FFF7C8FF002000E03E
:10D22800FF2040B210BD00BF03463038C0B2092805
:10D2380012D9A3F16102D2B2052A03D8A3F157008B
:10D24800C0B27047A3F14102D2B2052A03D8A3F1B4
:10D258003700C0B270471846704700BF70B5044623
:10D268000E46002305E003FB06F50134FFF7DCFF5B
:10D278002B18207808B12028F5D198B270BD00BFCE
:10D2880030B400231D4603E08A4208BF25700133ED
:10D29800C418C25C002AF7D130BC704730B4084CBF
:10D2A8009DF808502570074C206007480160074921
:10D2B8000A80074A13600122064B1A7030BC704777
:10D2C800202500201C2500200425002022250020E0
:10D2D800002500201008002082B002AB03E90300FB
:10D2E800009B044A1360BDF804201344024A1360EB
:10D2F80002B070470C2500202825002010B5094BE6
:10D308001C68094B1B689C4209D220460AF02CF97C
:10D31800C0B2421C2244034B1A60204610BD0020B4
:10D3280010BD00BF0C2500202825002010B504469C
:10D33800194B1878FEF7BAFE002829D0164B187832
:10D34800164B19680522FFF7A1F9052822D1134BBE
:10D358001A68117821701A68527862801868807883
:10D3680042EA002262801868C378A380007943EA01
:10D378000023100A40EA022292B26280180A40EAA8
:10D3880003239BB2A380064809F0FAFF012010BDD1
:10D39800002010BD002010BD202500200025002001
:10D3A8004C960108074B188850B9074A138801336F
:10D3B8009BB2138013B90122034B1A80024B1888C1
:10D3C800704700BFFC24002012080020014B186899
:10D3D800704700BF242500202DE9F84F83460F46EB
:10D3E80090461E460B9D484B1878400100F5427048
:10D3F800FEF798FD172804D044480AF04DF8BDE818
:10D40800F88F17B9FFF7CEFF0746390A41EA072117
:10D4180089B21FFA86FA1FFA85F973190AEB09000F
:10D42800C3F3072242EA002292B2394C206880F8FE
:10D4380000B0206841702068090A81702168CA70AC
:10D448002168120A0A71334859463A4609F098FF8A
:10D458002D4B187821680522FFF778F80746BBF1AD
:10D46800000F4BD0EEB13C2009F0A2FF00244FF092
:10D47800200B0AE018F8040010B109F099FF02E047
:10D48800584609F095FF0134A4B2B442F2D32248B9
:10D498000AF002F81C4B187841465246FFF756F836
:10D4A8000744EDB13C2009F083FF00244FF0200829
:10D4B8000AE00A9B185D10B109F07AFF02E04046C5
:10D4C80009F076FF0134A4B2AC42F2D3124809F055
:10D4D800E3FF0D4B18780A994A46FFF737F80744D7
:10D4E80005367219BA4209D00C48394609F048FF86
:10D4F800054B1878FEF7E2FFBDE8F88FFFF766FFE7
:10D50800074B1860BDE8F88F202500205C960108BD
:10D51800002500206C96010824B601087C960108B5
:10D52800102500202DE9F04389B00290ADF80C10C9
:10D538000023049305930693079302AB93E8030033
:10D54800FFF7CAFEFFF7DAFE0546002800F0EB8079
:10D55800764909F0F7FF38B90021009101911420AC
:10D56800734A4523FFF738FFFFF7C8FE0446002833
:10D5780000F0D9800A21FFF771FEC6B228466D492E
:10D5880009F0E0FFB0B9304600F084FB034604A878
:10D598006949324609F098FF044604A82021FFF79C
:10D5A8006FFE002100910191142004AAA3B2FFF795
:10D5B80013FFB8E02846614909F0C4FFB0B9304606
:10D5C80000F080FB034604A85D49324609F07CFF61
:10D5D800044604A82021FFF753FE00210091019181
:10D5E800142004AAA3B2FFF7F7FE9CE02846554989
:10D5F80009F0A8FFC8B9544809F04EFF304600F0BA
:10D6080093FB034604A85149324609F05DFF0446DE
:10D6180004A82021FFF734FE002100910191142075
:10D6280004AAA3B2FFF7D8FE7DE02846484909F0CE
:10D6380089FF60B9474809F02FFFFFF75FFE0446EE
:10D648000A21FFF70BFE0146304600F077FB28461B
:10D65800414909F077FF002833D039E0FFF74EFE43
:10D668000446394609F06EFF20B93046002100F023
:10D678003DFB1DE02046414609F064FF20B12046ED
:10D68800494609F05FFF20B93046012100F02EFB22
:10D698000EE02046314909F055FF20B930460221F5
:10D6A80000F024FB04E02E483146224609F068FECB
:10D6B800FFF724FE044658B10A21FFF7CFFDC6B292
:10D6C80004E0284FDFF8AC80DFF8AC90002CC5D11F
:10D6D800FFF714FE044630B32846234909F032FF09
:10D6E80078B920460A21FFF7B9FDC4B230460121B6
:10D6F80000F0FCFA3046211C18BF012100F0CEFAD8
:10D7080011E02846194909F01DFF40B920460A21B1
:10D71800FFF7A4FDC1B2304600F0DEFA03E014487A
:10D72800294609F02DFE09B0BDE8F0838C96010862
:10D73800100100209496010898960108A496010803
:10D74800A8960108B4960108B8960108E096010861
:10D75800EC960108F0960108189701082897010827
:10D768002C9701081C970108489701084C97010855
:10D7780050970108209701082497010870B584B0D4
:10D7880002A8FFF7D3FD002875D09DF808101429CA
:10D7980065D8DFE801F00B6464646464146464644D
:10D7A80064646464641E646464641E00BDF80C30C0
:10D7B800052B5CD1314B1878FEF780FE5BE0BDF895
:10D7C8000A100022009201921046C823FFF704FEB7
:10D7D8004DE0BDF80C40FF2C09D929482146FF220D
:10D7E80009F0CEFD254B1878FEF768FE43E0234B81
:10D7F8001878244B19682246FEF748FF844203D064
:10D80800214809F049FE36E0BDF80C301D4A12687F
:10D818000024D4543E2009F0CBFD1A4D20260AE0FE
:10D828002B68185D10B109F0C3FD02E0304609F01D
:10D83800BFFD0134A4B2BDF80C30A342F0D81348A0
:10D8480009F02AFEBDF80A30114C23800D4B1868E8
:10D85800BDF80C10FFF766FE0023238007E00D4893
:10D8680009F08EFD054B1878FEF728FE03E0FFF758
:10D87800ADFD094B186004B070BD00BF2025002025
:10D8880068970108002500209097010824B6010830
:10D89800FC240020A49701081825002010B5044690
:10D8A80048B10C4B1B6883B9FFF790FD2044094B26
:10D8B8001860002010BDFFF789FD064B1B689842D1
:10D8C80005D30020034B186010BD002010BD0120B7
:10D8D80010BD00BF0C0800202DE9F04184B0FFF70F
:10D8E80075FD04460020FFF7D9FF8046002840F068
:10D8F8009980504B1B78CBB9FFF754FD06464E4B29
:10D9080018804E4B1D68284609F02EFE034600225B
:10D9180000920192022031462A46FFF75DFD01225E
:10D92800444B1A70FFF752FD454B1860FFF74EFD48
:10D93800434B1B6803F59C530833984208D202A84E
:10D94800FFF7F4FC002870D000223A4B1A7005E06B
:10D958000123ADF80C300022364B1A709DF80830C0
:10D968005BB9BDF80A20344B1B889A4205D1BDF833
:10D978000C30C82B43D00B2B41D0BDF80C1001291B
:10D9880003D1304809F088FD30E0092903D12E4839
:10D9980009F082FD2AE02D4809F0F2FCFF228DF8FB
:10D9A80008200024ADF80A40ADF80C40284B19684F
:10D9B8000A701A68BDF80A1051701A68BDF80A1082
:10D9C80091701A68BDF80C10D1701B68BDF80C2056
:10D9D8001A71204F1E4E052506E0387831682A4610
:10D9E800FEF7B4FD0134E4B2092CF6D9194B1878C6
:10D9F800FEF764FD41F28830FFF750FF16E0FFF7AD
:10DA0800E5FC154B1860154D2860154B1860154836
:10DA180009F042FD29681448091B09F0B1FC4FF0D0
:10DA2800010803E04FF0000800E08046404604B0DB
:10DA3800BDE8F08108080020000800201C2500200F
:10DA480004080020C0970108CC970108E097010856
:10DA58000025002020250020102500201825002062
:10DA680014250020FC9701080498010870B586B0B9
:10DA7800764B1B78002B00F0E680754B1878400138
:10DA880000F54270FEF74EFA1C2800F2DC80DFE851
:10DA980010F0AE00DA00DA00DA00DA00DA00DA00B4
:10DAA800DA00DA00DA00DA00DA00DA00DA00DA009E
:10DAB800DA00DA00DA00DA00C300DA00DA00DA00A5
:10DAC8001D00DA00DA00DA00DA00A500604B1878E9
:10DAD800400100F50270FEF725FA10F0010F30D072
:10DAE8005B4C2078400100F502700121FEF738FAFE
:10DAF8002078400100F6084005A90422FEF750FAF4
:10DB08002078400100F580500830FEF70BFA0546F2
:10DB18002078400100F588500830FEF703FA00EB42
:10DB2800052085B29DF814209DF815309DF81660E3
:10DB38009DF817002178009601900295454809F054
:10DB48001FFC454B1B786BB9FFF7C6FE434B18709B
:10DB5800002878D00122404B1A7041483C4B197874
:10DB680009F00EFC3D4B1B780BB1FFF707FEFFF7E2
:10DB78002DFC04463B4B1968431A43F6A402934212
:10DB88000CD9394809F0FCFB0023334A1370334A97
:10DB980013702F4B1878FEF791FC54E042F2107284
:10DBA800934206D8314B1A68821A42F210739A428D
:10DBB80049D92F4B1A68A21A40F2DC539A4242D92B
:10DBC8002C4809F069FC00230093019306201946AC
:10DBD8001A46FFF701FC264B1C6034E01C4C264813
:10DBE800217809F0CDFB2078FEF768FC2BE00023B4
:10DBF800194A1370194A1370154C20781F490A885E
:10DC0800551C0D800121FEF723FB217888421AD18B
:10DC18001B4809F0B5FB16E00D4E1A48317809F09B
:10DC2800AFFB194D2868017842788378C078009056
:10DC3800164C20880190164809F0A2FB3078296814
:10DC48002288FEF7C9FB06B070BD00BF100800208F
:10DC58002025002018980108140800200908002031
:10DC680044980108182500206C9801081025002008
:10DC780014250020909801089C980108580100205C
:10DC8800B8980108D498010804250020222500200E
:10DC98003098010808B502F005FF08BD08B5084B23
:10DCA80003449974012902D102F0D0FE02E009B9B7
:10DCB80002F0E2FE02484FF4DB7103F003FD08BDF9
:10DCC800D428002008B50E2886BF0E38C0B2002020
:10DCD80003F086FD08BD00BF08B503460A460248A2
:10DCE800194609F04DFB08BDF098010808B521B99F
:10DCF8000C4B034401229A700CE0022904D1094B11
:10DD0800034401229A7005E0012903D1054B03441D
:10DD180002229A7002F070FE02484FF4DB7103F0A1
:10DD2800D1FC08BDD428002010B50446024821467D
:10DD380009F026FB204610BD2099010808B50346C6
:10DD48000A460248194609F01BFB08BD3899010824
:10DD580010B586B004F05EFE04460DF10600FEF72D
:10DD6800ABF80DF10E00FEF7B3F80DF10A00FEF75F
:10DD7800BBF80DF11200FEF7C3F8684604F1210163
:10DD8800062204F0F3FE04F127000DF10601042237
:10DD980004F0F0FE04F12B000DF10E01042204F052
:10DDA800E9FE04F12F000DF10A01042204F0E2FE5D
:10DDB80004F14F000DF11201042204F0DBFE94F887
:10DDC8004D301BB102238DF8163002E001238DF887
:10DDD800163000206946FFF7FDF906B010BD00BFF8
:10DDE800704700BF04E00A7802701A46013101301A
:10DDF800531E002AF7D17047C9B202E001701A46D3
:10DE08000130531E002AF9D1704700BF70B4034691
:10DE1800002001E029463346541E32B15E1C1878B2
:10DE28004D1C0B782246C01AF4D070BC704700BF56
:10DE380000E00130037813B15AB28A42F9D158B2DE
:10DE4800704700BFCA7E8B7E43EA02230278032A0A
:10DE580005D1487D0A7D42EA002243EA024318467A
:10DE6800704700BF8176C1F30723C376090C01759B
:10DE7800090A4175704700BFF0B40C7804F03F04FC
:10DE8800013C04EB440304EB830401260023154FF3
:10DE98004FF6FF7CFA5C551C4D5D8A5C42EA052210
:10DEA80036B1FE2C14D820F814201646013401E0AF
:10DEB80062450FD101330C2BECD90B7813F0400FCE
:10DEC8000AD0FE2C0AD8002320F81430012006E0DE
:10DED800002004E0002002E0012000E00020F0BC67
:10DEE800704700BF449A01082DE9F0014B730F23D6
:10DEF800CB7200240C738C76CC76531E03EB43064E
:10DF080003EB860623464FF6FF77DFF84480BB42D3
:10DF18001CBF30F81630013618F804504B5501353F
:10DF2800C3F3072C01F805C0002B08BF3B4601349A
:10DF38000C2CECD94FF6FF74A34202D030F81630FF
:10DF48000BB942F040020A70BDE8F001704700BF0B
:10DF5800449A0108F0B583B0064617461C460B22C2
:10DF6800FFF740FF052C13D816E0023711460CE0E6
:10DF780003F0010505EB44045B0814F4803F1CBF63
:10DF880084F4883484F0210401310F29F0D900E0A9
:10DF980000223B88002BE8D1072100E0114604F05D
:10DFA8000F0202F13003392B88BF02F137034A1EF2
:10DFB80002A8084400F8083C2409EFD17E2002ABEF
:10DFC800134403F8080C0023881E07E07F31C9B208
:10DFD8007D2902D8984206D001330133934202D2F8
:10DFE800F15C2029F2D12024591C3344072A05D892
:10DFF80002A8104410F8080C013200E020461870FE
:10E008000B460729F0D903B0F0BD00BF0B2200234F
:10E01800D90141EA530301780B4403F0FF030130AF
:10E02800013AF5D11846704710B4046824B94FF086
:10E03800FF3323E0013200E022461378D9B21F29CA
:10E0480002D959B23A29F5D15BB23A2B15D1611CE4
:10E0580094F90030303B092B06D8914207D1012BA7
:10E0680008D80132026009E04FF0FF3306E04FF0B4
:10E07800FF3303E04FF0FF3300E0002318465DF85C
:10E08800044B70472DE9F0410446037913B3C56A80
:10E0980000F13007407839462A460123FAF70CFE8A
:10E0A800D8B900232371236AEA1AA3699A4217D2BE
:10E0B800E6784FF0010808E0A2691544607839460F
:10E0C8002A464346FAF7F8FD013E012EF4D800200F
:10E0D800BDE8F0810020BDE8F0810120BDE8F081B5
:10E0E8000020BDE8F08100BF70B504460D46C36A44
:10E0F8008B4212D0FFF7C6FF064678B9607804F164
:10E1080030012A460123FAF7BBFD002818BF012673
:10E1180018BF4FF0FF35E56200E00026304670BDBD
:10E1280010B50446002303714FF0FF33C362FFF7B5
:10E13800DBFF58BB94F82F2294F82E3243EA0222D0
:10E1480012B2154B9A4223D194F8692094F868309A
:10E158001B0443EA026394F8672043EA022294F816
:10E1680066301A4322F07F420C4B9A4212D094F840
:10E1780084301B0494F8830094F8822043EA002337
:10E1880013430648181A18BF012010BD032010BDFC
:10E19800022010BD002010BD55AAFFFF46415400C3
:10E1A80008B588B103688BB1197889B1D988828894
:10E1B80091420FD15878FAF761FD00F0010000286C
:10E1C8000CBF0020032008BD092008BD092008BD98
:10E1D800092008BD092008BD2DE9F04184B0054695
:10E1E8001746002303600846FFF71EFF061EC0F20D
:10E1F8009781894B53F82640002C00F093812C60BE
:10E20800237883B16078FAF739FD10F0010F0AD14D
:10E21800002F00F0898100F00400C0B2002814BF6C
:10E228000A2000209FE1002323707C4B13F816007E
:10E238006070FAF721FD10F0010F40F077811FB1EF
:10E2480010F0040F40F0748120460021FFF768FFAA
:10E25800012822D0002844D1704B03EB46035B7899
:10E26800EBB900273EE004EB031292F8F21102F535
:10E27800F77251B1D07A917A090441EA0061507A73
:10E2880041EA0021127A114300E0294604A800EB74
:10E29800830242F8101C013303E0002300E000234E
:10E2A8000025032BDFD95D4B03EB46035D7805B1F1
:10E2B800013D4FF00208594B03EB460604AA02EB56
:10E2C800850353F8107C27B120463946FFF728FF0D
:10E2D80000E0404673782BB920B10135032DEDD904
:10E2E80000E00027032800F02581002840F0248161
:10E2F80094F83C2094F83B3043EA02231BB2B3F570
:10E30800007F40F01B8194F8472094F8463053EA88
:10E3180002230DD194F8572094F856301B0443EA91
:10E32800026394F8552043EA022294F854301343C8
:10E33800A36194F84020E270511EC9B2012900F28D
:10E34800FF8003FB02FC94F83D00A070002800F059
:10E35800F980421E104240F0F78094F8421094F879
:10E36800412042EA0121218111F00F0F40F0EE8097
:10E3780094F8445094F8432052EA05250DD194F8B6
:10E38800535094F85220120442EA056294F851500E
:10E3980042EA052594F85020154394F83F8094F8F4
:10E3A8003E2052EA082800F0D38008EB0C0606EB62
:10E3B8001116B542C0F0CE80AD1BB5FBF0F00028B9
:10E3C80000F0CA8040F6F575A8428CBF02250125E9
:10E3D8004FF6F572904288BF0325821C6261E7619F
:10E3E80007EB080020623E44A662032D18D10029DD
:10E3F80040F0B48094F85F0094F85E10090441EA94
:10E40800006194F85D0041EA002094F85C10014333
:10E418006162920012E000BF1C0A00205C0100202B
:10E42800002900F09D8060446062022D0FBF5200F9
:10E4380002EB420102F0010202EB510202F2FF126A
:10E44800B3EB522FC0F08E804FF0FF332361E360AF
:10E4580080236371032D5AD194F8612094F86030B9
:10E4680043EA02231BB2012B51D12046791CFFF746
:10E478003BFE00284BD10023637194F82F2294F8B7
:10E488002E3243EA022212B2384B9A423FD194F814
:10E49800332094F832301B0443EA026394F83120A5
:10E4A80043EA022294F830301A43314B9A422ED173
:10E4B80094F8172294F816321B0443EA026394F87E
:10E4C800152243EA022294F814321A43294B9A423D
:10E4D8001DD194F81B2294F81A321B0443EA0263F4
:10E4E80094F8192243EA022294F81832134323615C
:10E4F80094F81F2294F81E321B0443EA026394F82E
:10E508001D2243EA022294F81C321343E36025706B
:10E51800194A138801339BB21380E380002022E05C
:10E528000B2020E00C201EE000201CE003201AE055
:10E538000A2018E0012016E00D2014E00D2012E05A
:10E548000D2010E00D200EE00D200CE00D200AE05B
:10E558000D2008E00D2006E00D2004E00D2002E06B
:10E568000D2000E00D2004B0BDE8F08155AAFFFFA2
:10E578005252614172724161180900202DE9F0413F
:10E588000F4601F109040369002B3FD045690023B8
:10E598004FF02E0C21E05A1CEB5C5EB2202E1BD0F3
:10E5A800052E08BFE523092A04BF84F800C00134FA
:10E5B800D9B2A1F14106F6B2192E0BD895F80C8004
:10E5C800092A34BF0826102618EA060F1CBF01F1D5
:10E5D8002003DBB22370013413460A2BDBD9EB7A14
:10E5E8003B72EA7FAB7F1B0443EA02636A7F43EA1C
:10E5F80002232A7F13433B606A7E2B7E43EA022371
:10E60800BB80EA7DAB7D43EA0223FB8000232370B5
:10E61800BD6975B303690BB3FB690BB3028C4FF685
:10E62800FF739A421ED0C3690024A04611E04146F8
:10E6380002F0AEF80346B8B1FF2803D9C0F30722A9
:10E648002A550134FA69013AA2420FD92B553346AB
:10E6580001349E1C18880028E9D108E0002406E04F
:10E66800002404E0002402E0002400E00024002349
:10E678002B55BDE8F08100BF2DE9F04F83B0009025
:10E688008B460D6800E001352B785AB22F2AFAD054
:10E698005C2AF8D00099D1F81C80002426464FF057
:10E6A8000109DFF850A2731CA85780B21F2837D978
:10E6B8002F2835D05C2833D0FE2C00F20C81C0B254
:10E6C80000F17F02D2B27D2A15D85E1CEB5CA3F163
:10E6D8004102D2B2192A0AD9A3F16102D2B2192A87
:10E6E80005D903F17F02D2B27D2A00F2F68003EB4E
:10E6F800002080B200E01E46494602F049F807466D
:10E70800002800F0EC807F2806D850463946FFF7ED
:10E718008FFB002840F0E58028F814700134C2E728
:10E728002B44CBF800301F288CBF002604266FF03E
:10E73800004207E0A31838F81330202B01D02E2B05
:10E7480002D1013C002CF5D1002C00F0CC80002532
:10E7580028F81450009A906920210B22FFF74CFBEF
:10E768002B4600E0013338F81320202AFAD02E2A4D
:10E77800F8D023B146F0030601E0013C01E06FF058
:10E78800004154B1621838F812202E2AF5D14FF002
:10E7980008094FF0000AD34604E04FF008094FF08B
:10E7A800000AD34601945F1C38F81350002D67D037
:10E7B800202D03D02E2D05D1A74203D046F0030605
:10E7C8003B46F0E7CA4501D2A74215D1B9F10B0F74
:10E7D80002D146F0030653E0A74218BF46F00306ED
:10E7E800A7424DD84FEA8B0B5FFA8BFB019B4FF08A
:10E7F8000B094FF0080AD6E77F2D08D9284601F003
:10E80800E3FF002101F0C4FF054646F00206FF2D94
:10E8180011D909F1FF33534504D846F003063B46A6
:10E82800CA46C0E7009B9A690AF10103C5F30721AC
:10E8380002F80A101DE025B12D482946FFF7F8FA1D
:10E8480020B146F0030653465F2512E0A5F14103C7
:10E858009BB2192B03D84BF0020B534609E0A5F1E4
:10E8680061039BB2192B9EBF4BF0010B203DADB24B
:10E87800534600998A6903F1010AD5543B4692E749
:10E88800009A93691A78E52A04BF05221A70B9F12B
:10E89800080F04BF4FEA8B0B5FFA8BFB0BF00C03DE
:10E8A8000C2B03D00BF00302032A01D146F0020619
:10E8B80016F0020F0AD10BF0030BBBF1010F08BFD2
:10E8C80046F01006042B08BF46F0080600998B692D
:10E8D800DE72002008E0062006E0062004E006209C
:10E8E80002E0062000E0062003B0BDE8F08F00BF7C
:10E8F8007C990108709901082DE9F84F82460D4668
:10E908000F7827F04007013F07EB470307EB830722
:10E9180001260024DFF874804FF6FF7918F80430D8
:10E928005A1CA85CEB5C43EA002076B101F04CFF6E
:10E938000646FE2F1BD807F1010B3AF8170001F025
:10E9480043FFB04216D15F4601E0484515D1013476
:10E958000C2CE3D92B7813F0400F11D09EB13AF864
:10E968001700D0F1010038BF0020BDE8F88F002063
:10E97800BDE8F88F0020BDE8F88F0020BDE8F88FCB
:10E988000120BDE8F88F0120BDE8F88F449A0108FE
:10E9980070B50546FFF776FB0446002855D12B785D
:10E9A800032B4AD16B79012B47D105F1300630464C
:10E9B80000214FF40072FFF71FFA552385F82E3215
:10E9C800AA2385F82F32522385F8303085F8313064
:10E9D800612385F83230412285F83320722185F889
:10E9E800141285F8151285F8162285F817322B6946
:10E9F80085F81832C3F3072285F81922C3F30742B2
:10EA080085F81A221B0E85F81B32EB6885F81C3234
:10EA1800C3F3072285F81D22C3F3074285F81E2297
:10EA28001B0E85F81F32EA690132EA6268783146BE
:10EA38000123FAF741F900236B71687800210A462F
:10EA4800FAF760F9002818BF0124204670BD00BFFE
:10EA580002394369023B8B4283BF8278836A01FB98
:10EA680002300020704700BFF8B505460C46012962
:10EA78005AD943698B4259D90378022B28D0032BE2
:10EA880037D0012B54D101EB5106016A01EB562115
:10EA9800FFF72AFB00284DD1771CC6F308062E4441
:10EAA80096F83060296A284601EB5721FFF71CFBCE
:10EAB800002842D1C7F308073D4495F8300046EADC
:10EAC800002014F0010F14BF0009C0F30B00F8BDBB
:10EAD800016A01EB1421FFF707FB88BB640004F40B
:10EAE800FF742B1993F8310093F8303043EA002073
:10EAF800F8BD016A01EBD411FFF7F6FA18BBA400C0
:10EB080004F4FE7404F130032B44D8789A78120484
:10EB180042EA0062587842EA00202C4494F83030E7
:10EB2800184320F07040F8BD0120F8BD0120F8BD61
:10EB38000120F8BD4FF0FF30F8BD4FF0FF30F8BDB1
:10EB48004FF0FF30F8BD4FF0FF30F8BDF8B505467F
:10EB58000E46E9808468012C34D003685A69A242C1
:10EB680032D91CB91A78032A08BF5C6A24B91A89F1
:10EB7800B2422BD9586A17E09F783F010EE0286807
:10EB88002146FFF771FF0446B0F1FF3F20D001286E
:10EB980020D92B685B6983421ED9F61BBE42EED290
:10EBA80028682146FFF754FFEC60B8B100EB161057
:10EBB80028612B6806F00F0603EB461330336B61B0
:10EBC8000020F8BD0220F8BD0220F8BD0220F8BDE3
:10EBD8000120F8BD0220F8BD0220F8BD0220F8BDD2
:10EBE8002DE9F04105460C46164601297CD94369B2
:10EBF8008B427BD90378022B42D0032B54D0012BB4
:10EC080076D101EB5107016A01EB5721FFF76CFA46
:10EC1800034600286DD107F10108C7F3080714F06F
:10EC2800010409D0EB1993F83020F3B202F00F0277
:10EC380042EA0313DBB200E0F3B22F4487F8303026
:10EC480001232B71296A284601EB5821FFF74CFA5A
:10EC5800034600284DD1C8F3080814B1C6F30716B7
:10EC680008E005EB080292F8302022F00F02C6F304
:10EC780003261643A84488F8306001222A7138E038
:10EC8800016A01EB1421FFF72FFA034688BB6400E1
:10EC980004F4FF742A1982F83060C6F3072682F854
:10ECA800316001222A7124E0016A01EBD411FFF7D7
:10ECB8001BFA0346E8B9A40004F4FE7404F1300218
:10ECC8002A44D17809062C4401F070410E4384F897
:10ECD8003060C6F307215170C6F307419170360EB4
:10ECE800D67001222A7104E0022302E0022300E028
:10ECF80002231846BDE8F0812DE9F0410546884613
:10ED080031B9C66886B14369B34298BF01260CE0A1
:10ED1800FFF7AAFE012844D9B0F1FF3F4CD06B6938
:10ED2800834249D8464600E001263446022701348A
:10ED38006B69A34202D8012E36D93C4628462146A3
:10ED4800FFF792FE38B1B0F1FF3F30D0012830D044
:10ED5800B442ECD12FE0284621466FF07042FFF70D
:10ED68003FFF034640B9B8F1000F05D02846414699
:10ED78002246FFF735FF03465BB9EC602B69B3F118
:10ED8800FF3F0BD0013B2B616B7943F001036B71A3
:10ED980004E0012B14BF01244FF0FF342046BDE8E6
:10EDA800F0810120BDE8F0810020BDE8F081BDE8D8
:10EDB800F081BDE8F0810020BDE8F0812DE9F8433D
:10EDC80004460E46C5880135ABB2002B66D00369F0
:10EDD800002B66D015F00F0757D101330361C168C6
:10EDE80021B903681B89AB425ED94EE0006883787D
:10EDF800013B13EA151348D1FFF736FE8046012878
:10EE080055D9B0F1FF3F55D020684369434535D8FF
:10EE1800002E52D0E168FFF76FFF804600284FD0E0
:10EE2800012850D0B0F1FF3F50D02068FFF72AF9F1
:10EE380000284ED12068303000214FF40072FEF7D0
:10EE4800DBFF266830464146FFF702FEF0620026E7
:10EE58004FF001090BE083F804902068FFF712F9DE
:10EE6800002839D12368DA6A0132DA620136236868
:10EE78009A78B242EFD8DA6A921BDA62C4F80C8048
:10EE880020684146FFF7E4FD2061E580236803EB35
:10EE98004713303363610020BDE8F8830420BDE8E0
:10EEA800F8830420BDE8F8830420BDE8F883022035
:10EEB800BDE8F8830120BDE8F8830420BDE8F883A5
:10EEC8000720BDE8F8830220BDE8F8830120BDE8EB
:10EED800F8830120BDE8F8830120BDE8F88300BF6E
:10EEE8002DE9F84F04460021FFF730FE002861D1D4
:10EEF8004FF6FF7323844FF0FF0A57469946D046D2
:10EF08004FF00B0B20682169FFF7EEF80646002842
:10EF18004DD165692B78002B48D0EA7A02F03F0181
:10EF2800E52B04D012F0080F05D00F2903D0A4F860
:10EF38002090474632E00F291DD1E06970B313F0E5
:10EF4800400F06D095F80DA003F0BF03E288228495
:10EF58001F46BB4209D16B7B534508D12946FFF7B1
:10EF6800CBFC30B1013FFFB218E0474616E04746F8
:10EF780014E0474612E027B92846FFF747F85045FE
:10EF880015D0A169CB7A13F0010F04D128465A464F
:10EF9800FEF73CFF58B1A4F82090474620460021D0
:10EFA800FFF70CFF06460028ACD000E004263046E8
:10EFB800BDE8F88FBDE8F88F10B582B0044601911E
:10EFC8000B785AB22F2A01D05C2A01D10131019164
:10EFD8000023A360019B1B781F2B07D82046002124
:10EFE800FFF7B4FD03460022626123E0204601A931
:10EFF800FFF742FB0346E8B92046FFF771FFA36914
:10F00800DA7A034640B1042814D102F00402D2B2DD
:10F01800002A08BF05230DE012F0040F0AD1616928
:10F02800CB7A13F0100F04D02068FEF70BFFA06016
:10F03800DCE70523184602B010BD00BF2DE9F041FA
:10F0480004460F460021FFF781FD0246C8B9002596
:10F05800A846012620682169FFF746F8024680B9CC
:10F0680063691B78E52B00D01BB90135BD4201D17E
:10F0780007E0454620463146FFF7A0FE0246002835
:10F08800E8D0042A14BF10460720BDE8F08100BF6D
:10F098002DE9F04385B005468769C66901A8394658
:10F0A8000C22FEF79FFE9DF80F3013F0010F1BD0C6
:10F0B8000023FB72EB6101240BE0384601A93246BC
:10F0C8002346FEF747FF2846FFF70AFF804610B998
:10F0D8000134632CF1D9642C63D0B8F1040F62D1E8
:10F0E8009DF80F30FB72EE619DF80F3013F0020FA0
:10F0F80003D101260CE0013300E0002336F8132089
:10F10800002AF8D103F11906294AA2FB0636B608E7
:10F1180028463146FFF792FF044630BB013E24D013
:10F12800E9882846891BFFF711FD0446E8B9A86954
:10F13800FEF76CFF81464FF001080027286829690F
:10F14800FEF7D2FF044680B9E8696969F2B24B4616
:10F15800FEF7CAFE2A6882F8048028463946FFF777
:10F168002DFE044608B9013EE8D1C4B928682969CA
:10F17800FEF7BAFF044690B9686900212022FEF71D
:10F188003BFE6869A9690B22FEF72CFE6B69AA6928
:10F19800D27A02F018021A732B6801221A712046DB
:10F1A80002E0072000E0404605B0BDE8F08300BF5C
:10F1B8004FECC44E2DE9F047044689464FF0FF0A4C
:10F1C80056460425D04600274BE02068FEF78CFF02
:10F1D800054600284AD161690B78002B45D0CA7AC8
:10F1E80002F03F02E52B31D02E2B31D022F0200047
:10F1F800082814BF0020012048452BD10F2A1BD115
:10F2080013F0400F06D091F80DA003F0BF03E28879
:10F2180022841E46B34209D14B7B534508D1E0698D
:10F22800FEF72AFE30B1013EF6B214E0464612E07F
:10F23800464610E046460EE026B90846FEF7E6FECA
:10F24800504513D04FF6FF7323840FE0464602E083
:10F25800464600E0464620463946FFF7AFFD0546DC
:10F2680020B921690029B0D100E004250DB100239F
:10F2780023612846BDE8F0872DE9F8430446C7888E
:10F28800018C4FF6FF73994208BF3946FFF75EFCC1
:10F29800054610BB00264FF020094FF0E50820680E
:10F2A8002169FEF721FF0546A0B9606931464A4643
:10F2B800FEF7A2FD636983F80080236801221A71B2
:10F2C800E388BB4206D220463146FFF777FD054664
:10F2D8000028E4D0042D08BF02252846BDE8F8839D
:10F2E8002DE9F04104460D46012926D943698B4290
:10F2F80025D90027B8461CE020462946FFF7B4FB6D
:10F30800064608B301281CD0B0F1FF3F1BD02046A9
:10F3180029464246FFF764FC0746A8B92369B3F1BA
:10F32800FF3F05D001332361637943F00103637123
:10F3380035466369AB42DFD806E0022704E00227BE
:10F3480002E0022700E001273846BDE8F08100BF4F
:10F3580010B584B001900091144604A840F8041D2B
:10F36800FEF762FE002816DB0E4B53F820300BB177
:10F3780000221A70019B0BB100221A70019B094AE6
:10F3880042F820304BB1012C09D101A8694600226E
:10F39800FEF722FF04E00B2002E0002000E000203E
:10F3A80004B010BD1C0A00202DE9F043ADF50F7D17
:10F3B800019115460446002800F0A480002303604C
:10F3C80002F01F0885A801A902F01E02FEF704FF3B
:10F3D8000646002840F0948082AB8B9302AB8C9356
:10F3E80085A80199FFF7E8FD8A9F064610B9002F06
:10F3F80008BF062615F01C0F4AD04EB1042E03D1C3
:10F4080085A8FFF745FE064648F008088A9F0BE0E6
:10F41800FB7A13F0110F06D105F00405EDB2002DAB
:10F4280018BF082600E00726002E40D118F0080F64
:10F438003DD0F9F7ABFCB873C0F30723FB73C0F3F7
:10F4480007433B74000E78740025FD723D777D7785
:10F45800BD77FD7785983946FEF7F4FC8146384636
:10F468002946FEF7FFFC859801220271B9F1000FC9
:10F478001DD0C56A4946FFF733FF0646B8B98598D7
:10F4880009F1FF33C3602946FEF72EFE06460EE05B
:10F498006EB9FB7A13F0100F08D115F0020F06D0E1
:10F4A80003F00103002B18BF072600E0042646B925
:10F4B80018F0080F18BF48F02008859BDB6AE36145
:10F4C8002762EEB984F806804FF0000884F80780B8
:10F4D800859D28463946FEF7B5FC2061FA7FBB7F3B
:10F4E8001B0443EA02637A7F43EA02233A7F134309
:10F4F800E360C4F80880C4F818802560EB88A3800E
:10F50800304600E009200DF50F7DBDE8F08300BF0F
:10F518002DE9F04F83B004460F4690461E4600235F
:10F528003360FEF73DFE002840F0A780E079002810
:10F5380040F0A580A37913F0010F00F09F80A36825
:10F54800E568ED1A454528BF454604F124030193B3
:10F558008EE0A368C3F30802002A72D1206890F8ED
:10F5680002A00AF1FF3A5FFA8AFA1AEA532A11D17D
:10F578000BB9206902E06169FFF776FA012802D821
:10F588000220E0717BE0B0F1FF3F02D10120E07181
:10F5980075E06061D4F8008040466169FFF758FA69
:10F5A800814610B90220E07169E0D1445FEA552B29
:10F5B80025D00AEB0B0298F802309A4288BFCAEBB2
:10F5C800030B98F8010039464A465B46F9F758FBA1
:10F5D80010B10120E07152E0A37913F0400F0BD075
:10F5E800A369C9EB0300584506D207EB40200199EF
:10F5F8004FF40072FEF7F6FB4FEA4B2B2FE0A2699F
:10F608004A451CD0A37913F0400F0DD098F801009B
:10F6180001990123F9F750FB10B10120E0712EE0A8
:10F62800A37923F04003A3712368587801994A46C7
:10F638000123F9F725FB10B10120E0711FE0C4F8A0
:10F648001890A168C1F30801C1F5007BAB4528BF3C
:10F65800AB462144384624315A46FEF7C3FB5F4483
:10F66800A3685B44A36033685B443360CBEB050558
:10F67800002D7FF46EAF002001E000E0072003B00A
:10F68800BDE8F08F2DE9F04F83B004460F461546CC
:10F698001E4600233360FEF783FD002840F0C58036
:10F6A800E079002840F0C380A37913F0020F00F03E
:10F6B800BD80A3685A19934288BF002504F124032A
:10F6C8000193A4E0A368C3F30802002A40F08480F1
:10F6D800206890F802B00BF1FF3B5FFA8BFB1BEA46
:10F6E800532B1DD133B9236943B90021FFF704FB1C
:10F6F800034603E06169FFF7FFFA0346002B00F0B9
:10F708008980012B02D10220E07190E0B3F1FF3F24
:10F7180002D10120E0718AE06361226902B92361A4
:10F72800A37913F0400F0ED0236858780199A26985
:10F738000123F9F7C1FA10B10120E07177E0A3794C
:10F7480023F04003A371D4F8008040466169FFF7B5
:10F758007FF9814610B90220E07168E0D9445FEA78
:10F76800552A25D00BEB0A0298F802309A4288BF36
:10F77800CBEB030A98F8010039464A465346F9F795
:10F788009BFA10B10120E07151E0A369C9EB0301B4
:10F7980051450AD2019807EB41214FF40072FEF758
:10F7A80021FBA37923F04003A3714FEA4A2A25E0FD
:10F7B800A3694B450ED0A268E3689A420AD298F82A
:10F7C800010001994A460123F9F75AFA10B10120BC
:10F7D800E0712CE0C4F81890A068C0F30800C0F5E8
:10F7E800007AAA4528BFAA46204424303946524602
:10F7F800FEF7F8FAA37943F04003A3715744A368CE
:10F808005344A360336853443360CAEB0505002DA5
:10F818007FF458AFA368E268934288BFE360A37996
:10F8280043F02003A371002001E000E0072003B0AB
:10F83800BDE8F08F38B50446FEF7B2FC0346002851
:10F8480045D1A27912F0200F41D012F0400F0DD00F
:10F85800214651F8243B5878A2690123F9F72CFA7C
:10F86800002836D1A37923F04003A3712068E16909
:10F87800FEF73AFC034650BB256AEB7A43F02003B7
:10F88800EB72237B2B77A3891B0A6B77A37BAB7760
:10F89800E37BEB7728462169FEF7E4FAF9F776FA75
:10F8A800A875C0F30723EB75C0F307432B76000E4A
:10F8B80068760023AB74EB74A37923F02003A3715B
:10F8C800236801221A712068FFF762F80346184678
:10F8D80038BD012038BD00BF10B50446FFF7AAFFA8
:10F8E800034630B92046FEF75BFC034608B9002200
:10F8F8002260184610BD00BFF8B504460D46FEF755
:10F908004FFC0746002840F0A580E079002840F029
:10F91800A180E368AB4206D2A27902F00202D2B219
:10F92800002A08BF1D46A2680023A360002D5CD0F2
:10F938002068867876026AB1691EB1FBF6F1013A51
:10F94800B2FBF6F3994205D373421A40A260AD1A8E
:10F95800616911E0216971B9FFF7CEF90146012803
:10F9680002D10220E071F8BDB0F1FF3F02D10120C1
:10F97800E071F8BD2061616119BB002538E0A2790A
:10F9880012F0020F05D02068FFF7B6F9014620B93A
:10F998001AE02068FFF768F80146B1F1FF3F02D18D
:10F9A8000120E071F8BD012903D9226852698A4211
:10F9B80002D80220E071F8BD6161A2683244A260F9
:10F9C800AD1BB542DBD800E03546A2682A44A260E8
:10F9D800C5F308025AB12068FFF73AF810B90220B7
:10F9E800E071F8BD00EB552502E0002500E0002598
:10F9F800A368C3F3080313B3A269AA421FD0A3796B
:10FA080013F0400F0ED0214651F8243B58780123BB
:10FA1800F9F752F910B10120E071F8BDA37923F08C
:10FA28004003A371214651F8243B58782A46012304
:10FA3800F9F726F910B10120E071F8BDA561A368B6
:10FA4800E268934204D9E360A37943F02003A371E9
:10FA58003846F8BDF8BD00BF30B5ADF5077D01915A
:10FA6800054600282FD085A801A90022FEF7B4FB7F
:10FA7800044618BB859B2B6082ABAB6102ABEB6184
:10FA880028460199FFF798FA0446A0B9696949B16F
:10FA9800CB7A13F0100F04D08598FEF7D3F9A8603D
:10FAA80000E005243CB9859BDB88AB802846002113
:10FAB800FFF74CF80446042C08BF05240CB10023BA
:10FAC8002B60204600E009200DF5077D30BD00BF02
:10FAD800F0B5ADF5057D04460F46FEF761FB05461A
:10FAE80028BB2FB920460021FFF730F805461EE055
:10FAF80081ABA36101ABE36120460021FFF75AFB0C
:10FB08000646042802D1002323612E4676B92046F2
:10FB18003946FEF733FD20460021FFF74FF9054629
:10FB2800042804D100232361354600E035462846E1
:10FB38000DF5057DF0BD00BF2DE9F04798B00346EF
:10FB48000F46604A16924FF48072179207A819461A
:10FB5800FFF782FF0246002840F0B0800026DFF859
:10FB6800A0A1DFF8A091DFF8A08107A810A9FFF7EE
:10FB7800AFFF0246002840F0A1809DF84930002BD5
:10FB880000F09C805BB22E2BEFD0169D2B780BB922
:10FB98000DF14905BDF84420C2F34313013B0B2B7B
:10FBA80066D8DFE803F0060E161E262E363E464EB1
:10FBB800565E454B93E8030003908DF8101004241B
:10FBC80056E0424B93E8030003908DF8101004248C
:10FBD8004EE03F4B93E8030003908DF81010042487
:10FBE80046E03C4B93E8030003908DF81010042482
:10FBF8003EE0394B93E8030003908DF8101004247D
:10FC080036E0364B93E8030003908DF81010042477
:10FC18002EE0334B93E8030003908DF81010042472
:10FC280026E0304B93E8030003908DF8101004246D
:10FC38001EE02D4B93E8030003908DF81010042468
:10FC480016E02A4B93E8030003908DF81010042463
:10FC58000EE0274B93E8030003908DF8101004245E
:10FC680006E0244B93E8030003908DF81010042459
:10FC780003A82044514602F01F0207F025FC204447
:10FC8800BDF84420520A03AB1844494602F2BC723C
:10FC980007F01AFC9DF8483013F0100F14BF164BEC
:10FCA800164B1B88BB5301360095B8194146109A6C
:10FCB80003AB07F009FC0446064456E7104618B0A3
:10FCC800BDE8F08718080020849901088C9901087C
:10FCD800949901089C990108A4990108AC99010814
:10FCE800B4990108BC990108C4990108CC99010884
:10FCF800D4990108DC990108E8990108EC990108F0
:10FD0800E4990108289C0108F099010810B592B0FF
:10FD180003460C461C4A10924FF4807211920278E6
:10FD280022B901A81949FFF797FE03E001A819466F
:10FD3800FFF792FEE0B901A80AA9FFF7C9FED0B9FA
:10FD48009DF83130D3B15BB22E2BF4D010980378E4
:10FD58000BB90DF13100214607F0F4FB03460028EA
:10FD6800E9D19DF8302012F0100F09D10A9B07E065
:10FD78004FF0FF3304E04FF0FF3301E04FF0FF3363
:10FD8800184612B010BD00BF1C090020288F0108BA
:10FD98002DE9F04F83B002AB43F8040D8A461446B0
:10FDA800104619460022FEF717FA256880460028F3
:10FDB8005FD12B696C69A21E934202D8CAF8003041
:10FDC80057E02F78012F11D102240026284621461A
:10FDD800FEF74AFEB0F1FF3F3FD0012840D000B9FE
:10FDE800013601346B699C42F0D33BE0296A002359
:10FDF8001A461E464FF4007B52B901F10109284604
:10FE0800FEF772F9804668BB05F1300349465A4649
:10FE1800022F09D193F801C0187850EA0C2008BFC6
:10FE280001360233023A15E093F803C098780004CB
:10FE380040EA0C6093F801C040EA0C2093F800C037
:10FE480020F0704020F0FF0050EA0C0008BF013697
:10FE58000433043A013CCFD104E04FF0010801E03B
:10FE68004FF002082E616B7943F001036B71CAF8F9
:10FE78000060404603B0BDE8F08F00BF30B5ADF577
:10FE8800197D01908FA801A90122FEF7A5F9044662
:10FE980000284BD183AB959303AB96938FA8019918
:10FEA800FFF78AF80446002840D1949931B1CB7AFB
:10FEB80003F00103002B18BF072400E00624FCB957
:10FEC800CB7A13F0100F1DD08F98FDF7BBFF0546B6
:10FED800D0B186A88FA92422FDF784FF889586A82B
:10FEE8000221FEF733FE044678B986A80021FFF701
:10FEF80061F9002808BF0720042818BF044604E059
:10FF0800002502E0002500E002247CB98FA8FFF755
:10FF1800B3F9044628B925B18F982946FFF7E0F9C7
:10FF280004461CB98F98FEF733FD044620460DF5AC
:10FF3800197D30BD2DE9F04FADF50F7D0190F8F733
:10FF480025FF054685A801A90122FEF745F90446C3
:10FF5800002840F0A18082AB8B9302AB8C9385A8DC
:10FF68000199FFF729F8002808BF0820042840F065
:10FF7800928085980021FEF7BFFEB0F1000908BF06
:10FF88000724B9F1010F08BF0224B9F1FF3F08BFE8
:10FF980001241CB98598FEF775F80446002C59D140
:10FFA800859E30464946FEF753FD074606F1300A5E
:10FFB800504600214FF40072FDF71EFF50462021E5
:10FFC8000B22FDF719FF4FF02E0B86F830B01023E7
:10FFD80086F83B3086F84650C5F3072386F8473045
:10FFE800C5F3074386F848302B0E86F8493050464B
:08FFF8004946FDF737FF06F151
:020000040801F1
:100000005008404651462022FDF7F0FE86F851B0D8
:100010008799859B1A78032A03D15B6A8B4208BFB4
:1000200000214046FDF722FF859B9E784FF0010B93
:1000300012E0859807F10108C76280F804B0FEF766
:1000400025F8044650B9504600214FF40072FDF7E0
:10005000D7FE013EF6B24746002EEAD11CB985A86C
:10006000FFF71AF8044624B185984946FFF73CF992
:1000700016E08A981023C3728575C5F30723C375EC
:10008000C5F3074303762D0E45764946FDF7EEFE90
:10009000859801230371FEF77FFC044600E00446C7
:1000A00020460DF50F7DBDE8F08F00BF2DE9F04F24
:1000B0008DB009900C461546012988BF132000F227
:1000C000688309A8FDF7B4FF0028C0F23683BE4B51
:1000D00053F82060002E00F03B8300233370BB4BAD
:1000E00013F8107003EB400393F801803846F8F7DB
:1000F000C7FD10F0010F40F02D8310F0040F40F009
:100100002B83B8F1000F34D0384606F130010022BD
:100110000123F8F7B9FD002840F0208396F82F223C
:1001200096F82E3243EA022212B2A94B9A4240F0CC
:10013000178306EB081393F8E22103F5EF73002A07
:1001400000F01083D97A9A7A120442EA0162597A4D
:1001500042EA01211A7A41EA020AD97B9A7B120407
:1001600042EA0162597B42EA01221B7B13430A9354
:1001700014E0384601210AAAF8F7C8FD002840F02B
:10018000F3820A9B7F2B40F2F182002C0CBF4FF0D0
:100190003F0A4FF0000ACAEB03030A936B1E2B427F
:1001A00018BF00257DB94FF4FA600A9BB3FBF0F04D
:1001B0000023884900E0013331F813208242FAD845
:1001C000854A32F81350B5F5007F28BF6D0A002D1F
:1001D00008BF0125812D28BF80250A9AB2FBF5F3BF
:1001E00040F6F5794B458CBF4FF002094FF00109FD
:1001F0004FF6F5718B4288BF4FF00309B9F1030F39
:1002000009D19B0003F207235B0A019300210491AB
:100210002023029312E0B9F1010F05D103EB430350
:1002200001335B08033301E002335B0003F2FF1389
:100230005B0A019320210491012302930299514406
:1002400003918B46019B9B4404998B440BEB050364
:10025000CAEB03039A42C0F08B82384603210BAAF3
:10026000F8F754FD20B90B9B13B1B3F5004F01D93A
:1002700001230B930B9B0BEB0302013A5B421340F0
:10028000CBEB03030B93B9F1030F06D1029A1A4487
:10029000029203991944039102E0019A1A440192CF
:1002A0000A9B02995A1A0199521A0499521AB2FBDE
:1002B000F5F20592B9F1020F05D140F6F5720599F4
:1002C000914240F25782B9F1030F05D14FF6F57212
:1002D0000599914240F25082B9F1030F0DD0B9F166
:1002E000010F02D1B3F5803F0AD3B3F5803F2CBF95
:1002F0004FF0060B4FF0040B04E04FF00C0B01E045
:100300004FF0010BB8F1000F10D006EB081888F879
:10031000E2B1384606F1300100220123F8F7D0FCA3
:10032000002840F02B824FF0F80859E0002C55D1FE
:1003300006F13004204600214FF40072FDF760FD05
:10034000012386F8EF3186F8F031002286F8F1219A
:1003500086F8F2B1FE2186F8F3110A990AEB010E34
:1003600043F6C160BEFBF0F00B904FEA900E4EF0EA
:100370003F0E86F8F4E186F8F5013F2086F8F60195
:1003800086F8F72186F8F82186F8F92186F8FA111F
:10039000C1F3072086F8FB01C1F3074086F8FC0192
:1003A000090E86F8FD11552186F82E12AA2186F82D
:1003B0002F1238462146F8F783FC002840F0E081F0
:1003C0004FF0F8080CE000BF1C0A00205C01002080
:1003D00055AAFFFF58990108549A01084FF0F008F8
:1003E00006F1300B584600214FF40072FDF708FD6E
:1003F0005846D3490B22FDF7F9FC002386F83B3021
:10040000022386F83C3086F83D50029A86F83E205A
:10041000C2F3072386F83F30012386F84030B9F154
:10042000030F4FF0000386F8413018BF022386F80F
:1004300042300A9BB3F5803F06D286F84330C3F3BF
:10044000072386F844300CE086F85030C3F30722C7
:1004500086F85120C3F3074286F852201B0E86F817
:10046000533086F845803F2386F84830002386F8CD
:100470004930FF2286F84A2086F84B3086F84CA097
:10048000CAF3072386F84D30CAF3074386F84E3087
:100490004FEA1A6386F84F30F8F77CFC0B90B9F1FD
:1004A000030F3CD186F87300C0F3072386F874303D
:1004B000C0F3074386F87530000E86F87600019B7E
:1004C00086F854301946C3F3072386F85530C1F334
:1004D000074386F856300B0E86F85730022386F80D
:1004E0005C30002386F85D3086F85E3086F85F3039
:1004F000012286F8602086F86130062286F86220A4
:1005000086F86330802386F87030292386F87230AD
:1005100006F177008B491322FDF768FC1FE086F88F
:100520005700C0F3072386F85830C0F3074386F816
:100530005930000E86F85A00019A86F84620C2F318
:10054000072386F84730802386F85430292386F81D
:10055000563006F15B007C491322FDF747FC55231A
:1005600086F82E32AA2386F82F323846594652464C
:100570000123F8F7A5FB002840F00481B9F1030F2F
:1005800006D1384659460AF106020123F8F798FBCE
:100590000023029368F0FF010691CAB20792089502
:1005A000039D62E0584600214FF40072FDF728FCDD
:1005B000B9F1030F13D0B9F1010F644A18BF6FF0FE
:1005C000FF0242EA08030B9386F83030FF2286F8D8
:1005D000312086F832201B0E86F833301CE0069B53
:1005E0000B93079986F83010FF2386F8313086F890
:1005F000323086F8333086F8343086F8353086F875
:10060000363086F8373086F8383086F8393086F854
:100610003A300F2386F83B306C1C384659462A4640
:100620000123F8F74DFB002840F0AE80584600212A
:100630004FF40072FDF7E4FB01230B9322460CE01C
:10064000541C384659460123F8F73AFB002840F07D
:100650009D800B9B01330B9322460B9B01998B4290
:10066000EED31546029A01320292029B002B99D0DA
:100670000395089D0499B9F1030F08BF2946049119
:100680000124039A0D4602F10108384659462346D3
:10069000F8F716FB00287BD14246013DF3D1B9F1B2
:1006A000030F41D1522386F8303086F83130612370
:1006B00086F83230412286F83320722186F81412EF
:1006C00086F8151286F8162286F81732059A531EF8
:1006D00086F81832C3F3072386F81932531EC3F382
:1006E000074286F81A221B0E86F81B32022386F870
:1006F0001C32002386F81D3286F81E3286F81F321F
:10070000552386F82E32AA2386F82F3238465946CA
:100710000AF101020123F8F7D3FA384659460AF1E3
:1007200007020123F8F7CCFA384600210A46F8F709
:10073000EDFA003018BF01202BE00B2029E000BFAC
:10074000109A01081C9A0108309A010800FFFF0066
:100750000C201EE003201CE00A201AE0012018E013
:100760000E2016E00E2014E0012012E0012010E01F
:100770000E200EE00E200CE00E200AE0012008E022
:10078000012006E0012004E0012002E0012000E059
:1007900001200DB0BDE8F08F7F2815D971B1FF2879
:1007A0009DBF8038094B33F810000020704731F8A6
:1007B0001320824206D001339BB201E0002303499B
:1007C0007F2BF4D98033D8B2704700BF6C9A0108F0
:1007D000A0F161039BB2192B9CBF203880B27047F7
:1007E00070B592B001200146F6F794FF4FF4C06057
:1007F0000121F6F7B5FFF023ADF8443000248DF861
:100800004740374811A9F6F71FFB364D2846F5F744
:10081000CDFF354B0693354B079308940426099674
:100820000A9480230B934FF480730C934FF48063EE
:100830000D9320230E934FF400530F9310942846EA
:1008400006A9F6F76FF828460121F6F713F9019487
:1008500001258DF808508DF809504FF4602303935B
:1008600004948DF81460224C20460DEB0601F5F738
:1008700093FD204607212A460323F5F71FFF204654
:10088000062102220323F5F719FF20460521032242
:100890001346F5F713FF2046314632460323F5F79A
:1008A0000DFF20462946F5F745FE20462946F5F777
:1008B00017FE2046F5F764FE2046F5F77DFE00287A
:1008C000FAD10B48F5F796FE094C2046F5F7AEFE37
:1008D0000028FAD106480121F5F7C6FE12B070BD16
:1008E00000080140080002404C2401402C25002053
:1008F0000024014010B5044672B6F6F7E3F935203E
:10090000F6F7F4F92046F6F72DFA042804D1F6F7A5
:10091000E5F962B6002010BD4FF0FF3010BD00BFFA
:100920002DE9F04105460F46904672B6960812F042
:10093000030F18BF0136F6F7C5F93520F6F7D6F9DB
:10094000002408E0284657F82410F6F739FA04285E
:1009500009D104350134B442F4DBF6F7BFF962B6CD
:100960004046BDE8F0814FF0FF30BDE8F08100BFA8
:1009700010B4002302E0C45CCC5401339342FAD398
:1009800018465DF8044B7047194B1B88FF2B17D98D
:10099000184B4FF000621A6002F5C0425A604FF4E3
:1009A00000621A8140225A810C221A7303225A7360
:1009B0003122DA81104A1A61A2F500625A61704749
:1009C0000C4B4FF000621A6002F5C0425A604FF4BF
:1009D00080621A8180225A8118221A7303225A7364
:1009E0006522DA81054A1A61A2F580625A61704770
:1009F000E0F7FF1F3425002000F0010800F801088F
:100A000010B582B004460F4B53F820000121F6F7D1
:100A1000A7FE0D4B33F81430ADF804300B4B2344D4
:100A20009B78012B0CBF282310238DF8073003235C
:100A30008DF80630064B53F8240001A9F6F704FAA6
:100A400002B010BD6C9B0108AC9B0108D4280020AB
:100A50006001002008B50346064A02449278022A43
:100A600007D1054A52F82000044A32F81310F6F76D
:100A70003FFB08BDD428002060010020AC9B01088A
:100A800008B50346064A02449278022A07D1054A6D
:100A900052F82000044A32F81310F6F759FB08BD4B
:100AA000D428002060010020AC9B010808B5024654
:100AB0000D4B03449B78012B08D10C4B53F82000BD
:100AC0000B4B33F81210F6F75BFA08BD022B08D176
:100AD000064B53F82000064B33F81210F6F7ACFA29
:100AE00008BD002008BD00BFD42800206001002000
:100AF000AC9B010870B582B00E461546052806D19C
:100B00001048694601AAFFF747F9044609E0431E69
:100B1000DBB2032B05D80C48694601AAFFF73CF964
:100B2000044664B9019B5A69023A9B7803FB02F1BF
:100B3000009A02FB03F34A0832605B082B602046F0
:100B400002B070BDCC9B0108D09B010808B5F8F736
:100B500047F9F8F73DFA02280BD060B90748084971
:100B60000022FEF7F9FB0122064B1A60064B1878AB
:100B700008BD002008BD002008BD00BF4C25002096
:100B8000D09B0108301300201C03002008B5F8F7A3
:100B900085FD0F480F490022FEF7DEFBF8F714F839
:100BA00001280CBF012200220B4B1A6009480021CA
:100BB0004FF40072FFF77AFAF8F706F8012801D12E
:100BC000F8F718F80122044B1A60052008BD00BF91
:100BD0004C250020CC9B01082C13002010B5F6F703
:100BE0000FFC4FF48030F6F72BFCF6F737FE0128A8
:100BF00030D11020F6F74EF80220F6F737F8002033
:100C0000F6F7C4FC4FF48060F6F704FD4FF4806003
:100C1000F6F7E0FC4FF480304FF48011F6F73EFC1D
:100C20000120F6F787FC39242046F6F7E5FD002879
:100C3000FAD00220F6F78EFCF6F7A0FC0828FBD1CC
:100C40004FF410300121F6F7B1FD44F23D000121CF
:100C5000F6F786FD10BD00BF01604360826000238F
:100C60000361C3600120704738B504460568C26857
:100C70000369D21A43689A420DDAC268013B02EA5C
:100C80000300A26802FB005006F0D5FAE3680133C6
:100C9000E360012038BD002038BD00BFF8B5044630
:100CA0000F46D0F800E0C1680369C91A4368994249
:100CB0000BDBC1680269891A1D488B42CCBF002139
:100CC000012106F061FB0020F8BDC6680169761AB3
:100CD0009E1BC168581E0840811999422CBFC0EB69
:100CE00003053546761BAA42B8BF1546521BB242D1
:100CF000B8BF1646A26802FB00E0394602FB05F2C7
:100D000006F099FAE3682B44E36020686268013AD0
:100D10001340A26802FB030002FB057102FB06F20E
:100D200006F089FAE3683344E360A819F8BD00BF10
:100D3000D49B010838B504460568C26803699A4225
:100D40000ED003694268013A13408268084602FBEC
:100D5000035106F070FA236901332361012038BD85
:100D6000002038BDF8B504460F460168C068236905
:100D7000984231D0E6682369F61A23696568681ECF
:100D800003409819A8422CBFC3EB05053546761BD6
:100D9000AA42B8BF1546521BB242B8BF1646A26857
:100DA000384602FB031102FB05F206F044FA236900
:100DB0002B44236121686268013A1340A26802FB58
:100DC000057002FB031102FB06F206F034FA2369F8
:100DD00033442361A819F8BD0020F8BD08B50348C5
:100DE0004FF48051F6F7B4F908BD00BF000C014084
:100DF00008B503484FF48051F6F77AF908BD00BFF3
:100E0000000C014070B506460C4D022428462146D0
:100E1000F6F772FE0028F9D008483146F6F738FE9A
:100E2000064D012428462146F6F766FE0028F9D033
:100E30000248F6F747FEC0B270BD00BF0038004060
:100E400008B5FFF7DFFF08BD08B5FF20FFF7DAFFA1
:100E500008BD00BF30B58DB005460C464FF6FF7398
:100E6000ADF800302D4B01930023079308930593B1
:100E7000049209934FF440520A920B932848F5F7D5
:100E800095FC2848F5F792FC9DB102940024039448
:100E900080230693224801A9F5F744FD0DEB0403D6
:100EA00002931023039306941E4801A9F5F73AFD17
:100EB00011E000AB0293002303930693184801A9A5
:100EC000F5F730FD02941023039380230693154811
:100ED00001A9F5F727FD12480121F5F7CBFD1148CF
:100EE0000121F5F7C7FD104803210122F6F79AFD0D
:100EF0004FF400542046F5F703FE0028FAD00848C6
:100F00000021F5F7B7FD07480021F5F7B3FD0648C6
:100F100003210022F6F786FD0DB030BD0C380040ED
:100F200044000240580002400038004008B5034623
:100F30000A4601201946FFF78DFF08BD08B5034694
:100F40000A4600201946FFF785FF08BD70B586B038
:100F50004FF40053ADF8143003238DF816301823E6
:100F60008DF817302B4D284605A9F5F76DFF4FF486
:100F70000043ADF81430284605A9F5F765FF4FF496
:100F80008043ADF8143004238DF81730284605A9A6
:100F9000F5F75AFF4FF48053ADF8143010238DF855
:100FA0001730284605A9F5F74FFF0023ADF80030AC
:100FB0004FF48272ADF80220ADF804300222ADF891
:100FC00006200124ADF808404FF40072ADF80A2065
:100FD000ADF80C30ADF80E300723ADF810300E4EE2
:100FE00030466946F6F75CFC30462146F6F7EEFCE3
:100FF00028462146F6F7ACF82046F7F7DDFD2846EF
:101000002146F6F775F820462146F6F783FB06B031
:1010100070BD00BF000C01400038004010B586B024
:10102000FFF7E6FE14481549FBF7FCFD1448154987
:10103000FBF70AFE14481549FBF720FE144B01ACE0
:10104000186859689A68DB680FC4012001A9FBF78A
:101050009BFFB0F1FF3F02D10E4806F021FA0F24AA
:1010600020460DF11701FBF78FFF9DF81730002B7D
:10107000F6D006B010BD00BFDD0D0108F10D01086E
:10108000490E0108410E01082D0F01083D0F01080E
:10109000F09B0108009C010808B50128044B03BF20
:1010A00018891B69C0181869FFF762FC08BD00BFEA
:1010B0003425002070B50E4615460128074B03BFA6
:1010C0001C891B69E4181C692046FFF713FC2046A5
:1010D00031462A46FFF724FC70BD00BF34250020AE
:1010E00008B54FF080400121F6F76EFF40B34FF096
:1010F00080400121F6F70CFF4FF080400121F6F708
:10110000D1FF104B1A88013292B21A801A8892B21B
:1011100040F2E6339A420BD90B4B1A780132D2B225
:101120001A70F9F72BFAFAF7C3FE0022054B1A8062
:10113000054B1B78DBB23A2B02D90022024B1A7006
:1011400008BD00BF240A0020260A002010B584B084
:1011500001200146F6F72AFB1C238DF800300124FC
:101160008DF801408DF802408DF803406846F5F790
:101170008BF84FF47A73ADF808300023ADF80430E3
:10118000ADF80A30ADF806304FF0804001A9F6F70F
:10119000E7FC4FF0804047212246F6F75FFE4FF014
:1011A00080402146F6F78AFD4FF0804021462246D6
:1011B000F6F7E8FD04B010BDF8B505460F46164633
:1011C0001C4640F227710022F7F720F938463146D5
:1011D0002246FFF763FD0446284640F227710122AC
:1011E000F7F714F92046F8BD08B5044806F0C0F931
:1011F00080B20028014808BF002008BD90270020C9
:1012000008B50021044B1980044B198004484FF4A1
:10121000967206F019F808BD280A00202C1200204A
:101220009027002010B5184840F22551F7F706FA2C
:1012300048B3154840F22551F7F77CFA134B1C8848
:10124000134B1B889C4203D9E21AB2F5957F04DC4C
:101250009C4207D2621C934204D10B484021F7F70D
:101260004BF910BD0848F7F773F90A4B1855074BAF
:101270001B88B3F5957F03D80133044A138010BD52
:101280000022024B1A8010BD00380140280A0020BD
:101290002C1200209027002070B5064606483146E3
:1012A000F7F72AF9044D802428462146F7F772F90A
:1012B0000028F9D0304670BD003801400B480C4979
:1012C00003880A889342FBD0B3F5957F07D8013392
:1012D0009BB2064A1380013B064AD05C704700224D
:1012E000024B1A80034B93F82B0170472C120020FD
:1012F000280A002090270020F8B50D46174638B17F
:101300000CE0FFF7DBFF287001360134013501E006
:1013100000263446BC42F4DB3046F8BD05F048FFF9
:10132000092303604FF0FF30F8BD00BF70B51546CC
:10133000012809D0022812D015E04E1C0878FFF7CA
:10134000ABFF0134314600E00024AC42F5DB11E094
:101350004E1C0878FFF7A0FF0134314600E000245E
:10136000AC42F5DB06E005F023FF092303604FF0F4
:10137000FF3070BD284670BD30B585B00023364DB6
:1013800008E00A6855F82340A24202D100920123E6
:1013900003E00133092BF4D9002313B94FF4E133EF
:1013A00000930B79082B02D0092B04D008E000230E
:1013B000ADF8043009E04FF48053ADF8043004E098
:1013C0000023ADF8043008230B718B79012B02D078
:1013D000022B04D008E00023ADF8063009E04FF4FA
:1013E0000053ADF8063004E00023ADF806300123C9
:1013F0008B714B79012B07D013B1022B09D00DE073
:101400000023ADF808300DE04FF4C063ADF80830AC
:1014100008E04FF48063ADF8083003E00023ADF836
:1014200008304B714B7913B1012B04D008E0002335
:10143000ADF80C3007E04FF44073ADF80C3002E02B
:101440000023ADF80C300C23ADF80A306946F6F7EE
:1014500085FE05B030BD00BFA001002030B585B0CD
:1014600001F0DCFA05464FF49053ADF80430182330
:101470008DF8073003238DF80630164C204601A95D
:10148000F5F7E2FC04238DF807304FF44063ADF824
:101490000430204601A9F5F7D7FC0023ADF8083049
:1014A000ADF80A304FF40072ADF80C20ADF80E30F4
:1014B00004F54054204605F13301FFF75DFF204657
:1014C00002A9F6F721FF20460121F6F76BFF05B0D0
:1014D00030BD00BF00080140F8B505460F4616466E
:1014E0001C4640F225510022F6F790FF384631465F
:1014F0002246FFF737FC0446284640F225510122D8
:10150000F6F784FF2046F8BD70B582B005460C465C
:10151000164640F22771F7F791F888B130460DF181
:101520000701FFF707FC28B128469DF80710F6F7DA
:10153000E3FF05E0284640F227710022F6F766FF38
:10154000284640F22551F7F779F870B1E26823692F
:10155000D21A63689A4208DA2846F6F7F9FF02A918
:1015600001F8010D2046FFF77FFB02B070BD00BF00
:1015700008B503480349044AFFF7C6FF08BD00BF8A
:1015800000440040BC2800207C270020F0B585B036
:1015900001F044FA07462A482A4901224FF48063A1
:1015A000FFF75AFB2848294901224FF48063FFF7CF
:1015B00053FB26238DF8003000248DF801408DF870
:1015C000024001258DF803506846F4F75DFE0623BE
:1015D000ADF8043018238DF8073003238DF806305A
:1015E0001B4E304601A9F5F72FFC04238DF8073078
:1015F0000923ADF80430304601A9F5F725FCADF814
:101600000840ADF80A404FF40073ADF80C30ADF867
:101610000E40104C204607F13B01FFF7ADFE20467F
:1016200002A9F6F771FE204640F225512A46F6F748
:10163000EDFE20462946F6F7B5FE05B0F0BD00BF29
:10164000BC2800202C0E00207C2700202C0A002023
:10165000000801400044004008B502460B4602481D
:101660000249FFF739FF08BD00440040BC280020B4
:1016700008B502460B4602480249FFF79DFD08BD2A
:10168000004400407C270020024BD8681B69C01A28
:10169000704700BF7C27002008B504480449012298
:1016A0004FF48063FFF7D8FA08BD00BF7C27002005
:1016B0002C0A002008B503460A4603494869194622
:1016C000FFF756F908BD00BF3425002070B5064667
:1016D0000D46054B5C692046FFF70CF92046314664
:1016E0002A46FFF71DF970BD342500202DE9F04191
:1016F0003A4C20464FF4DB71FFF7DCFF2378AA2B2E
:1017000002D16378012B3ED0344BAA221A700122F9
:101710005A7002219970D970197159719971D971E2
:10172000197259729A72DA721A735A739A73DA7357
:101730001A745A7400232948194603E0C218917498
:101740000133DBB20F2BF9D90024DFF89080192781
:10175000234E11E004EB840505EB85054544223555
:10176000284600213A4605F06FFD284631462246BC
:1017700005F0AEFE0134E4B20F2CEBD917484FF45C
:10178000DB71FFF7A3FF17480121F5F711FD0024D6
:10179000124D0AE02B199B78013BDBB2FD2B02D8DE
:1017A0002046FFF72DF90134E4B20F2CF2D90024C2
:1017B0000A4D0FE02B199B78022B09D12B199B7C2A
:1017C0001BB92046FFF75CF902E02046FFF742F91B
:1017D0000134E4B20F2CEDD9BDE8F081D42800200B
:1017E0001C9C010800043000024B33F8100080B24A
:1017F000704700BF2C2500202DE9F04FC9B0429062
:10180000439101F00BF90023ADF81C31ADF818310C
:10181000ADF814314FF0040A08264FF007094FF0D5
:1018200009084FF0050C4FF0060E012502274FF076
:10183000030B7FE01A46991D00EBC101D1F803109C
:10184000B1F5165F39D00ED8B1F5966F44D003D8F4
:10185000B1F5167F45D04AE0B1F5166F37D0B1F536
:10186000965F2FD043E0B1F5614F17D006D8B1F5A0
:10187000964F1DD0B1F5164F15D038E0B1F5E13FC8
:1018800007D0B1F5613F32D148A9194401F8048C61
:1018900031E048A9194401F8046C2CE048A9194426
:1018A00001F8049C27E048A9194401F804EC22E05F
:1018B00048A9194401F804CC1DE048A9194401F8CD
:1018C00004AC18E048A9194401F804BC13E048A985
:1018D000194401F8047C0EE048A9194401F8045C9D
:1018E00009E0002448A9194401F8044C03E048A980
:1018F000114401F8046C00EBC20191F8371009297A
:1019000004D148A9114401F8085C04E0002448A966
:10191000114401F8084C00EBC20191F8391002297A
:1019200048A90A440EBF02F80C5C002102F80C1C06
:101930000133DBB2012B7FF67DAF827FC37F90F84E
:1019400020B000F1050A90F8029090F8038090F81A
:1019500004C090F821E090F82270279790F82310A7
:10196000289190F82470299790F825102A9190F8E2
:1019700026702B9790F84D102C9190F827702D978A
:1019800090F828102E9190F829702F9790F82A102F
:10199000309190F82B70319790F82C10329190F88C
:1019A0002D70339790F82E10349190F82F70359752
:1019B00090F83010369190F83170379790F83210D7
:1019C000389190F84F70399790F850103A9190F8FC
:1019D00051703B9790F852103C919DF81C713D97C7
:1019E0009DF818113E9190F838703F979DF814615A
:1019F00090F83A509DF81D419DF8191190F84070EB
:101A000040979DF81571419790F84200CDF800B0CD
:101A1000CDF804A0CDF80890CDF80C80CDF810C01A
:101A2000CDF814E0279F0697289F0797299F0897CE
:101A30002A9F09972B9F0A972C9F0B972D9F0C97F6
:101A40002E9F0D972F9F0E97309F0F97319F1097C6
:101A5000329F1197339F1297349F1397359F149796
:101A6000369F1597379F1697389F1797399F189766
:101A70003A9F19973B9F1A973C9F1B973D9F1C9736
:101A80003E9F1D973F9F1E971F9620952194229160
:101A900040992391419F249725904298034905F04E
:101AA00017FD439F388049B0BDE8F08F2C9C01089A
:101AB0002DE9F04FBDB0834688460020FEF7F6FFC3
:101AC00082460120FEF7F2FF81460220FEF7EEFF7C
:101AD0002E900320FEF7EAFF2F900420FEF7E6FF8A
:101AE00030900520FEF7E2FF31900620FEF7DEFF82
:101AF00032900720FEF7DAFF33900820FEF7D6FF7A
:101B000034900920FEF7D2FF35900A20FEF7CEFF71
:101B100036900B20FEF7CAFF37900C20FEF7C6FF69
:101B200038900D20FEF7C2FF39900E20FEF7BEFF61
:101B30003A900F20FEF7BAFF3B90354B9A782192EE
:101B4000DA7822921A7923925A7924929A792592F4
:101B5000DA7926921A7A27925A7A28929A7A2992D0
:101B6000DA7A2A921A7B2B925A7B2C929A7B2D92AC
:101B7000DF7B1E7C5D7C0020F6F7D2FF044601204F
:101B8000F6F7CEFF2E9B00932F9A0192309B029383
:101B9000319A0392329B0493339A0592349B0693B5
:101BA000359A0792369B0893379A0992389B0A9385
:101BB000399A0B923A9B0C933B9A0D92219B0E9370
:101BC000229A0F92239B1093249A1192259B129391
:101BD000269A1392279B1493289A1592299B169361
:101BE0002A9A17922B9B18932C9A19922D9B1A9331
:101BF0001B971C961D951E941F90584605495246EA
:101C00004B4605F065FCA8F800003DB0BDE8F08F3C
:101C1000D428002064A001082DE9F04FBDB0834610
:101C200088460020FEF742FF82460120FEF73EFF75
:101C300081460220FEF73AFF2F900320FEF736FF81
:101C400030900420FEF732FF31900520FEF72EFF82
:101C500032900620FEF72AFF33900720FEF726FF7A
:101C600034900820FEF722FF35900920FEF71EFF72
:101C700036900A20FEF71AFF37900B20FEF716FF6A
:101C800038900C20FEF712FF39900D20FEF70EFF62
:101C90003A900E20FEF70AFF3B900F20FEF706FF5A
:101CA0003D4A91780E91D3780F9317791097517917
:101CB000119193791293D7791397117A149192F81D
:101CC00009C092F80AE0D37A1793167B557B947B70
:101CD000D17B177C1C97537C2F9F0097309F0197D7
:101CE000319F0297329F0397339F0497349F059744
:101CF000359F0697369F0797379F0897389F099714
:101D0000399F0A973A9F0B973B9F0C970D90CDF800
:101D100054C0CDF858E0189619951A941B911D934C
:101D200002F122031E9302F13B031F9302F15403BD
:101D3000209302F16D03219302F18603229302F1B5
:101D40009F03239302F1B803249302F1D103259357
:101D500002F1EA03269302F20313279302F58E732E
:101D6000289302F23513299302F5A7732A9302F2FE
:101D700067132B9302F5C0732C9302F299132D93E2
:101D80005846064952464B4605F0A2FBA8F800000B
:101D90003DB0BDE8F08F00BFD4280020F8A30108B3
:101DA0002DE9F04184B007460C460020FFF71CFDEA
:101DB00006460120FFF718FD05460220FFF714FD37
:101DC00080460320FFF710FDCDF8008001906423CA
:101DD0000293C82303933846044932462B4605F044
:101DE00077FB208004B0BDE8F08100BF00A90108A6
:101DF00038B505460C46FFF7F7F902462846034971
:101E000005F066FB2080FFF7FBF938BDB4A9010897
:101E1000F0B583B0054600F001FE044690F8273087
:101E20008DF8043090F828308DF8053090F829307E
:101E30008DF8063090F82A308DF8073028464C4946
:101E4000F8F746F8064680B1671D3846002119228A
:101E500005F0FAF9304605F08BFBC2B2192A384674
:101E6000314628BF182205F0E6F928464149F8F71F
:101E70002FF850B1312105F05CFB18B1012384F833
:101E80004D3002E0002384F84D3094F84D309BBB78
:101E900028463949F8F71CF898B104F12701F7F7FB
:101EA000CFFF94F827308DF8043094F828308DF85F
:101EB000053094F829308DF8063094F82A308DF8E2
:101EC000073028462D49F8F703F818B104F12B0123
:101ED000F7F7B6FF28462A49F7F7FAFF18B104F1D9
:101EE0002F01F7F7ADFF28462649F7F7F1FF18B1A4
:101EF00004F14F01F7F7A4FF28462349F7F7E8FF5D
:101F000040B10A21F7F78AFFC0B2204B53F82030C6
:101F1000C4F8333028461E49F7F7DAFF20B10A210A
:101F2000F7F77CFF84F8370028461A49F7F7D0FF07
:101F300020B10A21F7F772FF84F8380028461649C5
:101F4000F7F7C6FF20B10A21F7F768FF84F83900D8
:101F500028461249F7F7BCFF20B10A21F7F75EFFC8
:101F600084F83A0000F0FCFD01A803B0F0BD00BF0A
:101F7000DCA90108E8A90108F0A90108F4A90108F1
:101F8000F8A90108FCA9010800AA0108C80100205D
:101F90000CAA010814AA01081CAA010824AA010815
:101FA00038B505461F49F7F793FF20B10A21F7F727
:101FB00035FFC4B200E0002428461B49F7F788FF2C
:101FC00020B10A21F7F72AFFC5B200E00025A4F1ED
:101FD0005A00C0B2012807D8012D02D1F6F790FDB2
:101FE0001EE0F6F77DFD1BE02246104B23449B7854
:101FF000022B15D1012D07D10C4B1A4400239374E9
:102000002046FEF73DFD06E0084B1A440123937479
:102010002046FEF71FFD05484FF4DB71FFF756FB26
:10202000284638BD30AA010834AA0108D428002067
:1020300070B505461649F7F74BFF28B30A21F7F7A5
:10204000EDFEC4B228461349F7F742FF0546A8B192
:1020500004EB840606EB86060F4B1E443046002137
:10206000192205F0F1F8284605F082FAC2B2192AC1
:102070003046294628BF182205F0DDF807484FF4FE
:10208000DB71FFF723FB00E00024204670BD00BF9A
:1020900030AA010834AA0108F6280020D42800201C
:1020A00038B504461B49F7F713FF20B10A21F7F7AB
:1020B000B5FEC5B200E0002520461749F7F708FF36
:1020C00020B10A21F7F7AAFEC4B200E00024022CD6
:1020D00007D1124B2B4402229A702846FEF790FC3F
:1020E00010E0012C07D10D4B2B4401229A70284699
:1020F000FEF786FC06E02846FEF7C2FC074B1D44AF
:102100000023AB7005484FF4DB71FFF7DFFA204680
:1021100038BD00BF30AA010838AA0108D428002021
:1021200038B50949F7F7D4FE0546002430B938BD63
:10213000285DFFF7B1F80134A4B2FFE7284605F0A7
:1021400017FA8442F4D338BD3CAA010808B50949FE
:10215000F7F7BEFE68B10A21F7F760FEC0B20128AA
:1021600007D10548FF23037043704FF4DB71FFF77D
:10217000ADFA08BD44AA0108D4280020F0B585B006
:1021800007460C4616461D4600F048FC90F84D10D8
:10219000012907D130460B49BD2205F04CF8BC237C
:1021A0002B800CE023786078A178E2780090019190
:1021B0000292304604493A4605F08AF9288005B073
:1021C000F0BD00BF50AA010810AB0108F0B583B004
:1021D00007460E4614461046FEF768FC0346094AB9
:1021E0001119897804EB840505EB85052A44223210
:1021F0000091019238460449224605F069F9308081
:1022000003B0F0BDD428002094AC010870B5064698
:102210000D4614461046FFF7E7FA034630460349D9
:10222000224605F055F9288070BD00BF04AD0108B5
:102230002DE9F04F8FB006460D4600F0EFFB044647
:10224000827FC37F90F820B000F1050A90F80290D9
:1022500090F8038090F804C090F821E090F8227084
:1022600090F8230094F824100C9194F825100D9107
:1022700094F82640CDF800B0CDF804A0CDF8089031
:10228000CDF80C80CDF810C0CDF814E0069707907B
:102290000C9908910D9909910A943046034905F06B
:1022A00017F928800FB0BDE8F08F00BF44AD0108DA
:1022B0002DE9F04F97B006460D4600F0AFFB0446FF
:1022C00090F8272090F8283090F829B090F82AA0AC
:1022D00090F82B9090F82C8090F82DC090F82E104C
:1022E000119190F82F70129790F83010139190F888
:1022F0003170149790F83210159190F84FE090F8E3
:102300005070109790F8510094F8521094F84D4086
:10231000CDF800B0CDF804A0CDF80890CDF80C8031
:10232000CDF810C0119F0597129F0697139F07972E
:10233000149F0897159F0997CDF828E0109F0B97D9
:102340000C900D910E943046034905F0C1F8288099
:1023500017B0BDE8F08F00BFE0AD0108F0B589B05F
:1023600007460E46154600F059FB0023ADF81C3019
:10237000ADF81830ADF81430022D28BF1D462C469C
:10238000AB1D00EBC303D3F80330B3F5165F3ED0AB
:102390000ED8B3F5966F4CD003D8B3F5167F53D053
:1023A0004DE0B3F5166F3ED0B3F5965F35D046E0FD
:1023B000B3F5614F19D006D8B3F5964F21D0B3F5D8
:1023C000164F18D03BE0B3F5E13F08D0B3F5613FBD
:1023D00035D1092108AB2B4403F8041C34E0082153
:1023E00008AB2B4403F8041C2EE0072108AB2B4458
:1023F00003F8041C28E0062108AB2B4403F8041C56
:1024000022E0052108AB2B4403F8041C1CE008ABB8
:102410001D44042305F8043C16E0032108AB2B44BB
:1024200003F8041C10E0022108AB2B4403F8041C41
:102430000AE0012108AB2B4403F8041C04E0082146
:1024400008AB234403F8041C00EBC40393F83730B3
:10245000092B0CBF0121002108AB234403F8081C01
:1024600000EBC40393F83930022B0CBF012100218B
:1024700008AB234403F80C1C08AD254415F8043CB4
:1024800015F808ECA11D00EBC102107A15F80C1C20
:10249000927ACDF800E00190029103923846034908
:1024A000224605F015F8308009B0F0BD88AE01086D
:1024B0002DE9F04784B006468846914600230093F4
:1024C00001930293ADF80C303D4905F03FF828B96F
:1024D00040464946FFF7ACFE01206DE030463949E1
:1024E00005F034F828B940464946FFF7E1FE0120DF
:1024F00062E03046344905F029F830B94046494693
:102500000022FFF72BFF012056E030462F4905F04F
:102510001DF8F8B9404649460122FFF71FFF012088
:102520004AE0009501950295ADF80C506846394691
:10253000224604F0CDFF3046694605F007F830B971
:10254000404649462246FFF741FEE4B208E0013426
:10255000E4B202E0002425461D4F0F2CE1D9FF24F0
:1025600014F0800F1AD1FF251FE000970197029702
:10257000ADF80C70684651462A4604F0A9FF304673
:10258000694604F0E3FF30B9404649462A46FFF762
:102590003DFEEDB209E00135EDB203E000252F4626
:1025A000DFF830A0032DE0D9FF2514F0800F1DBF08
:1025B00068B2C043C00F012004B0BDE8F08700BF7F
:1025C00030AF010840AF010850AF010864AF010807
:1025D00078AF010888AF010838B5044600F01EFA4C
:1025E000054620460E49F7F773FC044690B10535C1
:1025F00028460021192204F027FE204604F0B8FFE7
:10260000C2B2192A2846214628BF182204F013FE18
:10261000012400E000240CB100F0A2FA204638BDED
:1026200098AF010870B5064600F0F8F90546304647
:102630002049F7F74DFC60B1312104F07AFF18B161
:10264000012485F84D4005E0002385F84D30012434
:1026500000E0002495F84D303BBB30461649F7F7B3
:1026600037FC20B105F12701F7F7EAFB01243046DA
:102670001249F7F72DFC20B105F12B01F7F7E0FB2C
:10268000012430460E49F7F723FC20B105F12F0154
:10269000F7F7D6FB012430460A49F7F719FC20B1B9
:1026A00005F14F01F7F7CCFB01240CB100F058FA0B
:1026B000204670BDE8A90108A0AF0108F4A90108EF
:1026C000F8A90108FCA90108F8B504460F4600F076
:1026D000A5F9064620463249F7F7FAFB78B10A21F8
:1026E000F7F79CFBC0B20A2828BF08202D4B53F8EF
:1026F000202006EBC703C3F83320012500E00025A6
:1027000020462949F7F7E4FB78B10A21F7F786FB61
:10271000C0B2A0F1080303F0FF03022B28BF08207A
:1027200006EBC70383F83700012520461F49F7F75A
:10273000CFFB58B10A21F7F771FBC0B2032828BFBD
:10274000002006EBC70383F838000125204618490E
:10275000F7F7BEFB70B10A21F7F760FBC0B2431E6A
:1027600003F0FF03022B28BF012006EBC70383F809
:102770003900012520460F49F7F7AAFB58B10A2175
:10278000F7F74CFBC0B2042828BF002006EBC706B1
:1027900086F83A0001250DB100F0E2F92846F8BDAF
:1027A000A4AF0108C80100200CAA010814AA01085E
:1027B0001CAA0108ACAF010838B505461449F7F763
:1027C00087FBF8B10A21F7F729FBC4B20F2C1CD8FC
:1027D00028461049F7F77CFB38B10A21F7F71EFBB2
:1027E000C0B2032828BF022000E000200A4D2A19A9
:1027F00090702046FEF704F928464FF4DB71FEF78F
:1028000065FF00E00024E0B200E0FF2040B238BDE8
:1028100030AA010834AA0108D428002038B505469A
:102820001849F7F755FB30B30A21F7F7F7FAC4B2A6
:102830000F2C23D828461449F7F74AFB38B10A2150
:10284000F7F7ECFAC0B2022828BF012000E0002010
:102850000E4A22449074012803D12046FEF7FAF86C
:1028600003E010B92046FEF70BF908484FF4DB717E
:10287000FEF72CFF00E00024E0B200E0FF2040B2B1
:1028800038BD00BF30AA010834AA0108D4280020AE
:1028900070B505461849F7F71BFB38B30A21F7F75F
:1028A000BDFAC4B20F2C24D828461449F7F710FB00
:1028B0000546A8B104EB840606EB8606104B1E44C1
:1028C00030460021192204F0BFFC284604F050FED7
:1028D000C2B2192A3046294628BF182204F0ABFCA0
:1028E00008484FF4DB71FEF7F1FE00E00024E0B28F
:1028F00000E0FF2040B270BD30AA010834AA0108F0
:10290000F6280020D4280020F8B504460F461646C5
:102910001D46394904F01AFE50B93846FFF75CFEEF
:1029200002463046354904F0D3FD28800120F8BD29
:102930002046334904F00AFE50B93846FFF772FECC
:10294000024630462D4904F0C3FD28800120F8BD21
:1029500020462C4904F0FAFD58B938460021FFF70B
:10296000B3FE02463046254904F0B2FD288001201E
:10297000F8BD2046244904F0E9FD58B93846012144
:10298000FFF7A2FE024630461C4904F0A1FD288054
:102990000120F8BD20461D4904F0D8FD50B9384645
:1029A000FFF70AFFC2B23046144904F091FD2880B7
:1029B0000120F8BD2046164904F0C8FD50B938463C
:1029C000FFF72CFFC2B230460C4904F081FD28808D
:1029D0000120F8BD20460F4904F0B8FD50B9384633
:1029E000FFF756FFC2B23046044904F071FD28805B
:1029F0000120F8BD0020F8BDB4AF0108289C0108F3
:102A0000C4AF0108D4AF0108E8AF0108FCAF01086A
:102A10000CB0010820B00108002070470048704742
:102A200030120020F8B53D4C852323800127A77084
:102A30000223E37000252571DFF8E4C066460FCE5F
:102A4000C4F80500C4F80910C4F80D20C4F811300A
:102A500003CEC4F81500C4F8191033786377A7774C
:102A6000E77784F82070C02184F82710A82284F822
:102A700028200B2384F82930642084F82A0084F865
:102A80002B1084F82C2084F82D3084F82E70FF232E
:102A900084F82F3084F8303084F8313084F83250A4
:102AA00084F83350636B03F07F4343F4E173636353
:102AB000082384F8373084F8385084F8397084F863
:102AC0003A5084F83B50E26B02F07F4242F4E172EC
:102AD000E26384F83F3084F8405084F8417084F811
:102AE00042500CF11C0203CAC4F84300C4F847105A
:102AF0001288A4F84B2084F84D5084F84E5084F886
:102B00004F3084F8503084F8513084F8523004F15A
:102B100053002946322204F097FBF8BD3012002002
:102B200034B0010810B50D4C012021468522FEF776
:102B3000B3FA2288013A92B24FF6FD739A4206D94F
:102B4000FFF770FF012021468522FEF7B3FA034B01
:102B500001229A77DA7783F8202010BD3012002006
:102B600008B5012002498522FEF7A4FA08BD00BF7E
:102B70003012002008B504F05EFB08BD08B504F073
:102B80005AFB08BD38B50446154D05F12100214614
:102B90000622FFF7F3FF05F12700A11D0422FFF72E
:102BA000EDFF05F12B0004F10E010422FFF7E6FF13
:102BB00005F12F0004F10A010422FFF7DFFF05F100
:102BC0004F0004F112010422FFF7D8FFA37D012B6F
:102BD00007BF00222B460122014B83F84D2038BD50
:102BE0003012002038B50546144C04F121010622AC
:102BF000FFF7C0FFA81D04F127010422FFF7BAFF69
:102C000005F10E0004F12B010422FFF7B3FF05F1DB
:102C10000A0004F12F010422FFF7ACFF05F11200B6
:102C200004F14F010422FFF7A5FF94F84D3013B1D2
:102C30000223AB7538BD0123AB7538BD30120020BF
:102C400030B58BB0012004A9FAF7C8FA9DF810102E
:102C50009DF811209DF812309DF813509DF81440F6
:102C60009DF815000095019402901A4804F08CFB21
:102C70009DF816109DF817209DF818309DF8190042
:102C80000090154804F080FB9DF81E109DF81F2051
:102C90009DF820309DF821000090104804F074FB4E
:102CA0009DF81A109DF81B209DF81C309DF81D0002
:102CB00000900B4804F068FB9DF822109DF823203B
:102CC0009DF824309DF825000090064804F05CFB38
:102CD0000BB030BD5CB0010884B001089CB00108A5
:102CE000B4B00108CCB0010810B586B0FFF796FE6D
:102CF0000446684604F121010622FFF73BFF0DF16F
:102D0000060004F127010422FFF734FF0DF10E0045
:102D100004F12B010422FFF72DFF0DF10A0004F14D
:102D20002F010422FFF726FF0DF1120004F14F01DD
:102D30000422FFF71FFF94F84D301BB102238DF8DA
:102D4000163002E001238DF8163000206946FAF7AC
:102D500045FA06B010BD00BF10B50446FFF75EFE91
:102D60002368C0F82130A388A0F8253010BD00BF2B
:102D7000BFF34F8F044AD16801F4E061034B0B436A
:102D8000D360BFF34F8FFEE700ED00E00400FA05CB
:102D900010B4002304E0CC5C4440CC5401339BB21B
:102DA0009342F8D35DF8044B704700BF10B4002382
:102DB00004E0CC5C4440CC5401339BB29342F8D342
:102DC0005DF8044B704700BF2DE9F041CEB00546D9
:102DD00088461446FFF722FE074628460B210DF5CC
:102DE0009B72F9F76BFEB4F80560BDF83621964288
:102DF00057D10DF10A030093284627A9062203ABF9
:102E0000F9F764FD607810F0800F06D000F07F00C5
:102E100027A9BDF83621FFF7C9FF27A807F121012F
:102E2000062204F0F9F900283BD16FF074036371B6
:102E30000023A371552323713B4653F8210F0490BF
:102E40009B88ADF814300DF116003946852204F048
:102E5000F2F9607810F0800F05D000F07F0004A92F
:102E60008B22FFF795FF20682990A288A379ADF8FF
:102E7000A8208DF8AA300DF1AB0004A98B2204F034
:102E8000DAF9A37823B94046FF21042204F0DCF9E3
:102E9000B8F804300093284629A992224346F9F74E
:102EA00071FC4EB0BDE8F0812DE9F043A5B00546B8
:102EB00088461446FFF7B2FD074628460B210DF160
:102EC0008E02F9F7FBFDB4F80560BDF88E2096423E
:102ED00040F0FC80E378A13B042B00F2F780DFE8B0
:102EE00003F0AE03207B9A000DF13E0300932846C9
:102EF00002A9072210ABF9F7E9FC607810F0800F07
:102F000006D000F07F0002A9BDF88E20FFF74EFF2B
:102F100002A8B91C032204F07FF9002800F08F807A
:102F2000D4E00DF13E030093284602A90C2210AB19
:102F3000F9F7CCFC607810F0800F06D000F07F002D
:102F400002A9BDF88E20FFF731FF9DF8082097F801
:102F500021309A4200F2BA809DF8091097F8222099
:102F6000914200F2B3809DF80A0097F8231088423E
:102F700000F2AC809DF80B6097F82400864200F2C6
:102F8000A5809DF80CC097F82560B44500F29E809E
:102F90009DF80D9097F826C0E14500F297809DF8C6
:102FA0000E904B4500F292809DF80F309A4200F24D
:102FB0008D809DF81030994200F288809DF8113084
:102FC000984200F283809DF812309E427ED89DF890
:102FD00013309C4533D979E00DF13E030093284628
:102FE00002A9212210ABF9F771FC607810F0800F74
:102FF00006D000F07F0002A9BDF88E20FFF7D6FEB4
:103000007E1D02A804F0B4FA024602A8314604F07C
:1030100003F9A0B15AE00DF13E030093284602A93E
:10302000342210ABF9F752FC607810F0800F06D014
:1030300000F07F0002A9BDF88E20FFF7B7FE0C2339
:1030400063710023A371552323713B4633F8022F8C
:103050009B78ADF844208DF846303B4633F81E2F60
:103060009B78ADF847208DF8493057F8213FCDF8CF
:103070004A30BB88ADF84E30607810F0800F05D034
:1030800000F07F0011A90C22FFF782FE2068149047
:10309000A288A379ADF854208DF8563011AB07CB38
:1030A000CDF85700CDF85B10CDF85F20A37823B999
:1030B0004046FF21042204F0C7F8B8F8043000931A
:1030C000284614A913224346F9F75CFB25B0BDE856
:1030D000F08300BF2DE9F04190B0054688461446C4
:1030E000FFF79CFC074628460B210DF13E02F9F73D
:1030F000E5FCB4F80560BDF83E2096425BD10DF1C9
:103100000A030093284606A9172203ABF9F7DEFB52
:10311000607810F0800F06D000F07F0006A9BDF89F
:103120003E20FFF743FE06A807F12101062204F026
:1031300073F800283FD10DF11F0007F1430104F09F
:1031400005FA002837D1062363710023A3715523A4
:10315000237157F8210F0490BB88ADF814306078C4
:1031600010F0800F05D000F07F0004A90622FFF7C1
:103170000FFE20680C90A288A379ADF834208DF85A
:10318000363010AB53F8300DCDF837009B88ADF8D2
:103190003B30A37823B94046FF21042204F054F8C1
:1031A000B8F80430009328460CA90D224346F9F7DD
:1031B000E9FAFFF7DDFD10B0BDE8F0812DE9F0413F
:1031C000F4B0054688461446FFF728FC0746284613
:1031D0000B210DF5E772F9F771FCB4F80560BDF845
:1031E000CE2196426ED10DF10E030093284628A9F8
:1031F0009C2204ABF9F76AFB607810F0800F06D0D0
:1032000000F07F0028A9BDF8CE21FFF7CFFD28A848
:1032100007F12101062203F0FFFF002852D10DF132
:10322000A70007F1430104F091F900284AD138467C
:103230000DF1B7018522FFF7A1FC0123BB77FB77D6
:1032400087F82030FFF78CFC6FF074036371002364
:10325000A371552323713B4653F8210F05909B889A
:10326000ADF818300DF11A003946852203F0E3FF5E
:10327000607810F0800F05D000F07F0005A98B2248
:10328000FFF786FD20684F90A288A379ADF8402112
:103290008DF842310DF2431005A98B2203F0CBFFCC
:1032A000A37823B94046FF21042203F0CDFFB8F8EC
:1032B0000430009328464FA992224346F9F762FA58
:1032C000FFF756FD74B0BDE8F08100BF2DE9F04373
:1032D000B7B0054688461446FFF7A0FB8146FFF7C6
:1032E0009DFB074628460B210DF1C202F9F7E6FBCC
:1032F000B4F80560BDF8C220964240F0B4800DF1EC
:103300000A03009328461CA94F2203ABF9F7DEFA03
:10331000E378D12B40F0A780607810F0800F06D0C2
:1033200000F07F001CA9BDF8C220FFF73FFD1CA8DC
:1033300007F12101062203F06FFF002840F093807F
:103340000DF1770007F1430104F000F9002840F087
:103350008A800DF1C40E4E4656F8210F7168B2688E
:10336000F368AEE80F00338AAEF80030FFF7DAFBFF
:103370000DF1C40EBEE80F00C9F821007160B26003
:10338000F360BEF800303382FFF7EAFB2068049058
:10339000A288A379ADF814208DF81630D8F8003043
:1033A000CDF81730B8F80430ADF81B30DDF88730B1
:1033B000CDF81D30BDF88B30ADF821300DF18D0307
:1033C0000DF123020DF1BD01D3F800C0D3F804E0E4
:1033D0009E68D868C2F800C0C2F804E09660D06069
:1033E000103310328B42EFD11B881380002004A9C8
:1033F0004522FDF75FFE062363710023A371552369
:10340000237157F8210F1690BB88ADF85C306078B7
:1034100010F0800F05D000F07F0016A90622FFF7FC
:10342000B7FC20681890A288A379ADF864208DF8C5
:10343000663036AB53F8800DCDF867009B88ADF849
:103440006B30A37823B94046FF21042203F0FCFE31
:10345000B8F804300093284618A90D224346F9F71E
:1034600091F9FFF785FC37B0BDE8F0832DE9F04115
:1034700090B0054688461446FFF7D0FA074628461E
:103480000B210DF13E02F9F719FBB4F80560BDF808
:103490003E2096425FD10DF10A030093284606A90B
:1034A000172203ABF9F712FA607810F0800F06D0FC
:1034B00000F07F0006A9BDF83E20FFF777FC06A8C4
:1034C00007F12101062203F0A7FE002843D10DF1E8
:1034D0001F0007F1430104F039F800283BD1FFF742
:1034E000A1FAFFF73DFB062363710023A371552367
:1034F000237157F8210F0490BB88ADF81430607821
:1035000010F0800F05D000F07F0004A90622FFF71D
:103510003FFC20680C90A288A379ADF834208DF888
:10352000363010AB53F8300DCDF837009B88ADF82E
:103530003B30A37823B94046FF21042203F084FEE8
:10354000B8F80430009328460CA90D224346F9F739
:1035500019F9FFF70DFC10B0BDE8F08110B588B087
:1035600004460A210DF11F02F9F7A8FA9DF81F3051
:10357000002B51D0222B56D12046092107AAF9F75A
:103580009DFABDF81C30062B4DD906AB00932046A2
:1035900003A9072205ABF9F799F99DF80C30A52B83
:1035A00041D19DF81030AA2B3DD19DF80F3003F08A
:1035B000F003C02B18D004D8A02B09D0B02B0DD00D
:1035C00031E0E02B1CD0F02B20D0D02B2BD111E000
:1035D000204605A903AAFFF767FC24E0204605A9B9
:1035E00003AAFFF7F1FB1EE0204605A903AAFFF797
:1035F000E5FD18E0204605A903AAFFF767FE12E0E3
:10360000204605A903AAFFF765FD0CE0204605A9A1
:1036100003AAFFF72BFF06E02046022141F696128F
:103620000023F8F719FE08B010BD00BF2DE9F047E0
:1036300084B004460F4603F09BFF073808282DD8B6
:103640006846214603F08CFF6846194903F0ECFFF9
:10365000044600263546DFF85C80DFF854A0B1460A
:103660000EE0204603F0A0FDFF2819D807B17855D9
:1036700006440135EDB24846514603F0D5FF0446F5
:103680002CB14046214600F071F80028E9D0042D05
:1036900008D1002E14BF0020FF2004E0FF2002E02C
:1036A000FF2000E0FF2040B204B0BDE8F08700BF7B
:1036B0002C8F0108D17101082DE9F04387B0044631
:1036C0000F4603F055FF11282BD101A8214603F026
:1036D00047FF01A8164903F0A7FF04460025DFF8BD
:1036E00054802E46DFF848900FE0204631461022E5
:1036F00004F07AF8FF2816D807B178550135EDB2F5
:103700003046494603F090FF04462CB1404621461E
:1037100000F02CF80028E8D0062D0CBF0020FF2078
:1037200002E0FF2000E0FF2040B207B0BDE8F083D8
:10373000E4B00108E571010810B40028BABF4042A6
:1037400001220022002308E0013292B290FBF1F046
:1037500008B9D0B205E001339BB21CB2FE2CF3DDF8
:10376000FF2040B25DF8044B704700BF38B50C46EF
:10377000054658B169B10B7823B90DE040B2A847AE
:1037800068B1013420780028F8D138BD4FF0FF30FF
:1037900038BD4FF0FF3038BD4FF0FF3038BD4FF02F
:1037A000FF3038BDF0B484460068B0B10646771CDF
:1037B00096F900500B465C1C93F90020AA4207D1F1
:1037C00015B10023337000E00027CCF8007005E04D
:1037D0002346002AEFD13E46E9E70020F0BC7047BF
:1037E0002DE9F84F0646DFF86491DFF86481DFF8D1
:1037F00058A12AE09AF800200232121B4E4B1340C7
:1038000003D5013B63F0010301335FB24B4B53F827
:1038100027509DB1284603F0ABFEB8F80030181AC7
:10382000431EA8F80030284603F0EEFC0022434B6C
:1038300043F82720013C89F8004006E04048414910
:10384000E02203F0A1FD30BFFDE799F80040012C14
:10385000D0D824B1B8F900303344F92BCADC3A4B44
:103860001C78A04606F1010A504603F0C5FC334B14
:1038700043F82400354F1D4632E008F10203C9EB3E
:1038800003092D4B19EA030B05D50BF1FF3B6BF038
:10389000010B0BF1010B4FFA8BFB55F82B90B9F193
:1038A000000F16D0484603F063FE294B1A88101A01
:1038B000421E1A80484603F0A7FC002345F82B302F
:1038C0003B78013B3B70504603F096FC45F82800DE
:1038D00006E020481B49ED2203F056FD30BFFDE70E
:1038E00097F80090B9F1000F03D055F82830002B5D
:1038F000C3D0124B53F8240030B917481149F022B5
:1039000003F042FD30BFFDE7144903F029FE012C0E
:1039100003D100220C4B1A7002E001340A4B1C70D8
:1039200009F10109094B83F80090094B1A883244C8
:1039300001321A80BDE8F88F0100008020130020BA
:10394000E4B10108B0B101081D13002028130020C4
:103950001E13002008B201082CB20108B812002082
:1039600070B59AB0044619903D2103F0E2FD18B1FC
:103970000322B44BDA7510E020463F2103F0D9FD55
:1039800018B10122AF4BDA7507E020462D2103F074
:10399000D0FD10B10222AB4BDA7519A8AA49FFF786
:1039A00001FF064678B9FD2096E15DB20C682C4413
:1039B000647804F00304022C06BF2B46203B5BB264
:1039C00002F8013B01E00246A0491378002BECD13C
:1039D000304603F0CDFD0A280BD896F90030412B74
:1039E00007D196F90130542B03D196F902302B2BD5
:1039F0003FD096F90030412B36D196F90130542B47
:103A000032D1B378002B2FD18E4BDB7D5AB2012AF5
:103A100021D18F4B1B78012B05D88E480821FDF74B
:103A200027FE022058E18C4B1B78012B84BF023B00
:103A3000DBB28A4A52F82340204603F099FD024641
:103A400068468749234603F043FDC1B26846FDF747
:103A50000FFE022040E1002B40F03D81814805210E
:103A6000FDF706FE022037E17F48314603F078FD7E
:103A700003E07D48F11C03F073FD19A87B49FFF7B3
:103A800091FE0446002800F0188103F071FD232800
:103A900016D96C48002380F8443080F82030C37574
:103AA000037680F8A43080F8903080F87C3080F87D
:103AB000683020306E49012203F00AFDFB200BE143
:103AC0006C48214603F04CFD19A86849FFF76AFECF
:103AD0000446002800F0F38003F04AFD232816D99D
:103AE0005848002380F8443080F82030C3750376AE
:103AF00080F8A43080F8903080F87C3080F868300E
:103B000020305B49022203F0E3FCFB20E4E05A484A
:103B1000214603F025FD19A85449FFF743FE04464A
:103B2000002800F0CE8003F023FD132816D9454865
:103B3000002380F8443080F82030C375037680F885
:103B4000A43080F8903080F87C3080F868302030E5
:103B50004749032203F0BCFCFB20BDE04748214657
:103B600003F0FEFC19A84149FFF71CFE044600289B
:103B700000F0A98003F0FCFC132816D9314800237B
:103B800080F8443080F82030C375037680F8A43084
:103B900080F8903080F87C3080F8683020303449EC
:103BA000042203F095FCFB2096E03548214603F003
:103BB000D7FC19A82D49FFF7F5FD0446002800F0B1
:103BC000848003F0D5FC132816D91E48002380F802
:103BD000443080F82030C375037680F8A43080F834
:103BE000903080F87C3080F8683020302049052201
:103BF00003F06EFCFB206FE02248214603F0B0FC8E
:103C000019A81A49FFF7CEFD044600285FD003F03B
:103C1000AFFC132838D90B48002380F8443080F8D3
:103C20002030C375037680F8A43080F8903080F897
:103C30007C3080F8683020300D49062203F048FCC3
:103C4000FB2049E0902E002050B201082002002005
:103C50002813002054B201081D1300202013002057
:103C600060B2010870B20108A82E0020649101081A
:103C7000289C0108B02E0020D42E0020F82E002011
:103C80000C2F0020202F00201548214603F068FC4F
:103C9000199B1B78EBB1134B002283F8442083F867
:103CA0002020DA751A7683F8A42083F8902083F810
:103CB0007C2083F86820FB200EE000200CE0002030
:103CC0000AE0002008E0002006E0002004E00020D8
:103CD00002E0002000E0FC2040B21AB070BD00BF3E
:103CE000342F0020902E002008B5104800216422B7
:103CF00003F0AAFA00230E48194604E05AB240F82D
:103D000022100133DBB25AB2012AF7DD094BFF2240
:103D100083F8B820012283F8CE2083F8D020064A09
:103D2000C3F8C020054AC3F8C42008BDB81200205B
:103D300020130020902E00208C2A0020642F0020C9
:103D4000F8B50E469C4B93F920E093F94470003788
:103D500018BF012793F9685093F97C1093F99020CC
:103D600093F9A440BEF1000F0CBF3B467B1C002D15
:103D700018BF0133002918BF0133002A18BF0133CF
:103D8000002C0CBF1C465C1C5B228C4B1A70051E61
:103D90003DDB15B953225A701EE0032D07D1884828
:103DA00088494FF4BF7203F0EFFA30BFFDE7042DEE
:103DB00003D15722814B5A700EE0052D03D15222B8
:103DC0007E4B5A7008E080487E4940F281122B46B3
:103DD00003F0DAFA30BFFDE7B6F1FF3F0FD07748C6
:103DE0002C23837003307949324603F071FB30464F
:103DF0000A21FFF7A1FC033000F0FF03B9E0002C1B
:103E000000F0B6802C226D4B9A700323B1E06B4B0F
:103E100046225A702C229A70B6F1FF3F0CD0D81C63
:103E20006A49324603F054FB30460A21FFF784FC0E
:103E3000033000F0FF0300E003235A1CD2B22C2011
:103E40005E49C8541E351C2D00F28C80DFE805F059
:103E5000808A8A8A8A766C62584F458A8A8A8A8AD8
:103E60008A8A8A8A3F39332D27211B150F00531C5C
:103E7000DBB23020514988547BE0531CDBB2312047
:103E80004E49885475E0531CDBB232204B498854AC
:103E90006FE0531CDBB233204849885469E0531C5F
:103EA000DBB234204549885463E0531CDBB2352033
:103EB000424988545DE0531CDBB236203F498854A8
:103EC00057E0531CDBB237203C49885451E0531C67
:103ED000DBB23820394988544BE0511CC9B237480D
:103EE000312383544B1CDBB23022425441E0511C3D
:103EF000C9B23248312585544B1CDBB2455438E0F9
:103F0000511CC9B22D48312383544B1CDBB23222E1
:103F100042542EE0511CC9B22848312383544B1C13
:103F2000DBB23322425424E0511CC9B2234831236E
:103F300083544B1CDBB2342242541AE0511CC9B2E8
:103F40001E48312383544B1CDBB23522425410E00F
:103F5000511CC9B21948322383544B1CDBB23022A6
:103F6000425406E0531CDBB230201449885400E070
:103F70000223114A92F8202072B35E1CF6B22C2163
:103F80000E4AD154124803F0F3FA0246C5B2232D6B
:103F900007D910480B494FF4D47203F0F5F930BF3C
:103FA000FDE7064830440A49D2B203F044F97319D8
:103FB000DBB2013CE4B215E0902E0020B8120020E4
:103FC0009CB20108E8B00108D0B20108289C0108A1
:103FD000B02E002004B3010824B15A1C2C207049D3
:103FE000C854D3B26F4A92F84420F2B15E1CF6B2C4
:103FF0002C216B4AD1546C4803F0BAFA0246C5B280
:10400000232D07D969486A4940F2A91203F0BCF987
:1040100030BFFDE7624830446349D2B203F00BF988
:104020007319DBB2013CE4B205E024B15A1C2C2028
:104030005B49C854D3B25B4A92F86820F2B15E1C67
:10404000F6B22C21564AD1545A4803F091FA02464E
:10405000C5B2132D07D9554855494FF4D57203F011
:1040600093F930BFFDE74E4830445249D2B203F0D5
:10407000E2F87319DBB2013CE4B205E024B15A1C4A
:104080002C204749C854D3B2464A92F87C20F2B15A
:104090005E1CF6B22C21424AD154474803F068FA1C
:1040A0000246C5B2132D07D94048414940F2AB1230
:1040B00003F06AF930BFFDE7394830443E49D2B2D7
:1040C00003F0B9F87319DBB2013CE4B205E024B1A6
:1040D0005A1C2C203249C854D3B2324A92F890204C
:1040E000F2B15E1CF6B22C212D4AD154334803F0B4
:1040F0003FFA0246C5B2132D07D92C482C494FF47C
:10410000D67203F041F930BFFDE7254830442B4912
:10411000D2B203F090F87319DBB2013CE4B205E0CF
:1041200024B15A1C2C201E49C854D3B21D4A92F8FF
:10413000A420E2B15D1CEDB22C21194AD1542048D3
:1041400003F016FA0246C4B2132C07D917481849CF
:1041500040F2AD1203F018F930BFFDE710482844D3
:104160001749D2B203F067F82B19DBB205E024B18E
:104170005A1C2C200A49C854D3B25A1CD2B2084C3B
:104180005D21E1540023A354204603F0F1F90146D8
:104190002046FDF76DFA0B480221FDF769FAF8BDDC
:1041A000B8120020902E0020D42E002004B3010865
:1041B000E8B00108F82E00200C2F0020202F00204E
:1041C000342F00207C92010810B5844BDB7DB3B9FD
:1041D000824B002283F8442083F82020DA751A7677
:1041E00083F8A42083F8902083F87C2083F868204B
:1041F0006FF003004FF0FF31FFF7A2FD10BD5AB280
:10420000012A16D1754B002283F8442083F8202020
:10421000DA751A7683F8A42083F8902083F87C203E
:1042200083F868206FF003004FF0FF31FFF788FD3F
:1042300010BD5AB2022A16D1684B002283F84420DE
:1042400083F82020DA751A7683F8A42083F890206A
:1042500083F87C2083F868206FF003004FF0FF3173
:10426000FFF76EFD10BD5AB2032A40F0AE805B4BE3
:1042700093F82030002B45D059485A49FFF776FA79
:10428000D8B15648002380F8443080F82030C375F8
:10429000037680F8A43080F8903080F87C3080F885
:1042A000683020305049012203F012F96FF0040009
:1042B0004FF0FF31FFF744FD10BD4A4802F074FF94
:1042C000C4B263B2102B01DC002B1CDC434800237A
:1042D00080F8443080F82030C375037680F8A4302D
:1042E00080F8903080F87C3080F8683020303E498B
:1042F000012203F0EDF86FF005004FF0FF31FFF7FA
:104300001FFD10BDFF24354B93F84430002B46D0E1
:1043100033483649FFF72AFAD8B13048002380F8ED
:10432000443080F82030C375037680F8A43080F8DC
:10433000903080F87C3080F8683020302A490222A2
:1043400003F0C6F86FF004004FF0FF31FFF7F8FC00
:1043500010BD264802F028FFC1B24BB2012B02DC8F
:1043600011F0800F1CD01D48002380F8443080F8E5
:104370002030C375037680F8A43080F8903080F840
:104380007C3080F8683020301749022203F0A0F812
:104390006FF005004FF0FF31FFF7D2FC10BDFF2199
:1043A0000E4B002283F8442083F82020DA751A7619
:1043B00083F8A42083F8902083F87C2083F8682079
:1043C00060B249B202F04AFD10BD0948094940F205
:1043D00059325BB202F0D8FF30BFFDE7902E0020CB
:1043E000D1710108B02E0020289C0108D42E002095
:1043F00030B30108E0B3010810B5844BDB7DB3B9DD
:10440000824B002283F8442083F82020DA751A7644
:1044100083F8A42083F8902083F87C2083F8682018
:104420006FF003004FF0FF31FFF78AFC10BD5AB266
:10443000012A16D1754B002283F8442083F82020EE
:10444000DA751A7683F8A42083F8902083F87C200C
:1044500083F868206FF003004FF0FF31FFF770FC26
:1044600010BD5AB2022A16D1684B002283F84420AC
:1044700083F82020DA751A7683F8A42083F8902038
:1044800083F87C2083F868206FF003004FF0FF3141
:10449000FFF756FC10BD5AB2032A40F0AD805B4BCB
:1044A00093F82030002B45D059485A49FFF75EF960
:1044B000D8B15648002380F8443080F82030C375C6
:1044C000037680F8A43080F8903080F87C3080F853
:1044D000683020305049012202F0FAFF6FF00400EA
:1044E0004FF0FF31FFF72CFC10BD4A4802F05CFE94
:1044F000C4B263B2102B01DC002B1CDC4348002348
:1045000080F8443080F82030C375037680F8A430FA
:1045100080F8903080F87C3080F8683020303E4958
:10452000012202F0D5FF6FF005004FF0FF31FFF7D9
:1045300007FC10BDFF24354B93F84430002B45D0C9
:1045400033483649FFF712F9D8B13048002380F8D4
:10455000443080F82030C375037680F8A43080F8AA
:10456000903080F87C3080F8683020302A49022270
:1045700002F0AEFF6FF004004FF0FF31FFF7E0FBF9
:1045800010BD264802F010FEC1B24BB2022B01DC76
:10459000002B1CDC1D48002380F8443080F82030BC
:1045A000C375037680F8A43080F8903080F87C30B2
:1045B00080F8683020301849022202F089FF6FF03D
:1045C00005004FF0FF31FFF7BBFB10BDFF210F4B84
:1045D000002283F8442083F82020DA751A7683F8C5
:1045E000A42083F8902083F87C2083F8682060B2B0
:1045F00049B202F00FFC10BD09480A494FF451724C
:104600005BB202F0C1FE30BFFDE700BF902E00207C
:10461000D1710108B02E0020289C0108D42E002062
:1046200030B30108D4B3010808B5154BDB7D83B95D
:1046300000204FF0FF31FFF783FBBFF34F8F114A8C
:10464000D16801F4E061104B0B43D360BFF34F8F8F
:10465000FEE70B4B002283F8442083F82020DA7514
:104660001A7683F8A42083F8902083F87C2083F8BE
:1046700068206FF003004FF0FF31FFF761FB08BDCA
:10468000902E002000ED00E00400FA0508B5164B5E
:10469000DB7D93B9144B002283F8442083F820205B
:1046A000DA751A7683F8A42083F8902083F87C20AA
:1046B00083F8682002F09EFB08BD0B4B002283F8B4
:1046C000442083F82020DA751A7683F8A42083F832
:1046D000902083F87C2083F868206FF003004FF06F
:1046E000FF31FFF72DFB08BD902E002010B5FEF71F
:1046F00095F90446C24BDB7D13B90122C04BDA7534
:10470000BF4BDB7D5AB2012A60D1BD4B93F82030FC
:10471000002B45D0BB48BC49FFF728F8D8B1B848B2
:10472000002380F8443080F82030C375037680F889
:10473000A43080F8903080F87C3080F868302030E9
:10474000B249012202F0C4FE6FF004004FF0FF31C5
:10475000FFF7F6FA10BDAC4802F026FDC1B24BB22D
:10476000052B01DC002B1CDCA548002380F844301D
:1047700080F82030C375037680F8A43080F890303C
:1047800080F87C3080F868302030A049012202F0A7
:104790009FFE6FF005004FF0FF31FFF7D1FA10BD1B
:1047A000FF21974B002283F8442083F82020DA75FC
:1047B0001A7683F8A42083F8902083F87C2083F86D
:1047C0006820934849B202F077FA10BD5AB2022A23
:1047D00040F0B2828A4B93F82030002B00F08282A6
:1047E00088488949FEF7C2FFD8B18548002380F880
:1047F000443080F82030C375037680F8A43080F808
:10480000903080F87C3080F8683020307F49012279
:1048100002F05EFE6FF004004FF0FF31FFF790FAF8
:1048200010BD794802F0C0FCC0B243B2052B01DCD8
:10483000002B1BDC7248002380F8443080F82030C5
:10484000C375037680F8A43080F8903080F87C300F
:1048500080F8683020306D49012202F039FE6FF097
:1048600005004FF0FF31FFF76BFA10BD43B2012B8B
:1048700064D164486749FEF779FFD8B160480023E6
:1048800080F8443080F82030C375037680F8A43077
:1048900080F8903080F87C3080F8683020305B49B8
:1048A000022202F015FE6FF004004FF0FF31FFF717
:1048B00047FA10BD574802F077FC0023564908E03C
:1048C00051F82320824203D1C4F83B00012303E0C6
:1048D00001330A2BF4D90023D3B9494880F8443076
:1048E00080F82030C375037680F8A43080F89030CB
:1048F00080F87C3080F8683020304449022202F091
:10490000E7FD6FF004004FF0FF31FFF719FA10BD1B
:104910003B4B002283F8442083F82020DA751A7676
:1049200083F8A42083F8902083F87C2083F8682003
:10493000374804F13B0102F047FA10BD43B2022BA5
:104940006CD130483349FEF711FFD8B12C48002311
:1049500080F8443080F82030C375037680F8A430A6
:1049600080F8903080F87C3080F86830203027491B
:10497000022202F0ADFD6FF004004FF0FF31FFF7AF
:10498000DFF910BD234802F00FFCC3B25AB2092A66
:1049900001DC072A1BDC1A48002380F8443080F829
:1049A0002030C375037680F8A43080F8903080F80A
:1049B0007C3080F8683020301449022202F088FDF3
:1049C0006FF005004FF0FF31FFF7BAF910BD84F822
:1049D0003F000B4B002283F8442083F82020DA7537
:1049E0001A7683F8A42083F8902083F87C2083F83B
:1049F0006820074804F13B0102F0E6F910BD00BF52
:104A0000902E0020D1710108B02E0020289C0108B2
:104A100000440040D42E0020A001002043B2032B0C
:104A200040F08180BD48BE49FEF7A0FED8B1BD4828
:104A3000002380F8443080F82030C375037680F876
:104A4000A43080F8903080F87C3080F868302030D6
:104A5000B549022202F03CFD6FF004004FF0FF3137
:104A6000FFF76EF910BDAF4B93F84530ABB9AD4BC6
:104A700093F844305AB2AD4909680A44527802F0BA
:104A80000302022A5BB208BF203BDBB25AB24E2AB5
:104A90001FD04F2A1DD0452A1BD0A248002380F8E2
:104AA000443080F82030C375037680F8A43080F855
:104AB000903080F87C3080F8683020309A490222AB
:104AC00002F006FD6FF004004FF0FF31FFF738F9F8
:104AD00010BD5AB24E2A03D1002384F840300CE0B6
:104AE0005AB24F2A03D1012384F8403005E05BB26B
:104AF000452B04BF022384F840308A4B002283F800
:104B0000442083F82020DA751A7683F8A42083F8ED
:104B1000902083F87C2083F86820854804F13B01CD
:104B200002F052F910BD43B2042B5DD181487C499B
:104B3000FEF71CFED8B17B48002380F8443080F893
:104B40002030C375037680F8A43080F8903080F868
:104B50007C3080F8683020307349022202F0B8FCC3
:104B60006FF004004FF0FF31FFF7EAF810BD6C481A
:104B700002F01AFBC3B25AB2022A01DC002A1BDC83
:104B80006848002380F8443080F82030C3750376ED
:104B900080F8A43080F8903080F87C3080F868305D
:104BA00020306149022202F093FC6FF005004FF0C3
:104BB000FF31FFF7C5F810BD84F84100594B0022C2
:104BC00083F8442083F82020DA751A7683F8A4202D
:104BD00083F8902083F87C2083F86820544804F1FF
:104BE0003B0102F0F1F810BD40B205285ED15148FA
:104BF0004B49FEF7BBFDD8B14A48002380F844304A
:104C000080F82030C375037680F8A43080F89030A7
:104C100080F87C3080F8683020304349022202F06E
:104C200057FC6FF004004FF0FF31FFF789F810BD1B
:104C30003B4802F0B9FAC3B25AB2032A02DC13F0BD
:104C4000800F1BD03748002380F8443080F8203094
:104C5000C375037680F8A43080F8903080F87C30FB
:104C600080F8683020303049022202F031FC6FF0C9
:104C700005004FF0FF31FFF763F810BD84F84200E4
:104C8000284B002283F8442083F82020DA751A7616
:104C900083F8A42083F8902083F87C2083F8682090
:104CA000234804F13B0102F08FF810BD1D4800239A
:104CB00080F8443080F82030C375037680F8A43043
:104CC00080F8903080F87C3080F8683020301649C9
:104CD000022202F0FDFB6FF007004FF0FF31FFF7FB
:104CE0002FF810BD0F48002380F8443080F82030A2
:104CF000C375037680F8A43080F8903080F87C305B
:104D000080F8683020300849012202F0E1FB6FF0A2
:104D100004004FF0FF31FFF713F810BDBD7101081B
:104D2000D42E0020902E0020289C01082002002074
:104D300000440040D17101085AB2032A40F0DC81DE
:104D4000C34B93F82030002B4ED0C248C249FEF727
:104D50000DFDD8B1BE48002380F8443080F82030E3
:104D6000C375037680F8A43080F8903080F87C30EA
:104D700080F868302030B949012202F0A9FB6FF0B9
:104D800004004FF0FF31FEF7DBFF10BDB24802F028
:104D90000BFA0023B24908E051F82320824203D1E4
:104DA000C4F83B00012303E001330A2BF4D90023AC
:104DB000D3B9A74880F8443080F82030C375037613
:104DC00080F8A43080F8903080F87C3080F868302B
:104DD0002030A249012202F07BFB6FF004004FF06B
:104DE000FF31FEF7ADFF10BD994B93F84430002B17
:104DF00047D098489B49FEF7B9FCD8B194480023A6
:104E000080F8443080F82030C375037680F8A430F1
:104E100080F8903080F87C3080F8683020308F49FE
:104E2000022202F055FB6FF004004FF0FF31FEF755
:104E300087FF10BD8B4802F0B7F9C3B25AB2092AF6
:104E400001DC072A1BDC8248002380F8443080F80C
:104E50002030C375037680F8A43080F8903080F855
:104E60007C3080F8683020307C49022202F030FB30
:104E70006FF005004FF0FF31FEF762FF10BD84F8C0
:104E80003F00734B93F86830002B6DD0764877491C
:104E9000FEF76CFCD8B16E48002380F8443080F8EF
:104EA0002030C375037680F8A43080F8903080F805
:104EB0007C3080F8683020306849032202F008FB1B
:104EC0006FF004004FF0FF31FEF73AFF10BD604B6A
:104ED00093F86930C3B95E4B93F868305AB26449AD
:104EE00009680A44527802F00302022A5BB208BF42
:104EF000203BDBB2564A82F868305AB24E2A1FD0A5
:104F00004F2A1DD0452A1BD05148002380F8443039
:104F100080F82030C375037680F8A43080F8903094
:104F200080F87C3080F8683020304C49032202F051
:104F3000CFFA6FF004004FF0FF31FEF701FF10BD14
:104F40005AB24E2A03D1002384F840300CE05AB202
:104F50004F2A03D1012384F8403005E05BB2452B92
:104F600004BF022384F84030394B93F87C30002B87
:104F700047D038483F49FEF7F9FBD8B13448002301
:104F800080F8443080F82030C375037680F8A43070
:104F900080F8903080F87C3080F8683020302F49DD
:104FA000042202F095FA6FF004004FF0FF31FEF793
:104FB000C7FE10BD2F4802F0F7F8C3B25AB2022A5A
:104FC00001DC002A1BDC2248002380F8443080F8F2
:104FD0002030C375037680F8A43080F8903080F8D4
:104FE0007C3080F8683020301C49042202F070FACE
:104FF0006FF005004FF0FF31FEF7A2FE10BD84F800
:105000004100134B93F89030002B5FD011481A49A0
:10501000FEF7ACFB90B30E48002380F8443080F8D4
:105020002030C375037680F8A43080F8903080F883
:105030007C3080F8683020300849052202F048FAB8
:105040006FF004004FF0FF31FEF77AFE10BD00BF95
:10505000902E0020D1710108B02E0020289C01085C
:10506000A0010020D42E0020BD710108F82E0020E0
:10507000200200200C2F0020202F0020234802F0C7
:1050800093F8C3B25AB2032A02DC13F0800F1BD08C
:105090001F48002380F8443080F82030C375037621
:1050A00080F8A43080F8903080F87C3080F8683048
:1050B00020301849052202F00BFA6FF005004FF07E
:1050C000FF31FEF73DFE10BD84F84200104B002278
:1050D00083F8442083F82020DA751A7683F8A42018
:1050E00083F8902083F87C2083F868200A4804F134
:1050F0003B0101F069FE10BD0848094940F21E322B
:105100005BB202F041F930BFFDE700BF202F002065
:10511000902E0020289C01080044004030B3010874
:10512000C0B1010810B5FDF779FC0446C24BDB7D28
:1051300013B90122C04BDA75BF4BDB7D5AB2012A8D
:1051400060D1BD4B93F82030002B45D0BB48BC4903
:10515000FEF70CFBD8B1B848002380F8443080F843
:105160002030C375037680F8A43080F8903080F842
:105170007C3080F868302030B249012202F0A8F972
:105180006FF004004FF0FF31FEF7DAFD10BDAC48C0
:1051900002F00AF8C1B24BB2052B01DC002B1CDC7B
:1051A000A548002380F8443080F82030C37503768A
:1051B00080F8A43080F8903080F87C3080F8683037
:1051C0002030A049012202F083F96FF005004FF072
:1051D000FF31FEF7B5FD10BDFF21974B002283F88C
:1051E000442083F82020DA751A7683F8A42083F807
:1051F000902083F87C2083F86820934849B201F01E
:105200005BFD10BD5AB2022A40F0B2828A4B93F87D
:105210002030002B00F0828288488949FEF7A6FAE8
:10522000D8B18548002380F8443080F82030C37519
:10523000037680F8A43080F8903080F87C3080F8D5
:10524000683020307F49012202F042F96FF00400FB
:105250004FF0FF31FEF774FD10BD794801F0A4FF57
:10526000C0B243B2052B01DC002B1BDC72480023CB
:1052700080F8443080F82030C375037680F8A4307D
:1052800080F8903080F87C3080F8683020306D49AC
:10529000012202F01DF96FF005004FF0FF31FEF71B
:1052A0004FFD10BD43B2012B64D164486749FEF73E
:1052B0005DFAD8B16048002380F8443080F820308F
:1052C000C375037680F8A43080F8903080F87C3085
:1052D00080F8683020305B49022202F0F9F86FF064
:1052E00004004FF0FF31FEF72BFD10BD574801F0D1
:1052F0005BFF0023564908E051F82320824203D186
:10530000C4F83300012303E001330A2BF4D900234E
:10531000D3B9494880F8443080F82030C37503760B
:1053200080F8A43080F8903080F87C3080F86830C5
:1053300020304449022202F0CBF86FF004004FF015
:10534000FF31FEF7FDFC10BD3B4B002283F84420EB
:1053500083F82020DA751A7683F8A42083F8902049
:1053600083F87C2083F86820374804F1330101F08A
:105370002BFD10BD43B2022B6CD130483349FEF7F0
:10538000F5F9D8B12C48002380F8443080F820305B
:10539000C375037680F8A43080F8903080F87C30B4
:1053A00080F8683020302749022202F091F86FF02F
:1053B00004004FF0FF31FEF7C3FC10BD234801F09D
:1053C000F3FEC3B25AB2092A01DC072A1BDC1A48D1
:1053D000002380F8443080F82030C375037680F8CD
:1053E000A43080F8903080F87C3080F8683020302D
:1053F0001449022202F06CF86FF005004FF0FF3103
:10540000FEF79EFC10BD84F837000B4B002283F89A
:10541000442083F82020DA751A7683F8A42083F8D4
:10542000902083F87C2083F86820074804F133013A
:1054300001F0CAFC10BD00BF902E0020D171010800
:10544000B02E0020289C010800380140D42E0020F6
:10545000A001002043B2032B40F08180BD48BE492B
:10546000FEF784F9D8B1BD48002380F8443080F8B5
:105470002030C375037680F8A43080F8903080F82F
:105480007C3080F868302030B549022202F020F8E4
:105490006FF004004FF0FF31FEF752FC10BDAF4B30
:1054A00093F84530ABB9AD4B93F844305AB2AD499F
:1054B00009680A44527802F00302022A5BB208BF6C
:1054C000203BDBB25AB24E2A1FD04F2A1DD0452AAC
:1054D0001BD0A248002380F8443080F82030C375E8
:1054E000037680F8A43080F8903080F87C3080F823
:1054F000683020309A49022201F0EAFF6FF0040080
:105500004FF0FF31FEF71CFC10BD5AB24E2A03D1FA
:10551000002384F838300CE05AB24F2A03D101231B
:1055200084F8383005E05BB2452B04BF022384F8D1
:1055300038308A4B002283F8442083F82020DA7523
:105540001A7683F8A42083F8902083F87C2083F8CF
:105550006820854804F1330101F036FC10BD43B2E8
:10556000042B5DD181487C49FEF700F9D8B17B4816
:10557000002380F8443080F82030C375037680F82B
:10558000A43080F8903080F87C3080F8683020308B
:105590007349022201F09CFF6FF004004FF0FF31CD
:1055A000FEF7CEFB10BD6C4801F0FEFDC3B25AB24F
:1055B000022A01DC002A1BDC6848002380F8443002
:1055C00080F82030C375037680F8A43080F89030DE
:1055D00080F87C3080F8683020306149022201F088
:1055E00077FF6FF005004FF0FF31FEF7A9FB10BD0C
:1055F00084F83900594B002283F8442083F8202096
:10560000DA751A7683F8A42083F8902083F87C203A
:1056100083F86820544804F1330101F0D5FB10BD34
:1056200040B205285ED151484B49FEF79FF8D8B1EA
:105630004A48002380F8443080F82030C375037650
:1056400080F8A43080F8903080F87C3080F86830A2
:1056500020304349022201F03BFF6FF004004FF07D
:10566000FF31FEF76DFB10BD3B4801F09DFDC3B25D
:105670005AB2032A02DC13F0800F1BD037480023F4
:1056800080F8443080F82030C375037680F8A43069
:1056900080F8903080F87C3080F8683020303049D5
:1056A000022201F015FF6FF005004FF0FF31FEF709
:1056B00047FB10BD84F83A00284B002283F84420B1
:1056C00083F82020DA751A7683F8A42083F89020D6
:1056D00083F87C2083F86820234804F1330101F02B
:1056E00073FB10BD1D48002380F8443080F8203043
:1056F000C375037680F8A43080F8903080F87C3051
:1057000080F8683020301649022201F0E1FE6FF087
:1057100007004FF0FF31FEF713FB10BD0F480023C9
:1057200080F8443080F82030C375037680F8A430C8
:1057300080F8903080F87C3080F86830203008495C
:10574000012201F0C5FE6FF004004FF0FF31FEF7BB
:10575000F7FA10BDBD710108D42E0020902E002054
:10576000289C01082002002000380140D171010866
:105770005AB2032A40F0DC81C34B93F82030002B4F
:105780004ED0C248C249FDF7F1FFD8B1BE48002350
:1057900080F8443080F82030C375037680F8A43058
:1057A00080F8903080F87C3080F868302030B9493B
:1057B000012201F08DFE6FF004004FF0FF31FEF783
:1057C000BFFA10BDB24801F0EFFC0023B24908E077
:1057D00051F82320824203D1C4F83300012303E0AF
:1057E00001330A2BF4D90023D3B9A74880F84430F9
:1057F00080F82030C375037680F8A43080F89030AC
:1058000080F87C3080F868302030A249012201F015
:105810005FFE6FF004004FF0FF31FEF791FA10BD0C
:10582000994B93F84430002B47D098489B49FDF79B
:105830009DFFD8B19448002380F8443080F8203090
:10584000C375037680F8A43080F8903080F87C30FF
:1058500080F8683020308F49022201F039FE6FF065
:1058600004004FF0FF31FEF76BFA10BD8B4801F0DA
:105870009BFCC3B25AB2092A01DC072A1BDC82480E
:10588000002380F8443080F82030C375037680F818
:10589000A43080F8903080F87C3080F86830203078
:1058A0007C49022201F014FE6FF005004FF0FF3139
:1058B000FEF746FA10BD84F83700734B93F8683052
:1058C000002B6DD076487749FDF750FFD8B16E4870
:1058D000002380F8443080F82030C375037680F8C8
:1058E000A43080F8903080F87C3080F86830203028
:1058F0006849032201F0ECFD6FF004004FF0FF3126
:10590000FEF71EFA10BD604B93F86930C3B95E4BC9
:1059100093F868305AB2644909680A44527802F030
:105920000302022A5BB208BF203BDBB2564A82F870
:1059300068305AB24E2A1FD04F2A1DD0452A1BD09C
:105940005148002380F8443080F82030C375037636
:1059500080F8A43080F8903080F87C3080F868308F
:1059600020304C49032201F0B3FD6FF004004FF0EA
:10597000FF31FEF7E5F910BD5AB24E2A03D10023DC
:1059800084F838300CE05AB24F2A03D1012384F84E
:10599000383005E05BB2452B04BF022384F8383071
:1059A000394B93F87C30002B47D038483F49FDF7FE
:1059B000DDFED8B13448002380F8443080F8203030
:1059C000C375037680F8A43080F8903080F87C307E
:1059D00080F8683020302F49042201F079FD6FF003
:1059E00004004FF0FF31FEF7ABF910BD2F4801F076
:1059F000DBFBC3B25AB2022A01DC002A1BDC2248BC
:105A0000002380F8443080F82030C375037680F896
:105A1000A43080F8903080F87C3080F868302030F6
:105A20001C49042201F054FD6FF005004FF0FF31D6
:105A3000FEF786F910BD84F83900134B93F89030C7
:105A4000002B5FD011481A49FDF790FE90B30E4825
:105A5000002380F8443080F82030C375037680F846
:105A6000A43080F8903080F87C3080F868302030A6
:105A70000849052201F02CFD6FF004004FF0FF31C2
:105A8000FEF75EF910BD00BF902E0020D171010815
:105A9000B02E0020289C0108A0010020D42E002058
:105AA000BD710108F82E0020200200200C2F0020DC
:105AB000202F0020234801F077FBC3B25AB2012AFD
:105AC00002DC13F0800F1BD01F48002380F8443005
:105AD00080F82030C375037680F8A43080F89030C9
:105AE00080F87C3080F8683020301849052201F0B9
:105AF000EFFC6FF005004FF0FF31FEF721F910BD0C
:105B000084F83A00104B002283F8442083F82020C8
:105B1000DA751A7683F8A42083F8902083F87C2025
:105B200083F868200A4804F1330101F04DF910BDF3
:105B30000848094940F2AA225BB201F025FC30BFB7
:105B4000FDE700BF202F0020902E0020289C010898
:105B50000038014030B30108ECB3010808B5534BDD
:105B6000DB7D13B90122514BDA75504BDB7D5AB204
:105B7000012A5DD14D4B93F82030002B45D04C4885
:105B80004C49FDF7F3FDD8B14848002380F8443074
:105B900080F82030C375037680F8A43080F8903008
:105BA00080F87C3080F8683020304349012201F0D1
:105BB0008FFC6FF004004FF0FF31FEF7C1F808BD15
:105BC0003C4801F0F1FAC0B243B2012B01DC002BDA
:105BD0001BDC3648002380F8443080F82030C37541
:105BE000037680F8A43080F8903080F87C3080F81C
:105BF000683020303049012201F06AFC6FF0050066
:105C00004FF0FF31FEF79CF808BD284B002283F8C7
:105C1000442083F82020DA751A7683F8A42083F8CC
:105C2000902083F87C2083F8682001F02BF808BDD1
:105C30005AB2022A16D11D4B002283F8442083F861
:105C40002020DA751A7683F8A42083F8902083F850
:105C50007C2083F868206FF003004FF0FF31FEF7DF
:105C60006FF808BD5AB2032A16D1104B002283F8F0
:105C7000442083F82020DA751A7683F8A42083F86C
:105C8000902083F87C2083F868206FF003004FF0A9
:105C9000FF31FEF755F808BD0848094940F23622A1
:105CA0005BB201F071FB30BFFDE700BF902E00201A
:105CB000D1710108B02E0020289C010830B30108E2
:105CC000F8B3010800B583B0634BDB7D13B9012243
:105CD000614BDA75604BDB7D5AB2012A5DD15E4BB8
:105CE00093F82030002B45D05C485D49FDF73EFD20
:105CF000D8B15948002380F8443080F82030C3756B
:105D0000037680F8A43080F8903080F87C3080F8FA
:105D1000683020305349012201F0DAFB6FF00400B3
:105D20004FF0FF31FEF70CF892E04D4801F03CFADD
:105D3000C0B243B2012B01DC002B1BDC4648002320
:105D400080F8443080F82030C375037680F8A430A2
:105D500080F8903080F87C3080F8683020304149FD
:105D6000012201F0B5FB6FF005004FF0FF31FDF7A8
:105D7000E7FF6DE0384B002283F8442083F82020B1
:105D8000DA751A7683F8A42083F8902083F87C20B3
:105D900083F8682000F020FF5AE05AB2022A16D198
:105DA0002D4B002283F8442083F82020DA751A76E0
:105DB00083F8A42083F8902083F87C2083F868205F
:105DC0006FF003004FF0FF31FDF7BAFF40E05AB229
:105DD000032A34D122486946FDF76EFCD8B11E482B
:105DE000002380F8443080F82030C375037680F8B3
:105DF000A43080F8903080F87C3080F86830203013
:105E00001849012201F064FB6FF004004FF0FF31EC
:105E1000FDF796FF1CE0104B002283F8442083F826
:105E20002020DA751A7683F8A42083F8902083F86E
:105E30007C2083F86820684600F0FEFE08E00A48EF
:105E40000A494FF409725BB201F09EFA30BFFDE7D8
:105E500003B05DF804FB00BF902E0020D171010853
:105E6000B02E0020289C010830B30108D8B10108E9
:105E700008B5544BDB7D13B90122524BDA75514BF7
:105E8000DB7D5AB2012A5FD14E4B93F82030002BB4
:105E900045D04D484D49FDF769FCD8B1494800232C
:105EA00080F8443080F82030C375037680F8A43041
:105EB00080F8903080F87C3080F868302030444999
:105EC000012201F005FB6FF004004FF0FF31FDF7F8
:105ED00037FF08BD3D4801F067F9C0B243B2062B59
:105EE00001DC002B1CDC3748002380F8443080F8AC
:105EF0002030C375037680F8A43080F8903080F8A5
:105F00007C3080F8683020303149012201F0E0FA1D
:105F10006FF005004FF0FF31FDF712FF08BDFF20C5
:105F2000284B002283F8442083F82020DA751A7663
:105F300083F8A42083F8902083F87C2083F86820DD
:105F400040B200F067FD08BD5AB2022A16D11D4BBF
:105F5000002283F8442083F82020DA751A7683F82B
:105F6000A42083F8902083F87C2083F868206FF0C9
:105F700003004FF0FF31FDF7E3FE08BD5AB2032ADC
:105F800016D1104B002283F8442083F82020DA75C4
:105F90001A7683F8A42083F8902083F87C2083F875
:105FA00068206FF003004FF0FF31FDF7C9FE08BD18
:105FB0000848094940F20B225BB201F0E5F930BF15
:105FC000FDE700BF902E0020D1710108B02E002007
:105FD000289C010830B30108A4B1010810B58CB0A9
:105FE000BA4BDB7D13B90122B84BDA75B74BDB7DB9
:105FF0005AB2012A5FD1B54B93F82030002B45D01F
:10600000B348B449FDF7B2FBD8B1B048002380F8DB
:10601000443080F82030C375037680F8A43080F8CF
:10602000903080F87C3080F868302030AA49012216
:1060300001F04EFA6FF004004FF0FF31FDF780FEE3
:10604000E3E2A44801F0B0F8C0B243B2062B01DC91
:10605000002B1CDC9D48002380F8443080F8203061
:10606000C375037680F8A43080F8903080F87C30D7
:1060700080F8683020309849012201F029FA6FF049
:1060800005004FF0FF31FDF75BFEBEE2FF208F4BB6
:10609000002283F8442083F82020DA751A7683F8EA
:1060A000A42083F8902083F87C2083F8682040B2F5
:1060B00000F076FBA9E25AB2022A40F03781834B06
:1060C00093F82030002B00F0158181488149FDF7BD
:1060D0004DFBD8B17D48002380F8443080F8203053
:1060E000C375037680F8A43080F8903080F87C3057
:1060F00080F8683020307849012201F0E9F96FF02A
:1061000004004FF0FF31FDF71BFE7EE2714801F005
:106110004BF8C4B263B2062B01DC002B1BDC6B48CE
:10612000002380F8443080F82030C375037680F86F
:10613000A43080F8903080F87C3080F868302030CF
:106140006549012201F0C4F96FF005004FF0FF31FD
:10615000FDF7F6FD59E263B2012B4BD15B4B93F88F
:1061600045309BB9594B93F844305AB25B490968A2
:106170000A44527802F00302022A5BB208BF203BB5
:10618000D8B243B2442B1DD0532B1BD04F48002311
:1061900080F8443080F82030C375037680F8A4304E
:1061A00080F8903080F87C3080F8683020304A49A0
:1061B000022201F08DF96FF004004FF0FF31FDF77E
:1061C000BFFD22E2414A002382F8443082F82030A9
:1061D000D375137682F8A43082F8903082F87C3040
:1061E00082F868300093019340B219461A4600F0D5
:1061F000B9FB0AE23A480BA9FDF718FAD8B13348BF
:10620000002380F8443080F82030C375037680F88E
:10621000A43080F8903080F87C3080F868302030EE
:106220002D49022201F054F96FF004004FF0FF31C4
:10623000FDF786FDE9E1254B002283F8442083F831
:106240002020DA751A7683F8A42083F8902083F84A
:106250007C2083F8682063B2023B042B42D8DFE83D
:1062600003F0030C151E2800002300930193184629
:106270000BA91A4600F076FBC7E1002300930193B7
:10628000184619460BAA00F06DFBBEE100220092F1
:106290000192104611460BAB00F064FBB5E10BAB6D
:1062A000009300230193184619461A4600F05AFB42
:1062B000ABE108480849022201F00AF96FF0070033
:1062C0004FF0FF31FDF73CFD9FE100BF902E002015
:1062D000D1710108B02E0020289C01082002002066
:1062E000D42E0020BA48BB4940F2D91201F04CF834
:1062F00030BFFDE7B848002380F8443080F82030F4
:10630000C375037680F8A43080F8903080F87C3034
:1063100080F868302030B149012201F0D9F86FF0DF
:1063200004004FF0FF31FDF70BFD6EE15AB2032A76
:1063300040F06281A84B93F820309BB3A64A92F8B4
:1063400021209AB95AB2A64909680A44527802F043
:106350000302022A5BB208BF203BDBB29E4A82F8EE
:1063600020305AB2442A1FD0532A1FD09A48002303
:1063700080F8443080F82030C375037680F8A4306C
:1063800080F8903080F87C3080F868302030934975
:10639000012201F09DF86FF004004FF0FF31FDF78E
:1063A000CFFC32E1002402E0012400E001248A4B0A
:1063B00093F844302BB30134E4B28A480BA9FDF7BB
:1063C00035F9D8B18448002380F8443080F8203073
:1063D000C375037680F8A43080F8903080F87C3064
:1063E00080F8683020307D49022201F071F86FF0AA
:1063F00004004FF0FF31FDF7A3FC06E10BAB069361
:1064000001E000230693744B93F868302BB30134FA
:10641000E4B2754802A9FDF709F9D8B16E48002326
:1064200080F8443080F82030C375037680F8A430BB
:1064300080F8903080F87C3080F8683020306749F0
:10644000032201F045F86FF004004FF0FF31FDF733
:1064500077FCDAE002AB079301E0002307935E4B81
:1064600093F87C302BB30134E4B2604803A9FDF704
:10647000DDF8D8B15848002380F8443080F8203047
:10648000C375037680F8A43080F8903080F87C30B3
:1064900080F8683020305149042201F019F86FF07B
:1064A00004004FF0FF31FDF74BFCAEE003AB089367
:1064B00001E000230893484B93F890302BB301344C
:1064C000E4B24B4804A9FDF7B1F8D8B14248002323
:1064D00080F8443080F82030C375037680F8A4300B
:1064E00080F8903080F87C3080F8683020303B496C
:1064F000052200F0EDFF6FF004004FF0FF31FDF7D3
:106500001FFC82E004AB099301E000230993324BA6
:1065100093F8A4302BB30134E4B2364805A9FDF753
:1065200085F8D8B12C48002380F8443080F820301A
:10653000C375037680F8A43080F8903080F87C3002
:1065400080F8683020302549062200F0C1FF6FF046
:1065500004004FF0FF31FDF7F3FB56E005AB0A9363
:1065600001E000230A93B4B91B4B002283F84420B6
:1065700083F82020DA751A7683F8A42083F8902017
:1065800083F87C2083F868206FF007004FF0FF311C
:10659000FDF7D6FB39E0104B93F82000002283F87A
:1065A000442083F82020DA751A7683F8A42083F833
:1065B000902083F87C2083F86820099B00930A9B35
:1065C000019340B20699079A089B00F0CBF91CE0B2
:1065D00058B30108CCB10108902E0020289C010876
:1065E00020020020D42E0020F82E00200C2F0020A6
:1065F000202F0020342F0020054806494FF4FC725C
:106600005BB200F0C1FE30BFFDE70CB010BD00BFB3
:1066100030B30108CCB1010870B50024144D154EFB
:106620000AE0304600F092FF28B9114B03EB041446
:106630006368984770BD01342301E9580029F0D1FF
:106640000D4B002283F8442083F82020DA751A7657
:1066500083F8A42083F8902083F87C2083F86820B6
:106660006FF002004FF0FF31FDF76AFB70BD00BF15
:10667000F4B00108A82E0020902E002000B583B0B1
:106680000DF107000121FAF7E7FF002878DD9DF8FA
:1066900007305AB23C4909680A44527812F0170F81
:1066A00037D15BB20A2B04D01B2B28D0082B3FD14B
:1066B00012E0364B93F8CE3043B13548354B19785C
:1066C000FAF7D6FF34480221FAF7D2FF314B1B7894
:1066D00000212F4AD1542BE02E4B1B7843B3013BB2
:1066E000DBB22C4A13700021294AD154274B93F86E
:1066F000CE30EBB129480321FAF7BAFF18E0234B5B
:1067000093F8CE30A3B10DF107000121FAF7B0FFE5
:106710000EE0204B1B78622B0AD80BB9FAF7BCFFAE
:106720001C4A1378591C11709DF80710184AD1544F
:106730009DF907300A2B23D1164B187800B3FDF7CB
:106740004FF80023134A1370104A82F8443082F83D
:106750002030D375137682F8A43082F8903082F816
:106760007C3082F868300A48FDF7FAF810B9FFF774
:1067700053FF05E0022803D04FF0FF31FDF7E0FAA8
:1067800003B05DF804FB00BF20020020902E002023
:10679000B81200201C1300207C92010880B301086D
:1067A00030B589B004460023029303930493059304
:1067B0000693ADF81C308DF81E30012002A9F6F7C3
:1067C0000DFD012C13D19DF81E30022B604861494C
:1067D0000CBF4422532200F07BFE00204FF0FF311B
:1067E000FDF7AEFA00225C4B83F82020AEE0012CCE
:1067F00054DD023C042C47D8DFE804F003122130BA
:106800003F009DF80E209DF80F309DF810009DF878
:106810001110009001914E48504900F059FE33E0AC
:106820009DF812209DF813309DF814009DF8151066
:10683000009001914648494900F04AFE24E09DF845
:1068400016209DF817309DF818009DF8191000903B
:1068500001913F48414900F03BFE15E09DF81A20A8
:106860009DF81B309DF81C009DF81D1000900191B3
:1068700037483A4900F02CFE06E06FF007004FF071
:10688000FF31FDF75DFA61E000204FF0FF31FDF7C9
:1068900057FA0022304B83F8202057E09DF81E3035
:1068A000022B2B482B490CBF4422532200F010FE30
:1068B0009DF80E209DF80F309DF810009DF81110E6
:1068C000274C264D009001912046294600F000FEFD
:1068D0009DF812209DF813309DF814009DF81510B6
:1068E0000090019104F12400294600F0F1FD9DF88B
:1068F00016209DF817309DF818009DF8191000908B
:10690000019104F13800294600F0E2FD9DF81A20BB
:106910009DF81B309DF81C009DF81D100090019102
:1069200004F14C00294600F0D3FD00204FF0FF3168
:10693000FDF706FA002304F8243C443C84F8443074
:1069400084F8683084F87C3084F8903009B030BD29
:10695000B02E002004B40108902E002008B40108D5
:10696000D42E00202DE9F04387B081468846174693
:106970001E460E9D002400940194029403940494F6
:10698000ADF814408DF816406846FCF72BF9B8F1C5
:10699000000F03D0D8F80030CDF8063017B13B68AF
:1069A000CDF80A3016B13368CDF80E3015B12B682A
:1069B000CDF812300F9B83B1144C204614490622A7
:1069C00000F086FD6FF007004FF0FF31FDF7B8F9DA
:1069D000203C002384F8203015E0B9F1530F04BFA8
:1069E00001238DF81630B9F1440F04BF02238DF84E
:1069F00016306846FCF7C6F8FCF776F900204FF031
:106A0000FF31FDF79DF907B0BDE8F083B02E0020FF
:106A1000289C010830B589B00446002302930393F3
:106A2000049305930693ADF81C308DF81E300120B9
:106A300002A9F6F7D3FB012C13D19DF81E30022BCF
:106A4000604861490CBF4422532200F041FD002000
:106A50004FF0FF31FDF774F900225C4B83F82020E2
:106A6000AEE0012C54DD023C042C47D8DFE804F0F2
:106A7000031221303F009DF80E209DF80F309DF845
:106A800010009DF81110009001914E48504900F0FF
:106A90001FFD33E09DF812209DF813309DF814007F
:106AA0009DF81510009001914648494900F010FDED
:106AB00024E09DF816209DF817309DF818009DF8E9
:106AC0001910009001913F48414900F001FD15E087
:106AD0009DF81A209DF81B309DF81C009DF81D1094
:106AE0000090019137483A4900F0F2FC06E06FF05F
:106AF00007004FF0FF31FDF723F961E000204FF070
:106B0000FF31FDF71DF90022304B83F8202057E0BC
:106B10009DF81E30022B2B482B490CBF44225322D8
:106B200000F0D6FC9DF80E209DF80F309DF8100067
:106B30009DF81110274C264D0090019120462946C2
:106B400000F0C6FC9DF812209DF813309DF814004B
:106B50009DF815100090019104F12400294600F0E1
:106B6000B7FC9DF816209DF817309DF818009DF889
:106B700019100090019104F13800294600F0A8FC9A
:106B80009DF81A209DF81B309DF81C009DF81D10E3
:106B90000090019104F14C00294600F099FC00207E
:106BA0004FF0FF31FDF7CCF8002304F8243C443CBF
:106BB00084F8443084F8683084F87C3084F890306D
:106BC00009B030BDB02E002004B40108902E002082
:106BD00008B40108D42E002070B58AB000240494B3
:106BE0000594069407940894ADF824408DF8264047
:106BF000012004A9F6F7F2FA9DF810209DF8113053
:106C00009DF812609DF813509DF814009DF8151022
:106C100000960195029003910548064900F058FC42
:106C200020464FF0FF31FDF78BF80AB070BD00BF72
:106C3000B02E002014B4010830B587B005460024FA
:106C400000940194029403940494ADF814408DF8D8
:106C50001640FCF781F8FBF783FF01206946F6F741
:106C6000BDFA28680090AB88ADF80430204669462C
:106C7000F6F7B4FA20464FF0FF31FDF761F807B0A0
:106C800030BD00BF10B582B0094C012300932046EF
:106C900008491A4600F01CFC00204FF0FF31FDF7B8
:106CA0004FF8203C002384F8203002B010BD00BF14
:106CB000B02E002034B4010870B50C463B4B98420E
:106CC00004D1FBF7ABFE00F1330503E0FBF7A6FEB2
:106CD00000F13B05002C37DD013C042C24D8DFE813
:106CE00004F003090F171D00314832492A6800F0EB
:106CF000EFFB1FE02E4830492A7900F0E9FB19E04C
:106D00006B792B482D492E4AD25600F0E1FB11E059
:106D100027482949AA7900F0DBFB0BE024482649E3
:106D2000EA7900F0D5FB05E06FF007004FF0FF3186
:106D3000FDF706F800204FF0FF31FDF701F80022C3
:106D4000204B83F8202070BD194C204619492A6831
:106D500000F0BEFB184E04F1240031462A7900F001
:106D6000B7FB6B7904F148001449154AD25600F07C
:106D7000AFFB04F15C003146AA7900F0A9FB04F1F5
:106D800070003146EA7900F0A3FB00204FF0FF319C
:106D9000FCF7D6FF002304F8203984F8443084F847
:106DA000683084F87C3084F8903070BD0038014041
:106DB000B02E0020608E0108289C010804B4010850
:106DC000F0010020902E002038B505460C4600202A
:106DD0004FF0FF31FCF7B4FFFAF756FC0028FBD167
:106DE0000348F1F7ADFE28462146FAF7C5FA38BD4B
:106DF0003F420F0008B5FBF7B3FE05484FF4DB71C7
:106E0000FAF764FC00204FF0FF31FCF799FF08BD52
:106E1000D428002008B5013840B2B1F1FF3F0BD1B2
:106E20000B4B18448278531E012B0A480A4988BF2D
:106E3000002200F04DFB05E0054B03449970C0B201
:106E4000F9F7DEFD00204FF0FF31FCF779FF08BDB8
:106E5000D4280020B02E0020289C010808B5013855
:106E600040B2B1F1FF3F08D1C0B2F9F71FFE0246B0
:106E70001048114900F02CFB16E0104B03449B789E
:106E8000022B0BD10D4B0344997419B1C0B2F9F721
:106E9000E1FD09E0C0B2F9F7F3FD05E06FF007008E
:106EA0004FF0FF31FCF74CFF00204FF0FF31FCF7B3
:106EB00047FF08BDB02E0020289C0108D4280020E0
:106EC000BFF34F8F044AD16801F4E061034B0B43D9
:106ED000D360BFF34F8FFEE700ED00E00400FA053A
:106EE00010B582B004460023019300931B4800F0C4
:106EF000D7FA1B4800F048FA631E042B18D8DFE8C5
:106F000003F003070B0F1300164800F0C9FA12E054
:106F1000154800F0C5FA0EE0144800F0C1FA0AE086
:106F2000134800F0BDFA06E0124800F0B9FA02E09A
:106F3000114800F0B5FA204601A96A46F9F7DAFDD2
:106F4000019C009B0D4819462246E31A00F01CFAEA
:106F5000094800F0A5FA02B010BD00BF40B4010816
:106F60005CB4010868B4010870B4010874B4010885
:106F70007CB4010884B4010824B601088CB401086B
:106F8000F0B589B0FBF74AFD0646F9F727FEF1F7A1
:106F900061FDFAF7DBF80020F1F780FD0120F1F741
:106FA0007DFD0020F1F7ACFD0120F1F7A9FD0023E4
:106FB0005D4A13605D4A1360F9F7E6FCFBF7B2FD2A
:106FC000FAF74CFAFAF7E2FAF9F7C0FFFAF726F8FF
:106FD000F9F706FC564800F063FA564800F060FAEC
:106FE000554800F05DFA554801210A460B4600F06D
:106FF000CBF9534800F054FA5248711D00F0C4F91F
:1070000096F84D308BB3504800F04AFA01204F49B2
:10701000F4F7F0FE4E4908464E4AF4F7BDF9002455
:107020004D4F2546F4F702FE042806D1F4F778FF09
:1070300001464A4800F0A8F919E038B90134E4B231
:10704000032C03D83846214600F09EF9032C08D9BA
:10705000434800F025FA002386F84D30FBF744FE44
:1070600005E02846FCF77AFADCE7FBF73DFEFBF784
:10707000E7FDF9F78BFD044628B10120F1F730FD5B
:107080002046FFF72DFFF9F761FD044610B935489A
:1070900000F006FA2CB10020F1F722FD2046FFF7A0
:1070A0001FFFFCF721FE294C20462F4903222F4BBE
:1070B000F3F782F92E482F49F3F78CF9FAF716FB0C
:1070C000012002A9F6F78AF80DF10E00F3F73CFB58
:1070D000F1F7CEFC072300932748284942F2FA0231
:1070E0002346F6F7DFF80025254FF0F779F9284613
:1070F000FCF734FAFFF7C2FA96F84D300BB1F4F70B
:1071000095FDF1F793FD2C4604E02046F3F76EF968
:107110000134E4B2022CF8D93846F3F7D7FEF0F781
:107120005FF9F6F7A7FCE0E7301300201803002012
:10713000CCB40108F8B4010818B5010838B5010845
:1071400058B5010884B501089CB50108683D0020C8
:1071500059DD0008E9DD0008E8B50108B4B501080B
:1071600014B6010828B6010868350020F80100208F
:10717000C16E0108E1730008FC010020F401002049
:1071800068330020704700BFFEE700BFFEE700BF86
:10719000FEE700BFFEE700BF704700BF704700BFBB
:1071A000704700BF704700BF00210A2200F01CBBDF
:1071B000014B1868704700BF84020020034B1B6816
:1071C0001844407800F00300704700BF2002002000
:1071D000034B1B681844407800F00400704700BF60
:1071E00020020020034B1B681844407800F0440044
:1071F000704700BF20020020024B0146186800F0D3
:107200006FB800BF84020020024B0146186800F0EE
:1072100023B800BF8402002030B50023934208D079
:10722000C55C0133CC1814F8014CA542F6D0281BDC
:1072300030BD002030BD10B50023934203D0CC5C9C
:10724000C4540133F9E710BD02440346934202D00F
:1072500003F8011BFAE7704730B500293CD051F81C
:10726000042C0B1F1D49002AB8BF9B180A680C4646
:1072700012B95A600B6030BD93420DD2196858188C
:10728000904203D15A581144426819605A602360F1
:1072900030BD994203D80A4651680029F9D11468D3
:1072A00015199D420AD11B682344D01888421360E7
:1072B00012D10868034413604B680CE002D90C2318
:1072C000036030BD18681C188C4203D10C684968F3
:1072D000204418605960536030BD00BF381300204F
:1072E00070B5CD1C25F0030508350C2D38BF0C25D5
:1072F000002D06463FDB8D423DD3214B1C681846CE
:107300002146A1B10B685B1B0ED40B2B03D90B607C
:10731000CC18CD501FE08C4202D1626802601AE0A6
:107320004B6863600C4616E00C464968E9E7154C6B
:1073300023681BB9304600F0BBF820602946304670
:1073400000F0B6F8431C014615D0C41C24F0030419
:1073500084420AD1256004F10B00231D20F00700B0
:10736000C31A0BD05A42E25070BD3046611A00F089
:107370009FF80130EED10C233360002070BD00BFB8
:1073800038130020341300200FB40A4B13B51C68C7
:1073900024B1A36913B9204601F02CF805AB2046AF
:1073A000A168049A019300F09DFB02B0BDE8104073
:1073B00004B070478402002038B5084B05461C68AD
:1073C00024B1A36913B9204601F014F820462946D8
:1073D000A268BDE8384001F013B900BF8402002064
:1073E00070B50E46054618B183690BB901F002F875
:1073F000AC68A389190701D5236983B928462146BA
:1074000000F088FE58B14FF0FF3070BD002B0EDB4E
:10741000236816F8012C1A70236801332360A368CF
:1074200016F8012B013BA360002AEFD117E0A269F7
:10743000934209DB236816F8012C1A702368197827
:107440000A29EAD1284602E016F8011C28462246FD
:1074500000F00CFEB0F1FF3250425041D2E7002B59
:1074600016DAA269934208DB23680A221A7023689D
:107470001978914210D1284601E028460A21224677
:1074800000F0F4FDB0F1FF335842584130B1BAE793
:1074900023680A221A702368013323600A2070BD12
:1074A000024B01461868FFF79BBF00BF8402002013
:1074B00038B5064C0023054608462360F1F796F9D7
:1074C000431C02D1236803B12B6038BD3C1300205C
:1074D0000EB400B54FF402719CB0ADF814106FF00B
:1074E0000041049107914FF6FF711DABADF81610E6
:1074F000084953F8042B02900690086802A90193EA
:1075000000F0DCF9029B00221A701CB05DF804EB5D
:1075100003B070478402002010B504462246137859
:107520000134002BFAD1CC5CD4540133002CFAD1B5
:1075300010BDC9B2024610F8013B1BB18B42F9D114
:10754000104670470029FBD01846704710F8012BF1
:1075500011F8013B012A28BF9A42F7D0D01A704790
:10756000034611F8012B03F8012B002AF9D17047CB
:10757000034613F8012B002AFBD1181A0138704773
:1075800070B58AB10B4605461C7810F8016B0131C5
:10759000B44201D1012A03D128781B78C01A70BDEA
:1075A000013A002CEED1F7E7104670BD10B5034646
:1075B00032B111F8014B013A03F8014B002CF7D11D
:1075C0001A44934203D0002103F8011BF9E710BDD0
:1075D00038B502460D4641B1002410462946FFF752
:1075E000A8FF30B1421C0446F7E7BDE83840FFF77A
:1075F000A0BF204638BD30B503780BB1044604E087
:107600000B78002B18BF002030BD224610780134C3
:1076100038B10023C85C28B1D55C8542F5D101336F
:10762000F8E730BD104630BD174B2DE9F0411D681D
:107630000646AC6D0F46FCB95020FFF7DDFDA8658E
:107640008460AB6D046044601C61DC60AB6D9C6168
:107650005C61AB6DDC629C62AB6D5C631C63AB6DAB
:10766000DC639C63AB6D5C641C64AB6DDC649C642C
:10767000AB6D1C77AB6D5C6230463946AA6D012359
:10768000BDE8F04100F002B884020020F0B508B96E
:10769000106828B3044614F8015B0F4617F8016B15
:1076A0003EB1B542FAD10BB12046F3E71460037046
:1076B000F0BD4DB915602846F0BD17F8016BAE421C
:1076C00007D0002EF9D11C46234613F8015B0F4664
:1076D000F3E715B10021217000E02B461360F0BDE7
:1076E000F0BD000084463F482DE9F04FD0F80080FF
:1076F0000E46344614F8015B08EB0500407800F0B4
:10770000080000F0FF0708B12646F2E72D2D03D14F
:10771000B41C7578012703E02B2D04BF7578B41CC9
:1077200033F010000DD1302D08D1207800F0DF00AB
:10773000582851D165781023023402E0002B08BF8D
:107740000A23002F0CBF6FF0004A4FF0004ABAFB2B
:10775000F3F903FB19AA0026304608EB050B9BF84A
:1077600001B01BF0040F01D0303D0BE01BF0030B08
:107770001BD0BBF1010F14BF4FF0570B4FF0370B6D
:10778000CBEB05059D4210DAB6F1FF3F0AD0484524
:1077900006D801D1554503DC03FB0050012601E06A
:1077A0004FF0FF3614F8015BD7E7731C0CD1002FA4
:1077B0004FF022030CBF6FF000404FF00040CCF8B8
:1077C00000302AB9BDE8F08F07B1404242B106B19E
:1077D000611E1160BDE8F08F002B08BF0823B0E7E1
:1077E000BDE8F08F2002002030B51346044A05465C
:1077F0000C46106829462246BDE83040FFF772BFAC
:10780000840200202DE9F0478D688146AB420C468A
:1078100092461F4643D38B8913F4906F3DD0266860
:1078200009690222C1EB0608666906EB460696FB6B
:10783000F2F608F101023A44964238BF16465B055B
:107840000FD53146FFF74CFD054698B121694246F8
:10785000FFF7F1FCA38923F4906343F08003A38135
:1078600013E0324600F0A5FE054670B9484621698E
:10787000FFF7F2FC0C23C9F80030A3894FF0FF306A
:1078800043F04003A381BDE8F0872561666145446C
:10789000C8EB06062560A6603D46AF4200D23D46D5
:1078A0002A462068514600F069FEA36800205B1B51
:1078B000A36023681D442560BDE8F0872DE9F043EF
:1078C0009DB003938B8907461C060D4616460CD5C2
:1078D0000B6953B94021FFF703FD2860286110B9F7
:1078E0000C233B60C7E040236B61002309932023F6
:1078F0008DF8293030238DF82A3033461C4613F892
:10790000012B1AB9B4EB06090FD002E0252AF5D1F4
:10791000F8E73846294632464B46FFF773FF0130F9
:1079200000F0A480099B4B4409932378002B00F0BE
:107930009D8000234FF0FF32049307930592069336
:107940008DF853301A9304F101094D4E4C463046E0
:107950002178052200F004FE09F10109049B28B1F9
:10796000861B0120B04003430493EEE7D90644BFD1
:1079700020228DF853201A0744BF2B228DF8532064
:1079800022782A2A02D0079B21460EE0039A111D75
:1079900012680391002A01DB079204E0524243F08F
:1079A00002030792049301340AE00C462278013165
:1079B000303A092A03D80A2000FB0323F5E707938E
:1079C00023782E2B19D163782A2B09D1039B0234FB
:1079D0001A1D1B680392002BB8BF4FF0FF330BE05A
:1079E000611C00230C4622780131303A092A03D861
:1079F0000A2000FB0323F5E70593224E2178304649
:107A0000032200F0ADFD30B1861B4020B040049B46
:107A100001340343049321781B480622661C8DF829
:107A2000281000F09DFD88B1184B33B9039B073334
:107A300023F007030833039314E003AB00933846A5
:107A400004A92A46124BAFF3008007E003AB009372
:107A5000384604A92A460E4B00F0BAF9B0F1FF3FB0
:107A6000804603D0099B4344099346E7AB895B06F4
:107A700001D4099801E04FF0FF301DB0BDE8F0835C
:107A80007CB7010882B7010886B701080000000032
:107A900005780108936810B5013B002B936005DA67
:107AA0009469A34208DBCBB20A2B05D01368581C9B
:107AB00010601970C8B210BDBDE8104000F0D6BA11
:107AC000F8B505460E461446D718BC4208D02846DD
:107AD00014F8011B3246FFF7DDFF431CF5D100E02F
:107AE0000020F8BD2DE9F0439DB00D4617460393E5
:107AF000064618B183690BB900F07CFC734B9D42BC
:107B000001D1756808E0724B9D4201D1B56803E070
:107B1000704B9D4208BFF568AB8918070AD52B69E1
:107B200043B10023099320238DF8293030238DF8A9
:107B30002A3038E03046294600F0ECFA0028F0D030
:107B40004FF0FF30BEE0039A111D12680391002A26
:107B500070DB0792013423782E2B7DD05E4F217885
:107B60003846032200F0FCFC30B1C71B4020B8406F
:107B7000049B013403430493217858480622671C70
:107B80008DF8281000F0ECFC002800F08980544BA0
:107B9000002B7CD1039B073323F0070308330393A7
:107BA000099B434409933B461C4613F8012B1AB921
:107BB000B4EB07090ED002E0252AF5D1F8E73046EC
:107BC00029463A464B46FFF77BFF013075D0099BAB
:107BD0004B4409932378002B6FD000234FF0FF32E2
:107BE00004930793059206938DF853301A9304F18A
:107BF00001093C4F4C4638462178052200F0B0FC84
